:10000000544649530001000064E80100CDCAAD4BDD
:100010000511012316052017483241300511015200
:100020001605201748324130051101061605171430
:1000300048324130030000000000000000000000D2
:10004000544643530020000014D801000000000073
:10005000004001200121000025210000272100008F
:10006000292100002B2100002D2100003D2100004E
:100070003D2100003D2100003D2100002F21000016
:10008000312100003D210000332100007B5700009A
:100090007B580000372100003D210000BD07001003
:1000A000372100007D390000D13900003D210000DA
:1000B0003D2100004F54000037210000372100008F
:1000C00043510000372100003D2100003D21000088
:1000D0000000000000000000000000000000000020
:1000E0000000000000000000000000000000000010
:1000F0000000000000000000000000000000000000
:1001000000000000000000000000000000000000EF
:1001100000000000000000000000000000000000DF
:1001200000000000000000000000000000000000CF
:1001300000000000000000000000000000000000BF
:1001400000000000000000000000000000000000AF
:1001500000F003F800F020F8FEE70D48016821F0F8
:100160000301002001C101C101C101C170470000AC
:10017000940D0010FEE7FEE7FEE7FEE7FEE7FEE770
:10018000FEE7FEE7FEE703480047FEE7FEE7000064
:10019000202100003D21000000F002F800F068F886
:1001A0000AA090E8000C82448344AAF10107DA45D2
:1001B00001D100F05DF8AFF2090EBAE80F0013F0BC
:1001C000010F18BFFB1A43F00103184748C801008C
:1001D00078C801000A444FF0000C10F8013B13F0FE
:1001E000070408BF10F8014B1D1108BF10F8015B90
:1001F000641E05D010F8016B641E01F8016BF9D183
:1002000013F0080F1EBF10F8014BAD1C0C1B09D1D9
:100210006D1E58BF01F801CBFAD505E014F8016B4B
:1002200001F8016B6D1EF9D59142D6D370470000DD
:10023000103A24BF78C878C1FAD8520724BF30C812
:1002400030C144BF04680C607047000000230024E4
:1002500000250026103A28BF78C1FBD8520728BFD6
:1002600030C148BF0B6070471FB51FBD10B510BD32
:10027000DFF80CD0FFF7F8FF05F00CF91AF027FAB9
:100280000040012003B4FFF7F1FF03BC1AF026FA87
:1002900008B5002103200B460A46009119F0ACFB7B
:1002A00008BD38B5AF4D0024AC80EC8019F081FB5F
:1002B000E860FF206870AC48234622460460446032
:1002C00004720120A87003202146009419F094FBC9
:1002D000012038BD38B5A34D02286C7822460DD0D8
:1002E000052814D0A24208BF38BD002003460246AC
:1002F0002146009019F080FB6C7038BD022908BFC0
:100300000224EFD00D2914BF01240024EAE70229BA
:1003100014BF64246524E5E738B5944B944C0A4631
:100320001B7824784FF0010C6343002401465B00E6
:100330006046009419F060FB38BD38B54FF0010CF1
:10034000062400250B46024621466046009519F01A
:1003500053FB38BD2DE9F04104460127002503F089
:100360000700804E8846012804BF0020F08046D058
:10037000022844D1F08804280BD2002818BFB068A6
:1003800002D119F05AFBB06010F8011B2170B06067
:100390002EE0062808D219F052FBF188C1F10501C0
:1003A000C900C840207023E0082808D219F04BFB90
:1003B000F188C1F10701C900C840207018E00C287D
:1003C00008D219F0F6FAF188C1F10B01C900C84052
:1003D00020700DE00E2808D219F0EDFAF188C1F175
:1003E0000D01C900C840207002E0FF2020700027E6
:1003F000F088401C80B2F0800E2828BF012588F8C4
:1004000000503846BDE8F08130B403F00700002406
:10041000DFF850C1012804BFACF80440ACF8064036
:1004200014D05048BCF806308088022B05D2120246
:1004300042EA1020ACF8040005E0DCF80C50184447
:10044000284400F8022C581CACF806000C7030BC94
:100450000020704770B40546002003F0070C414CA3
:100460000646BCF1010F08BFE68008D03D4BBCF149
:10047000020F9B8806D0120242EA1322A2800E705D
:1004800070BC7047E0881A18E368401C9A5C2A70B8
:10049000E0800120F3E738B503F0070000240D46A3
:1004A000012809D12F4821460B46C48084800220B0
:1004B0000A46009419F0A0FA2C70002038BD2A4A90
:1004C0001154704700225A2101200BF0F8BD002280
:1004D0005B2101200BF0F3BD00284FF0000001D09C
:1004E0000CF029B90CF033B91E4900200870704790
:1004F0001C48007870471B49012008707047194953
:10050000002818BF01208870704708B5B9B10023D2
:100510000221012808BF8DF8001017D0022808BF5B
:100520008DF8001015D00522642808BF8DF8002032
:100530000CD0652808BF8DF800200AD00BE0012000
:100540000CF0D0F8012009F0FFF808BD8DF801305B
:1005500001E08DF80110684608F089F908BD0148EE
:100560008078704700400020C84200209E40002054
:100570009F4000207047002818BF0120FE490968ED
:1005800008627047FC480068006A002818BF012014
:100590007047F94A126802EBC00041637047F649A0
:1005A000096801EBC000006B00F480707047F24AEC
:1005B0001021126802EBC00041637047EE490A68DF
:1005C000D2F8402160F30D220868C0F8402170473E
:1005D000E9480068D0F84001C0F305207047E64ABA
:1005E00000F00F03C0F303101268002902EBC312DE
:1005F00002EB4010D0F8401114BF41F0010121F08E
:100600000101C0F840117047DB4A00F00F01C0F350
:100610000310126802EBC11101EB4010D0F8400149
:1006200000F001007047D44900230A681362026891
:10063000D1F800C0CCF800204268D1F800C0CCF856
:1006400004208268D1F800C0CCF80820C268D1F834
:1006500000C0CCF80C20426AD1F800C0CCF8402091
:10066000826AD1F800C0CCF844200269D1F800C0F9
:10067000CCF818204269D1F800C0CCF81C20826B5D
:10068000D1F800C0CCF86020C26BD1F800C0CCF823
:100690007020026CD1F800C0CCF87420426CD1F804
:1006A00000C0CCF87820826CD1F800C0CCF8802053
:1006B000C26CD1F800C0CCF88420026DD1F800C023
:1006C000CCF88820426DD1F800C0CCF88C20426E66
:1006D000D1F800C0CCF89C20826ED1F800C0CCF8D4
:1006E000A020C26ED1F800C0CCF8A420026FD1F8CF
:1006F00000C0CCF8A820826FD1F800C0CCF8C02090
:10070000C26FD1F800C0CCF8C420D0F88020D1F856
:1007100000C0CCF8C820D0F88420D1F800C0CCF8B4
:10072000CC20D0F88820D1F800C0CCF8D020D0F868
:100730008C20D1F800C0CCF8D420D0F89420D1F887
:1007400000C0CCF8DC20D0F89C20D1F800C0CCF858
:10075000F020D0F8A020D1F800C0CCF8F420D0F8D8
:10076000A420D1F800C0CCF8F820D0F8A820D1F807
:1007700000C0CCF8FC20D0F8AC20D1F800C0CCF8F8
:100780000021D0F8B020D1F800C0CCF80421D0F876
:10079000B420D1F800C0CCF80821D0F8B820D1F8A6
:1007A00000C0CCF80C21D0F8BC20D1F800C0CCF8A7
:1007B0001021D0F8C020D1F800C0CCF81421D0F816
:1007C000C420D1F800C0CCF81821D0F8C820D1F846
:1007D00000C0CCF81C21D0F8CC20D1F800C0CCF857
:1007E0002021D0F8D020D1F800C0CCF82421D0F8B6
:1007F000D420D1F800C0CCF83021D0F8D820D1F8DE
:1008000000C0CCF84021D0F8DC20D1F800C0CCF8F2
:100810004421D0F8E020D1F800C0CCF84821D0F82D
:10082000E420D1F800C0CCF84C21D0F8E820D1F871
:1008300000C0CCF85021D0F8EC20D1F800C0CCF8A2
:100840005421D0F8F020D1F800C0CCF85821D0F8CD
:10085000F420D1F800C0CCF85C21D0F81821D1F8F0
:1008600000C0CCF88021D0F81C21D1F800C0CCF811
:100870008421D0F82021D1F800C0CCF88821D0F80C
:100880002421D1F800C0CCF88C21D0F82821D1F84F
:1008900000C0CCF89021D0F82C21D1F800C0CCF8C1
:1008A0009421D0F83021D1F800C0CCF89821D0F8AC
:1008B0003421D1F800C0CCF89C21D0F83821D1F8EF
:1008C00000C0CCF8A021D0F83C21D1F800C0CCF871
:1008D000A421D0F84021D1F800C0CCF8B021D0F844
:1008E0004421D1F800C0CCF8C021D0F84821D1F87B
:1008F00000C0CCF8C421D0F84C21D1F800C0CCF80D
:10090000C821D0F85021D1F800C0CCF8CC21D0F8C3
:100910005421D1F800C0CCF8D021D0F85821D1F81A
:1009200000C0CCF8D421D0F85C21D1F800C0CCF8BC
:10093000D821D0F86021D1F800C0CCF8DC21D0F863
:100940006421D1F800C0CCF8E021D0F86821D1F8BA
:1009500000C0CCF8E421D0F86C21D1F800C0CCF86C
:10096000E821D0F87021D1F800C0CCF8EC21D0F803
:100970007421D1F800C001E038E30100CCF8F02187
:10098000D0F87821D1F800C0CCF8F421D0F87C213F
:10099000D1F800C0CCF8F821D0F88021D1F800C0FF
:1009A000CCF8FC21D1F800C02122CCF83420D1F8B9
:1009B00000C0CCF83C20C269D1F800C0CCF824209B
:1009C000C26AD1F800C0CCF84820026BD1F800C050
:1009D000CCF84C20426FD1F800C0CCF8AC20D0F855
:1009E0009820D1F800C0CCF8E020D0F88421D1F8CC
:1009F00000C0CCF80022D0F88821D1F800C0CCF893
:100A00000422D0F88C21D1F800C0CCF80822D0F80C
:100A10009021D1F800C0CCF80C22D0F89421D1F864
:100A200000C0CCF81022D0F89821D1F800C0CCF842
:100A30001422D0F89C21D1F800C0CCF81822D0F8AC
:100A4000A021D1F800C0CCF81C22D0F8A421D1F804
:100A500000C0CCF82022D0F8A821D1F800C0CCF8F2
:100A60002422D0F8AC21D1F800C0CCF83022D0F844
:100A7000B021D1F800C0CCF84022D0F8B421D1F890
:100A800000C0CCF84422D0F8B821D1F800C0CCF88E
:100A90004822D0F8BC21D1F800C0CCF84C22D0F8C4
:100AA000C021D1F800C0CCF85022D0F8C421D1F830
:100AB00000C0CCF85422D0F8C821D1F800C0CCF83E
:100AC0005822D0F8CC21D1F800C0CCF85C22D0F864
:100AD000D021D1F800C0CCF86022D0F8D421D1F8D0
:100AE00000C0CCF86422D0F8D821D1F800C0CCF8EE
:100AF0006822D0F8DC21D1F800C0CCF86C22D0F804
:100B0000E021D1F800C0CCF87022D0F8E421D1F86F
:100B100000C0CCF87422D0F8E821D1F800C0CCF89D
:100B20007822D0F8EC21D1F800C0CCF87C22FA4A27
:100B3000126832F0FF0C08D1D1F800C0DCF890C088
:100B400062F3030C0A68C2F890C0F44A1370836F12
:100B500013F0010F1CBF02231370D0F8880010F0AF
:100B6000010F03D0107840F0010010700868D0F831
:100B7000C0000A6820F00100C2F8C0000868D0F880
:100B8000D000096820F00100C1F8D0007047E349A7
:100B900008707047E2480068D0F8C00000F001001B
:100BA0007047DF480068C068704770B5DC4D044688
:100BB0002868D0F8400114F0020F20F00D0118BF92
:100BC00041F0010114F0080F18BF41F0040114F0C6
:100BD000040F18BF41F008012868C0F8401114F054
:100BE000010F70D001F075F8064601F075F8014666
:100BF0002868C06800280EBF3046084631460028E5
:100C00002868D0F8C00114BF40F0010020F00100B6
:100C10002A68C2F8C00128680029D0F8E00114BF92
:100C200040F0010020F001002968C1F8E001BB4854
:100C300090F800C01CF0010F5DD0BA480168496C03
:100C4000026841F4803151640168896CC1F3090282
:100C500040F2E73103689B6CC3F30903934202D16E
:100C6000491EF7D117E0B1B11CF0010F07D0286879
:100C7000D0F8D000296840F00100C1F8D0001CF085
:100C8000020F38D02868D0F8C000296840F0010071
:100C9000C1F8C0002FE02968D1F8D0102A6821F0EF
:100CA0000101C2F8D0102968D1F8C0102A6821F0DB
:100CB0000101C2F8C0100168496C006821F480315C
:100CC000416418E0FFE72868D0F8C001296820F0E7
:100CD0000100C1F8C0012868D0F8E001296820F0BF
:100CE0000100C1F8E0012868D0F8C000296820F0B0
:100CF0000100C1F8C00014F0200F18BF002413D069
:100D0000204600F0F0FF0028286800EB4410D0F8DF
:100D1000401214BF41F0010121F00101C0F840125E
:100D2000641C022CECD370BD2868D0F840022968FE
:100D300020F00100C1F840022868D0F8600229685C
:100D400020F00100C1F8600270BD2DE9F003744984
:100D5000024602F00F03D1F800C000200CEBC315CF
:100D6000C2F3031305EB4313D3F8403113F0010F23
:100D70000DD142F01003C3F3031305EB4313D3F873
:100D8000403113F0010F04BFBDE8F00370470CEBD6
:100D9000C214D4F81C31DCF81C10C3F3080901F0AC
:100DA0000807D4F80011C1F30A08002142EA011330
:100DB000C3F3031305EB4313D3F8403113F0010FD2
:100DC00014D004EB4113D3F844C1CCF3080617F157
:100DD000000C1CBFD3F844C1CCF3023CD3F8403123
:100DE00006FA0CFCC3F3054360441844491C02296D
:100DF000DCD300FB08F0C9EB0911BDE8F00300EB00
:100E00004100704770B5464801680968006801F004
:100E10001F064068C0F30C050120FFF796FF04464B
:100E20000220FFF792FF044400F078FB211805FB35
:100E300006F0C0EB001001EB40004FF47A7148431C
:100E400047F23051B0FBF1F070BD2DE9F041344F65
:100E500005463868006810F01F0408BF012401200F
:100E6000FFF773FF06460220FFF76FFF064400F00E
:100E700055FB2D4A3118B5B1B2FBF5F0884298BF49
:100E800000200AD9C4EB0413401A5B00B0FBF3F056
:100E9000B0F5005F88BF41F6FF703B685B6860F3A8
:100EA0000C033868436038684068C0F30C00604346
:100EB000C0EB001001EB4000B2FBF0F0BDE8F081A8
:100EC00070B5174801680968006801F01F0540689F
:100ED000C0F30C060120FFF738FF04460220FFF79D
:100EE00034FF044400F01AFB06FB05F1C1EB0111CD
:100EF00004EB410108440C49B1FBF0F070BD084916
:100F00000A6852680B68C2F30C025B6860F30C035A
:100F10000868436010467047E0FE03001040002060
:100F200038E3010034E3010000389C1CFB480068F2
:100F30004068C0F30C007047F849096801EBC01025
:100F4000D0F800014EF66021C0F30A00B1FBF0F0CA
:100F5000401C400870474EF66022B2FBF1F1491C7C
:100F60004908B2FBF1F2F0B4EC4D521C56082A6865
:100F70004FEA510C02EBC01238B1D2F804318C1F89
:100F800024F00104012806D019E0ACF10603981FF3
:100F900020F0010413E02868D0F8D00010F0010F11
:100FA0000DD04800B0F5006F88BF40F2FF702F6889
:100FB000D7F8E07060F30A072868C0F8E07041EAEB
:100FC0000C40C2F80001C2F80431C2F810413046AA
:100FD000F0BC7047D14A00F00F01C0F30310126853
:100FE00002EBC11101EB4010D0F84401C0F308003E
:100FF0007047CA4A00F00F03126802EBC312D2F81E
:101000001431C0F3031002EB4010CB1AD0F8442186
:1010100061F30802C0F84421D0F844119B1E63F329
:101020001841C0F844117047BC490A68D269096880
:1010300012F0100F00F00F0201EBC211D1F82021C5
:10104000C0F3031001EB4010D2B2D0F84401C0F35A
:10105000080008BF0022801A0004000C08BF01200D
:1010600070474FEA101C0007C00EAD4B02FA00F0AB
:101070001B6803EBCC1303EB810101F5C0410B6846
:10108000184308607047A64B020900071B68C00E92
:1010900003EBC21202EB810101F5C041096821FA9C
:1010A00000F000F0030070479C480068006D704736
:1010B0009A4910200968C8657047984B00F00F02E4
:1010C000C0F303101B6803EBC21202EB4010C0F820
:1010D0004C117047914A00F00F01C0F303101268E1
:1010E00002EBC11101EB4010D0F84C0170478B4B63
:1010F00000211A68D26912F0080F0CD000F00F011D
:101100001A68C0F3031002EBC11101EB4010D0F8D4
:101110004401C0F3023108467047804A1368DB6916
:10112000D2F800C043F00803CCF81C3000F00F03E5
:101130001268C0F3031002EBC31202EB4010D0F8A8
:10114000442161F30E32C0F844217047734B0021F3
:101150001A68D26912F0080F0CD000F00F011A685B
:10116000C0F3031002EBC11101EB4010D0F84801AD
:10117000C0F3024108467047684A00F00F03C0F30D
:101180000310126802EBC31202EB4010D0F84821A2
:1011900061F31242C0F848217047042988BF7047A4
:1011A00030B400235D4C2268D269254612F0080F46
:1011B00000F00F022D68C0F3031005EBC21202EB22
:1011C00040121CBFD2F84401C0F302330020D4F80F
:1011D00000C0DCF81CC01CF0080F1CBFD2F848018E
:1011E000C0F30240C91A0844042803DD081A011D8F
:1011F000042003E00028BCBF0144002019442368F8
:10120000DB69D4F800C043F00803CCF81C30D2F8F6
:10121000443161F30E33C2F84431D2F8481160F31F
:101220001241C2F8481130BC70473C490028086898
:10123000806904D0096840F0080088617047096837
:1012400020F0080088617047344800688069C0F366
:10125000C0007047314A00F00F01C0F3031012685C
:1012600002EBC11101EB4010D0F8480180B2704789
:101270002A4B00211A68D26912F0080F0CD000F036
:101280000F011A68C0F3031002EBC11101EB40100B
:10129000D0F84801C0F30051084670471F490200CA
:1012A000086880690A6800F00100926904D0096842
:1012B00042F001028A617047096822F001028A61E6
:1012C000704730B4022ADDF808C026BF921E5208CB
:1012D0000022022B26BF9B1E5B080023114C00F04E
:1012E0000F05A4FB0C4C4FEA1C14DFF830C0C0F310
:1012F0000310DCF800C00CEBC51C0CEB4010D0F860
:1013000054C161F3196C62F3134C63F30B2C64F357
:10131000070CC0F854C130BC7047000038E301002E
:1013200050E30100CDCCCCCC70B49B4D00F00F0449
:10133000C0F303102D68DDF80CC005EBC41404EBFA
:101340004010D0F854010029C0F30166C0F30345F2
:10135000C0F30324C0B218BF0E6012B16900891C2B
:10136000116013B16100891C1960BCF1000F04BF4A
:1013700070BC704700EB80008000CCF8000070BCAF
:10138000704770B491B000224FF480456C10EC4669
:1013900001E0082A05D2531C03EB8303B5FBF3F3EA
:1013A00004E0D31F03EB8303B4FBF3F35B1A48BFE2
:1013B0005B424CF82230521C102AEAD30026009BD4
:1013C00001215CF821209A42BCBF13460E46491CFD
:1013D0001029F6D3704900F00F02C0F3031009681A
:1013E00001EBC21101EB4011D1F85801C1F858616D
:1013F000082807D2401C00EB8000B5FBF0F011B0CC
:1014000070BC7047C01F00EB8000B4FBF0F011B05F
:1014100070BC7047604A00F00F01C0F303101268FF
:1014200002EBC11101EB4010D0F85801082834BF7D
:10143000401CC01F00EB800034BF4FF480414FF4CC
:101440000051B1FBF0F0704710F00F0F08BF70476C
:10145000514A00F00F000029126802EBC010D0F8CA
:1014600024110CBF21F4803141F48031C0F82411E3
:101470007047002110F00F0F0BD0474A00F00F000B
:10148000126802EBC010D0F8240110F4803F18BF9E
:10149000012108467047404902460868D0F8AC0070
:1014A00012F0010F0A68C0F3C000D2F8AC2005D0DA
:1014B000096842F00802C1F8AC207047096822F0C0
:1014C0000802C1F8AC207047334A136858671068A7
:1014D00081677047304900280868D0F8AC0005D013
:1014E000096840F00200C1F8AC007047096820F0BC
:1014F0000200C1F8AC007047274900280868D0F8FE
:10150000AC0005D0096840F00100C1F8AC0070479C
:10151000096820F00100C1F8AC00704770B41E4E9D
:1015200000203168D1F8401111F0010F04BF70BCE8
:10153000704711F0040F336801F00805D3F81C312F
:10154000D6F800C0C3F30803DCF800C1CCF30804EC
:10155000D6F800C0DCF844C1CCF3080C18BFC1F3C6
:1015600007403268D269C1F3052112F0080204D0A5
:101570003268D2F84421C2F30232002D18BF491C50
:101580000CFA02F201FB0200604370BCC3EB0311D2
:1015900000EB41007047000038E30100FEF7F2BFA6
:1015A00010B5FEF7EFFF012818BF10BD0020FEF7B1
:1015B000E2FF21210020FEF7ECFF2121BDE81040D1
:1015C0000120FEF7E6BF10B5FEF7D4FFFEF7DAFF05
:1015D00001280AD10020FEF7CEFF21210020FEF7CE
:1015E000D8FF21210120FEF7D4FF0121052001F0C1
:1015F000A4FC0121052001F0A0FCFF490020487057
:1016000010BD10B5602001F0EEFCBDE81040602078
:1016100001F0DCBCF84A0146507A002818BF0120CE
:10162000002918BF012151727047F34A91699061F6
:1016300008467047F04800210172C1717047EE48BA
:1016400000210172C17170472DE9F34F00F00F05C1
:101650006800861E9DB0002445EA0410FEF7D4FF02
:10166000002845D01E9AC4EBC400002102EB0017ED
:10167000EC46C1EBC10307EBC30200200CEBC30334
:1016800052F8208043F82080401C0E28F8D3491CD3
:101690000229EED3D9490022301909684FF0020817
:1016A000C0EBC000434601EB001723FA02F101F042
:1016B0000101C2EBC200C1EBC1010CEBC10107EBA0
:1016C000C000B1E8004E00F5E76000F58040521C14
:1016D000A0E8004EB1E8004EA0E8004EB1E8004E90
:1016E000A0E8004ED1E90091C0E900914245DCD369
:1016F000641C022CB0D31FB0BDE8F08F70B5054656
:10170000FEF766FF29460446BC4DC0EBC400C2008C
:10171000286800F5804018F0E7FF2968C4EBC40092
:1017200001EBC00000F58040002101604160816054
:10173000C160016141618161C16101624162816297
:10174000C1620163416370BDAB494861FFF72DBAC7
:10175000AB4801688968AB4A11430268916001682F
:101760000968A94A00681143016000F0BBBE2DE979
:10177000F047A34A06460D4610688068A149014318
:1017800010688160106800689F490843116808600C
:1017900000F0A8FE0024984F002D63D00020FEF733
:1017A000EAFE286820B1FEF73EFF0020FEF7E3FEC8
:1017B00030467E61FFF7F9F90020FEF725FF00288B
:1017C00034D0DFF838826E6816B3FEF701FF814629
:1017D000C0EBC900C200D8F80000314600F58040D7
:1017E00018F082FFD8F80010C9EBC90001EBC00067
:1017F00000F58040046044608460C460046144611A
:101800008461C461046244628462C46204634463A8
:10181000E96841B1D8F800004FF4807200F5C0408B
:1018200018F062FF02E0794800F084FD0120FEF725
:10183000EBFE18B91120FEF7E7FE28B1A9680029D0
:101840001CBF0120FFF700FF0220FEF7DDFE18B9E4
:101850001220FEF7D9FE28B1296900291CBF0220F9
:10186000FFF7F2FE3C72FC71BC61787A002078725E
:10187000602001F0B8FBBDE8F047602001F0A6BB96
:1018800010B50020FEF777FE00F00EFE5C48016800
:101890000968026821F0030141F00D7141F08051A7
:1018A000116001688968006821F0020141F00D7142
:1018B00041F08051816010BD602001F08BBB10B5FC
:1018C000602001F087FBFEF75DFE01280AD10020B1
:1018D000FEF751FE21210020FEF75BFE21210120B1
:1018E000FEF757FE4A480168496C006821F48031D0
:1018F00041640020FEF73FFE00F0D6FD404801683D
:101900000968026821F0030141F00D7141F0805136
:10191000116001688968006821F0020141F00D71D1
:1019200041F08051816010BD10B501F058FB10F0FE
:10193000600018BF012010BD2F48406970472E4835
:101940000078002818BF0120704770B5FEF71AFE16
:10195000002818BF70BD0025274C2572E571212194
:101960002846FEF716FE21210120FEF712FE257003
:10197000BDE870400120FEF7FEBD10B5FEF702FE87
:10198000002818BF10BD00201B4C2072E0712121DF
:10199000FEF7FFFD21210120FEF7FBFD0120FEF7F0
:1019A00006FE01202070BDE81040FEF7E4BD0020D7
:1019B000FEF7E1BD10490020C8710120FEF7DBBD34
:1019C0000D49C86170470C48C069704770B50A4C32
:1019D0000025E069411CE161207800281CBF00203F
:1019E000FEF7C9FD20212846FEF7D3FDA169002995
:1019F0001CBF284688470DE01440002050E301003A
:101A000040E301000200341203003412D4420020EB
:101A100034E30100FE48016841F02001016070BD1F
:101A200070B5FC4C0125E069411CE161207800287B
:101A30001CBF0020FEF79FFD20212846FEF7A9FDD0
:101A4000A16900291CBF28468847F148016841F078
:101A50002001016070BDF0487047F0487047ED48C4
:101A6000006A7047EB48406A7047EA48806A7047EE
:101A70002DE9F00FE84E4FF0000C87B006F1380763
:101A8000E1464FF0FF3806F80C8007F80C900CF197
:101A9000010CBCF11C0FF6DB4FF0000C002807D93D
:101AA00012F80C4006F80C400CF1010C6045F7D818
:101AB0000024A4464FF0010A00280FD93257002A0B
:101AC00009DB082AB4BF1432083A1C2A3CBF0AFAC0
:101AD00002F242EA0C0C641C8442EFD3002214464A
:101AE0006D460AFA02FB1BEA0C0F1ABFAC54641CC9
:101AF00005F80280521C1C2AF3DB0022002817D9AB
:101B000016F902C0BCF1000F0FDBBCF1080FB4BF27
:101B10000CF1140CACF1080CBCF11C0F3ABF15F819
:101B20000CC007F802C007F80280521C8242E7D3BB
:101B3000B84C00220028C4F8209008D917F902C038
:101B4000944501D0276202E0521C8242F6D3B44F82
:101B50000020A7F1540CA7F11C060CF8008006F831
:101B6000009007F80090401C1C28F6DB002000299C
:101B700005D91A5C0CF80020401C8142F9D80020DD
:101B8000024600290BD91CF90230002B04DB1C2B68
:101B90003CBF0AFA03F31843521C8A42F3D30022D3
:101BA00013460AFA02FB1BEA000F1ABFAB545B1C78
:101BB00005F80280521C1C2AF3DB002200290AD9F6
:101BC0001CF90230002B03DB1C2B3CBFEB5CBB542D
:101BD000521C8A42F4D30022C4F82890002907D965
:101BE000BB56934201D0A76202E0521C8A42F7D34F
:101BF00011F0010F18BF1B2209D00AFA02F30342A9
:101C000003D10AFA02F2104301E0521EF5D5002278
:101C100013460AFA02F707421ABFAB545B1C05F8D9
:101C20000280521C1C2AF4DB002000290AD91CF96E
:101C30000020002A03DB1C2A3CBFAA5C3254401C53
:101C40008842F4D30020C4F8249000299EBF07B036
:101C5000BDE8F00F70473256824204D0666207B08A
:101C6000BDE8F00F7047401C8842F4D307B0BDE8D0
:101C7000F00F7047C0EB00106A4900EBC00001EBA9
:101C8000C0007047C0EBC00101EB0010664901EBDA
:101C900080007047DFF87CC1012B8CF802008CF8C3
:101CA000031003D9401C20F00100114600FB01F293
:101CB0004FF6FF718CF8040001EA4202ACF80C20E8
:101CC00001EA4000ACF80E007047524A5071917121
:101CD00070475048807970474E4840797047534A62
:101CE0001070517070475149085C704770B5494D8C
:101CF0000446687A002804BFE87918F0E2FD287AE3
:101D0000002808BF70BD4FF0000C6869634662464A
:101D1000614610F0020F1CBFDFF808C110F0040F7D
:101D200004D0AB893F4E23F00103334410F0010F80
:101D300004D010F0100F0CBF3B4A3B49ED69256001
:101D4000C4E90321C4E901C310F0200F14BF3848CF
:101D500000206061012070BD2E490020087270478C
:101D600010B50446FEF734FCC0EBC000C200314899
:101D7000006800F580412046BDE8104018F0B4BC72
:101D80002DE9F041FEF724FC04460020FFF7A2F9FC
:101D900000220546002C84BF0126264F21D93B682E
:101DA000C2EBC200002103EBC00C06FA01F028428E
:101DB00011D048080CEB800000F58040CB0700688C
:101DC000DB0E20FA03F3C3F30B00B0F57F6F02D9EB
:101DD0000020BDE8F081491C1C29E6D3521CA24218
:101DE000DDD30120BDE8F0812DE9F05F00F00F06A2
:101DF0000024104F8846750046EA0410FEF704FCE4
:101E0000002849D002218A460023C4EBC40013E015
:101E10004440002014400020D4420020F042002022
:101E200044430020D0430020084800201E400020EA
:101E30006448002050E3010008EB001B002000294B
:101E400008D92AFA00F202F001029A421CBF401C93
:101E50008842F6D388421CD2A5F10209A144D7F8E2
:101E600000E0C3EBC302C9EBC9090BEBC20C0EEBDC
:101E70000919C0EBC000002209EBC00909EB820080
:101E800000F58040D0F838074CF82200521C0E2A8A
:101E9000F4D35B1C022BD1D3641C022CACD3BDE861
:101EA000F09F2DE9F05F00F00F0670000025DFF8CD
:101EB0007494A0F10208012746EA051A5046FEF77D
:101EC000A3FB002839D05046FFF711F907FA00F4B8
:101ED000022C88BF02245046FFF7FCF80022002C99
:101EE0002BD908EB0501D9F80030C1EBC10103EB98
:101EF000011BC2EBC20300210BEBC30A07FA01F37B
:101F0000034214D04B080AEB830303F580434FEAE6
:101F1000C17CD3F838374FEADC6C23FA0CF3C3F3F7
:101F20000B03B3F57F6F02D90020BDE8F09F491C79
:101F30001C29E3D3521CA242DBD36D1C022DBBD360
:101F40000120BDE8F09FC1EBC103F6494FF6FF7CCD
:101F5000096801EBC301430801EB830101F58041EE
:101F6000C007C00E0CFA00FC0B6802FA00F023EA6E
:101F70000C03184308607047EA4AC1EBC1011268BC
:101F800002EBC101420801EB820101F58041C0076B
:101F90000968C00E21FA00F080B270472DE9FF4FAA
:101FA000E04883B01D460068109C00F5804017464D
:101FB0000E460190FEF7E6FA5FEA00081CBF00201B
:101FC000FEF7D9FA0020FFF785F8824670190090D5
:101FD000B04284BF4FF0010B4FF6FF7E28D9019825
:101FE000C6EBC6014FF0000C00EBC101039B17E0EC
:101FF0000BFA03F010EA0A0F11D05808DD0751F868
:102000002020ED0E0EFA05F922EA090234F8029BAF
:102010000CF1010C09FA05F52A4341F820205B1C5C
:10202000BC4538BF1C2BE3D30098761C8642D6D320
:10203000B8F1000F04BF07B0BDE8F08F0020BA4927
:10204000C87107B00120BDE8F04FFEF794BA2DE942
:10205000F0470746B3489A46144600680E46089D66
:1020600000F58049FEF78EFA5FEA00081CBF0020E9
:10207000FEF781FA06EB0A03B34284BFAB4907EBD4
:10208000040C1CD9C6EBC6003C4609EBC0000FE0AF
:102090000A571C2A0BD202EBD27A4FEA6A0AD207FD
:1020A00050F82AA0D20E2AFA02F225F8022B641C5C
:1020B000644538BF1C2CEBD3761C9E42E2D3B8F1AA
:1020C000000F08BFBDE8F08700209749C871BDE840
:1020D000F0470120FEF74FBA2DE9F05F0027DFF847
:1020E0004882904A4FF6FF7600280C4647D0116888
:1020F00001F5804900F00F01C0F3031001290EBF64
:1021000000210229BDE8F09F022828BFBDE8F09F0A
:1021100001EB000AFEF736FA05001CBF0020FEF7AF
:102120002AFA0020CAEBCA0109EB0119C0EBC00171
:10213000002209EBC10153084FEAC27C4FEADC6C74
:1021400001EB830306FA0CFBD3F838A704FA0CFC66
:102150002AEA0B0A4AEA0C0C521CC3F838C71C2A9C
:10216000E9D3401C0228E1D3002D08BFBDE8F09F51
:1021700088F80770BDE8F05F0120FEF7FCB9106831
:1021800000F58049FEF7FEF905001CBF0020FEF7B0
:10219000F2F94FF0000CCCEBCC00002209EBC001AF
:1021A0005308D007C00E06FA00FB51F823A004FA2A
:1021B00000F02AEA0B0A4AEA0000521C41F8230008
:1021C0001C2AEDD30CF1010CBCF1210FE3D3002D3F
:1021D000CED1BDE8F09F10B5FEF726FF5249088228
:1021E00010BD514AC1B200F47063128A914288BF97
:1021F00011464FF0640C01FB0CF1B1FBF2F11A0A2D
:1022000002FB0C1189B210F4805F12BF08B2484281
:1022100000B270470028B8BF404280B2B4BF00216E
:102220004FF4805100F4706211433F4AC0B2128AE9
:10223000504341EA102070473D4800F07BB870B52C
:102240003B4800F077F8374840F6F801006800F5A1
:10225000804018F04EFA0020FEF751FE002108469B
:10226000FEF75BFF0020FEF7E0FF00210120FEF7F4
:1022700054FF00211120FEF750FF00210846FEF711
:102280007BFF00210120FEF777FF00211120FEF7E0
:1022900073FF0120FEF750FE04460120FEF79AFE70
:1022A00006461120FEF796FE0546A64288BF264642
:1022B000A54288BF254631460120FEF79AFE2946F1
:1022C0001120FEF796FE0020FEF761FC002102209F
:1022D000FEF723FF00211220FEF71FFF002102203E
:1022E000FEF74AFFBDE8704000211220FEF744BF10
:1022F0000D4910B502204861FEF757FC094C4FF418
:102300008071206800F5C04018F0F3F920684FF4A0
:10231000E76100F5804018F0ECF9BDE810400020BE
:10232000FEF7EDBD50E3010014400020F042002014
:10233000D442002070B5144D04464FF480712868D3
:1023400000F5C04018F0D5F9002101206256002A9E
:1023500015DBD31702EB137C4FEA2C132E682CF0FD
:102360000F0C06EBC31303EB810303F5C043A2EB91
:102370000C0252001E6800FA02F232431A60491C35
:102380001C29E3D370BD000050E3010070B40024A9
:102390006B4982B04FF0010C002814BF0C7081F81B
:1023A00000C0684D28680068674A10432A681060BA
:1023B0000978664A31B113686548D8601368654882
:1023C000986006E013686448D86013684FF0BB70EB
:1023D00098606248006830F0FF0305D11368DB683D
:1023E00060F303031068C36040F2E243C1B11068B8
:1023F0008068166840F01800B0600120009004E08A
:102400000198461E0196FBD20098461E009628BFF2
:102410000193F5D210688068166840F48050B0606F
:102420000120009004E00198461E0196FBD200981E
:10243000461E009628BF0193F5D21068C068166842
:1024400040F03000F0601068D0F8B000166840F03E
:102450000100C6F8B0000120009004E00198461E7B
:102460000196FBD20098461E009628BF0193F5D234
:102470001068C0F87CC013684FF4E0601861106801
:10248000C0F8884000291CBF1068C0F894C02868B4
:102490000068296820F0040040F00D7040F0805082
:1024A000086002B070BC704728480168C9680268BB
:1024B00021F03001D1602249097839B10168896879
:1024C000006821F0180121F4805181601D480168E5
:1024D0000968006821F0040141F00D7141F080515C
:1024E00001607047174801680968174A006811437E
:1024F000016013480178154831B10168896841F2DB
:1025000018021143026891600168C968026841F0CD
:102510003001D1600168D1F8B010006841F00101CC
:10252000C0F8B01070470E49C0B241EA0020074918
:1025300009680864704705490A48096808647047D3
:102540004040002040E30100040034123CE301005D
:10255000057601002000760105F40100D0FE03009D
:1025600013005FA000005FA05948584902689161BC
:102570000268891CD1610268491E516302681268B1
:10258000036822F0030242F00D7242F080521A609A
:1025900002685269036822F0010242F00D7242F0B3
:1025A00080525A610268126911430268116102681F
:1025B0004849916000684849C16048490020086066
:1025C000704770B501F071F9444D2C682CB10020B2
:1025D000286001F06FF9204670BD30BF00F0A3FD08
:1025E0000028F2D000F0B2FD6860EEE72DE9F0417E
:1025F00001F05BF9354E364CDFF8E080771CD8F8F7
:1026000000503DB10020C8F8000001F053F9284601
:10261000BDE8F08172B6206846632068876120BFFC
:10262000206886612068476362B6BFF36F8FBFF38F
:102630004F8F00F078FD0028E1D000F087FDC8F84A
:102640000400DCE7224801680968026821F0030100
:1026500041F00D7141F08051116002682049916094
:10266000016809691F4A00681143016130BF704762
:1026700072B616491648026851630268C91CD161D6
:102680000068891E816162B6704711480168096857
:10269000154A00681143016070470D4801680968D8
:1026A000006821F0030141F00D7141F0805101609B
:1026B000704772B605490648026891610268891C34
:1026C000D1610068491E416362B670470000341250
:1026D00040E301003C003412280034124440002042
:1026E000080034120100341203003412704700282D
:1026F00018BF0120B64909684860704700220029C8
:1027000009D950F8043BB3F1FF3F01D000207047D6
:10271000521C8A42F5D30120704730B44FF0000CB0
:102720006346002A13D950F8044B51F82350AC42A9
:102730001CBF0CF1010C1FFA8CFC5B1C9BB293427A
:10274000F1D3BCF1000F1EBF002030BC7047012048
:1027500030BC70472DE9F041054601F0B0F8002487
:102760009B4B21274FF482582646186807602E603D
:1027700018680068196840F004000860186800686C
:1027800010F0040FFAD11868C0F8008040202946E4
:10279000002251F804CBBCF1FF3F08D01868066056
:1027A000601CC4B2082CE0D30220BDE8F081521CAA
:1027B0008242EED3186806600120BDE8F0812DE961
:1027C000F041044601F07BF80020814B0925844646
:1027D00019680D60C4F800C0196809681A6841F0EA
:1027E000040111601968096811F0040FFAD121463B
:1027F0004FF48066002251F8047BB7F1FF3F09D007
:102800001968C1F800C0401CC0B20328E0D3022000
:10281000BDE8F081521CB242EDD31868C0F800C088
:102820000120BDE8F0812DE9F05F0F4680460426C7
:102830004FF0020A4FF0000BDFF8949101F03FF8DF
:10284000D9F8001044463846C1F800A00F21B0E87E
:102850002C10A4E82C10491EF9D2D9F80000006809
:10286000D9F8001040F004000860D9F800000068B2
:1028700010F0040F07D000BF00BFD9F800000068B7
:1028800010F0040FF7D1D9F80000C0F800B04546A9
:1028900038460F21D5E90023D5E902C4D0F800E07D
:1028A000964504BF42689A4205D18268624504BFDA
:1028B000C268A24208D0761E03D34046FFF74AFF03
:1028C000BCE70220BDE8F09F10301035491EE1D270
:1028D0000120BDE8F09F70B50D46044600F0EFFF03
:1028E0004FF480722146284617F0FEFE012070BD8D
:1028F0002DE9F041C0B014460E46054610F0FF0F1A
:1029000023D025F0FF086F4600F0D9FF4FF4807206
:102910004146384617F0E8FEE8B2C0F58077A74296
:1029200088BF274668443A46314617F0E7FE4046DE
:10293000FFF710FF022843D069464046FFF773FFB8
:10294000022841D03D443E44E41BB4F5807F19D3B6
:102950004FF480723146684617F0D0FE2846FFF7E4
:10296000F9FE02282CD069462846FFF75CFF0228B2
:102970002AD0A4F5807405F5807506F58076B4F547
:10298000807FE5D2C4B16F4600F099FF4FF48072AA
:102990002946384617F0A8FE22463146684617F009
:1029A000ADFE2846FFF7D6FE022809D06946284624
:1029B000FFF739FF022807D040B00120BDE8F081C1
:1029C00040B00A20BDE8F08140B00B20BDE8F081A6
:1029D00024E3010028490A6810600968086100F0D2
:1029E00016B825490A6810600968486100F00FB8F8
:1029F00021490968486770471F4909688867704717
:102A00001D480121026811660068016570471B4A74
:102A10001168096B10F0010F18BF21F4404110F04C
:102A2000020F1CBF21F4405141F4805110F0040FFB
:102A300018BF41F4406110F0080F18BF41F4407115
:102A400010F0100F18BF41F0C00110F0200F18BF98
:102A500041F0300110F0400F18BF41F00C0110F0B0
:102A6000800F18BF41F0030141F4BE00116840F02F
:102A700020400863704700002CE3010034E30100AC
:102A8000FE4801688A68FE4903680A439A60026842
:102A9000D26811430268D16001684969F94A006847
:102AA000114341617047F54801684969026821F0A6
:102AB000010141F00D7141F0805151610168C96817
:102AC000026821F0400141F00D7141F08051D16068
:102AD00001688968006821F0400141F00D7141F002
:102AE00080518160704710B5E44C20688168E448EB
:102AF0002268014391602168C96808432168C86061
:102B000020684069DF49084321684861DE483F2169
:102B10000268D160026800219163026891640068D4
:102B2000C0F8B01003210A2000F007FA0A2000F0D4
:102B300028FA20684069216820F0010040F00D70FB
:102B400040F0805048612068C068216820F0400053
:102B500040F00D7040F08050C860206880682168A7
:102B600020F0400040F00D7040F08050886010BDB3
:102B7000C54A136818601368596048431168886033
:102B80007047C14A1368186013685960484310F0D1
:102B9000010F18BF401C116888607047BA49096866
:102BA000C1F8B0007047B84918B1096801208864BD
:102BB00070470968002088647047B3490A689063C9
:102BC0000868C068096840F00200C8607047DFF814
:102BD000B8C210B4DCF800402062DCF800004162AA
:102BE000DCF800008262DCF80000C362DCF8001050
:102BF00001200863DCF80000406B10F0010F09D0E1
:102C000000BF00BF00BF00BFDCF80000406B10F049
:102C1000010FF5D110F0020018BF4FF0FF3010BCCB
:102C2000704799480168C968006821F00201C160D5
:102C3000704795480168C968006841F00101C160AA
:102C40007047914BD3F800C0CCF82000186841625F
:102C5000186882621968012008641868406C10F0D6
:102C6000010F08D000BF00BF00BF00BF1868406C54
:102C700010F0010FF6D110F0060018BF4FF0FF3032
:102C8000704781480168C968006821F00101C1608E
:102C900070477D480168C968006841F00401C1605F
:102CA0007047027C017B02F03F0241EA0241764A12
:102CB00013689965136801685962136841689962DD
:102CC00013688168D9621368012119651168496D1B
:102CD00011F0010F08D000BF00BF00BF00BF116896
:102CE000496D11F0010FF6D11368DB6D8382136813
:102CF000DB6D1B0CC38213681B6E038313681B6E92
:102D00001B0C438313685B6E83831268526EC2F39D
:102D10000E42C28311F0020018BF4FF0FF3070471F
:102D200059480168C968006821F00401C160704712
:102D300055480168C968006841F00801C1607047E2
:102D4000DFF844C110B4DCF80040A267DCF80020D2
:102D50001062DCF800004362DCF800008162DCF8FD
:102D6000001001200867DCF80000406F10F0010F30
:102D700009D000BF00BF00BF00BFDCF80000406FFB
:102D800010F0010FF5D110F0060018BF4FF0FF3022
:102D900010BC70473C480168C968006821F0080110
:102DA000C160704701684FEA314237490B68C3F888
:102DB00098200A684068C2F89C000868C0680968E2
:102DC00040F02000C86070472F4A136818621068EE
:102DD000416211680120C1F890001068D0F8940099
:102DE00010F0010F09D000BF00BF00BF00BF106886
:102DF000D0F8940010F0010FF5D110F0060018BFC4
:102E00004FF0FF30704720480168C968006821F022
:102E10002001C16070471C480168C968006841F022
:102E20001001C1607047A3F1050C174B10B41C686A
:102E3000C4F888C0D3F800C0CCF8200018684262FB
:102E40001868816219680120C1F880001868D0F8FC
:102E5000840010F0010F09D000BF00BF00BF00BF09
:102E60001868D0F8840010F0010FF5D110F00600BA
:102E700018BF4FF0FF3010BC7047000040E3010066
:102E8000400034120100341244E301000348016899
:102E9000C968006821F01001C160704744E3010077
:102EA000234810B5026802211165026801211166EC
:102EB000036810225A67036841F206025A660368E3
:102EC00000229A660268C2F8881002689021C2F84F
:102ED00084100168D1F88410026841F00101C2F841
:102EE000841002684FF48171116600680166032046
:102EF00000F047F80021032000F01FF8002010BD6B
:102F000010B5032000F048F809484FF480710268BA
:102F1000116602680021116602681021916700683D
:102F200002214165002010BD024900200870704751
:102F300030E301004C400020704700F00303DA004A
:102F40004FF0FF0C0CFA02F24FF0050C0CEBC30330
:102F5000994000F00C03002808DA30480068184453
:102F60004369114093431943416170472C480068FD
:102F70001844D0F80033114093431943C0F80013AC
:102F8000704700F01F01012202FA01F1244A4009B2
:102F9000126842F82010704700F01F01012202FA67
:102FA00001F11F4A4009126802EB8000C0F880104E
:102FB000704700F01F01012202FA01F1184A40098E
:102FC000126802EB8000C0F880117047144909684C
:102FD0000860704712490968C1F8800070471048BE
:102FE0000068006870470E490968C1F880017047A1
:102FF0000A4800688068704708490A68926809684A
:10300000886010467047054A1268926800F1100304
:1030100052F8230042F823107047000020E301001B
:103020001CE3010002210C20FFF787BFC74801689D
:103030008A68C74903680A439A600268D2680068D0
:103040001143C1607047C14801688968026821F472
:10305000805141F00D7141F0805191600168C96863
:10306000006821F4805141F00D7141F08051C16040
:103070007047B84881B00168096F11F4007FFAD138
:103080000168896E11F0010F09D00168D1F8841030
:1030900000910168D1F88410009A9142F9D001683A
:1030A000096F11F4007F03D102684CF271011166BF
:1030B000006842F24131816601B07047A5494FF482
:1030C0000D520B689A660A68126F0B68DA66002860
:1030D00008BF012080B24FF05C5242EA00200A682B
:1030E000506609684FF01140C1F88000C1E7994867
:1030F00081B00168096F11F4007FFAD10168896E0F
:1031000011F0010F09D00168D1F884100091016815
:10311000D1F88410009A9142F9D000684FF40D5113
:10312000816601B0704789480068806810F480505B
:1031300008BF704787480068806E00F00100704744
:1031400084480068406EC0F30F20704781480068D3
:10315000D0F88400704710B50C20FFF72AFF0C2030
:10316000FFF70FFF7B4902200968486710BD7949C6
:1031700010B50968032088670C20FFF70DFFBDE834
:1031800010400C20FFF715BF734A11681060084605
:103190007047704810B50168096F0068C1666E48D5
:1031A0000068002818BF80476C48016841F48051CE
:1031B000016010BD684840687047644810B50168F8
:1031C0008A68634903680A439A600268D2680068A3
:1031D0001143C1605F4C0320216888670C20FFF712
:1031E000DBFE0C20FFF7E5FE00F0B2F95C4B04209B
:1031F0001968C1F8880019684FF6FF70C1F88C0093
:1032000072B621684FF40D5088662068006F2168FF
:10321000C86621685348486621684FF01140C1F8DC
:103220008000FFF726FF19684FF40070086662B649
:1032300010BD38B572B647480168096F11F4007FB8
:10324000FAD10168896E11F0010F09D00168D1F837
:10325000841000910168D1F88410009A9142F9D04D
:1032600002684FF40D5191663D494FF400330A68EE
:10327000136662B60968D1F80412344C002948D0AC
:10328000354B4FF6FF72511A996022689269D4F853
:1032900000C002F00F02DCF81CC00CF00F0C6244FE
:1032A000121D9140A1F5EA42DFF8BCC0313A6245F7
:1032B0002FD20068D0F88400C0F10110D860B0F5BA
:1032C000803F26D20004B0FBF1F040F2C911484320
:1032D0001861B0F57A7F38BF4FF47A70DFF88CC090
:1032E000DCF80810002908BFCCF80800DCF804203E
:1032F000CCF80020DCF80810CCE901108A421FD974
:10330000824205D9814201D9596002E0586000E04B
:103310005A6000F02EF920688068216820F48050FF
:1033200040F00D7040F0805088602068C0682168CF
:1033300020F4805040F00D7040F08050C86038BDDF
:103340008242E5D88142E1D8DEE7000040E3010097
:10335000001034124CE30100504000204440002093
:1033600048E3010000FFFF372F6E16009048002051
:10337000134801688968134A006811438160124844
:1033800001684969026841F4007151610168096985
:10339000026841F00401116101680969006841F0A7
:1033A0001001016170470849096888607047BFF3E0
:1033B0004F8F054905480968C860BFF34F8FFEE786
:1033C00040E301000400341220E301000400FA0588
:1033D000254801688968254A0068114381602448AE
:1033E00001684969026841F0010151610168096B96
:1033F000204A21F440511143026811630168096AAF
:10340000036821F00F021C490A431A621B4B8A1EF3
:103410001B68C3F8C4200068016570471448006841
:10342000006900F070007047114815490268116387
:103430000268144951630168496C026821F4003143
:1034400051640168496C40F2FF32114302685164D3
:103450000168496C006821F4803141647047044878
:10346000006840687047000040E301000400341227
:1034700034E3010000205FA003005FA03CE30100F3
:10348000C08C5FA095995FA0022824BF00207047E0
:10349000B84B53F8202043F820101046704770B501
:1034A000B54C2068006FB34D10F0010F06D02168B5
:1034B0000120C8662868002818BF80472068006F70
:1034C00010F0020F08BF70BD02202168C86668684E
:1034D000002808BF70BDBDE870400047A74810B580
:1034E00001688A68A64903680A439A600268D2683C
:1034F00011430268D160A04902220B681A65D1F815
:1035000000C00123CCF86030D1F800C00323CCF810
:103510006C3009684A6501688968026821F0800199
:1035200041F00D7141F0805191600168C9680068F7
:1035300021F0800141F00D7141F08051C1600920FE
:10354000FFF71FFD0221BDE810400920FFF7F5BC81
:103550008A4801688A688A4903680A439A6002684F
:10356000D26800681143C160834902200968086578
:103570007047814902200968486580480168896868
:10358000026821F0800141F00D7141F0805191609D
:103590000168C968006821F0800141F00D7141F0B7
:1035A0008051C1607047754800688068C0F3C010E2
:1035B000704771480168096F11F4007F04D00068FA
:1035C0004FF440710166704700684FF480710166E6
:1035D000704710B5684C2068C06F10F0020F4FF0B4
:1035E000010018BF03202168486700F0F3F8634921
:1035F0000A689269096802F00F02D040C96922681E
:1036000001F00F01C8400521B0FBF1F04FF4057146
:103610000009C2F8801018F096FD5A4A5A4B18F06B
:10362000A5FD18F063FD2168C1F884002068006FD3
:1036300010F4007F04D021684FF44070086610BD7C
:1036400021684FF48070086610BD4B480168096F0F
:1036500011F4807F04D000684FF440710166704718
:1036600000684FF4007101667047434B30B41A682C
:10367000D26F12F0010F1DBF4FF0030C1A68C2F891
:1036800074C0022204BFD3F800C0CCF874204FF0FD
:10369000020C00EB4005C5EBC0104FF49674C1EB73
:1036A000C0004C4300EB8000384904EB4010A1FB04
:1036B000001032490022C0080C68A469096804F0AF
:1036C0000F04C96901F00F012144C8400521B0FB76
:1036D000F1F0B0F5803F05D3511C4008CAB2B0F5F7
:1036E000803FF9D242EA0C211A6841F01001C2F879
:1036F00088101968C1F88C001868006F10F4807F7A
:1037000005D019684FF44070086630BC70471968DE
:103710004FF40070086630BC704717480168096FA5
:1037200011F4003F04D000684FF440310166704747
:1037300000684FF48031016670470F480168096FD7
:1037400011F4803F04D000684FF4403101667047A7
:1037500000684FF400310166704707480068006F49
:10376000C0F30020704704480068006FC0F3402099
:10377000704700006440002048E3010040E301007E
:10378000800034127B14AE47E17A843FCDCCCCCCA0
:10379000244900200A68906009680860224948604E
:1037A000704710B51F4C2168486021680020886070
:1037B0000221401EFFF7C1FB21680720086010BDF1
:1037C0001849002009680860704717480188491C9B
:1037D000018070471448806870472DE9F041124C11
:1037E000002705462780A0684FF47A71B0FBF1F0FE
:1037F0000C4E401E31684860306887600221C81E48
:10380000FFF79BFB3168072008602188A942FCD3A1
:1038100030680760BDE8F081044948430249886088
:103820007047000018E301006C40002040420F0088
:10383000704770B52C4C05464FF40D5021688866D2
:1038400021680320C86621682848486621684CF230
:103850007100086621682648C1F88000216842F29C
:103860004630886602210020FFF767FB0020FFF743
:1038700088FB002D08BF70BD2068806E42F2413188
:1038800008432168886670BD174810B50268012199
:10389000916700684FF40D5181660020FFF77CFBB3
:1038A000BDE810400020FFF784BB0F4901200968E4
:1038B000486770470C4901200968886770470A49C2
:1038C0004CF27100096808667047074881B04CF2F5
:1038D0007101026811660168096F0268D1660068AB
:1038E000006F009001B0704728E3010007383937B6
:1038F000009C1C9170B5FF4D00244FF480612C702A
:103900006C70FD4816F0F5FE4FF48061FB4816F030
:10391000F0FEFB486C60AC70046044608460C4607E
:10392000046144618461C461046244628462C4626B
:10393000046344638463C463046444648464C4644B
:10394000046544658465C465046644668466C4662B
:10395000EC705821703016F0CCFE5821E94816F072
:10396000C8FEAC6070BDE3488078002818BF012015
:103970007047E048C078002818BF01207047DD4834
:103980004078002818BF01207047DF48704770B5A5
:10399000DE4EDF4D0446014632782878DA4B10447B
:1039A0004200184616F0AAFE32782878D54B10440B
:1039B00042002146184616F0A1FECE490120C870EB
:1039C00070BDCC4880687047CB4870472DE9F04106
:1039D000C84F80463878002814BFCE48CE480578B6
:1039E00014BFCE48CE48047805FB04F6FFF748F82C
:1039F00021462846FFF7BCF8C04A4346A2F580613D
:103A00000846FFF7E4F8FFF74EF872004146BB485E
:103A100016F074FE01207870BDE8F0812DE9F047C2
:103A2000B44D044601462878DFF8CCC2DFF8E482C2
:103A3000DFF8E492B94EBA4F002815BF98F800207D
:103A400099F8002033783B7802FB03F04FEA4002FC
:103A5000604616F053FE2878DFF8A0C22146002801
:103A600015BF98F8002099F8002033783B7802FBC6
:103A700003F04FEA4002604616F040FE01206870F5
:103A8000BDE8F0879B484068704770B5A54C054677
:103A9000014622789A48520016F030FE22782946D4
:103AA0005200A14816F02AFE92490120887070BD8C
:103AB0002DE9F04F8F4DADF2344D95F801B095F8EA
:103AC00002A095F80390FDF769FDCDF82C04FDF7F1
:103AD00036FFCDF82804FDF763FD0020FDF70FFA4F
:103AE000CDF82404FDF749FF00240127CDF8184440
:103AF00004F088FF012811D00DF58060FEF7F6F87C
:103B0000002800F07F810DF5806005F0BFFCDDF836
:103B1000080410B3BAF1000F05D01EE00120CDF863
:103B2000180400F072B906460CB3FEF7A9FF7D4DEC
:103B300001212878FFF71CF87B4A3346A2F13801AF
:103B40000846FFF744F8FEF7AEFF287831464200FA
:103B5000754816F0D3FD67488770DDF80404002827
:103B600000F0B480BBF1000F11D000F0AFB86D4D84
:103B7000314628784200624816F0C0FD2878314668
:103B80004200694816F0BAFD5A488770E5E7DFF849
:103B90006481054698F8000000283DD1D8F80460FB
:103BA00026B35C480078CDF820045C480078CDF856
:103BB0001C04FEF765FFDDF81C14DDF82004FEF799
:103BC000E0FF294632460846FFF73BF8FEF76BFF59
:103BD00056480078022804BF304605F015FA5348CD
:103BE0000078092804BF284605F00EFA50480078EE
:103BF000012811D94D4E3078042804BF284605F01D
:103C000003FA2946684617F0DFFA0546307805289A
:103C100004BF284605F0F8F944B3CDF81C5498F8D1
:103C2000000000280CBF3C483A48057814BF3B48C8
:103C30003B48067805FB06F8FEF722FF314628468A
:103C4000FEF796FF2D4ADDF81C34A2F58061084688
:103C5000FEF7BDFFFEF727FF4FEA48022748DDF8D1
:103C60001C1416F04BFD2348477028E098F800001C
:103C7000214B2946002814BF26482748027814BF44
:103C800026482748007802FB00F04FEA4002184619
:103C900016F034FD98F8002018482946002A14BF71
:103CA0001C4A1D4A127814BF1C4B1D4B1B7802FB8B
:103CB00003F24FEA420216F021FD88F801701B481A
:103CC0000078032804BF0C4805F09EF9DDF81004C5
:103CD000002877D0B9F1000F74D1DFF818800546BD
:103CE00098F8000030BBD8F808601EB30748017888
:103CF000074820E0784000209C4800209C4C002091
:103D00009C540020645500200C550020A340002046
:103D1000A4400020A14000209E400020A24000209E
:103D20009F400020A5400020D45400200D410020D9
:103D3000A040002021E000780844401C4008019089
:103D400002200090FEF79CFEDDE90010FEF719FF4F
:103D5000294632460846FEF774FFFEF7A4FEFE48E9
:103D60000078022804BF304605F064FAFA4800786B
:103D7000092804BF284605F05DFA5CB32E46F748D3
:103D80000178F74800780D18FEF77AFE681C4008A5
:103D90000221FEF7EDFEF34A3346A2F15801084630
:103DA000FEF715FFFEF77FFE6A003146ED4816F07C
:103DB000A5FC88F80370E8480078032804BFEA48A7
:103DC00005F038FAFDF7C8FF641C042C1DD2FDF77E
:103DD000D4FD8DE6E14EE248E34B32780078294687
:103DE00010444200184616F089FCDD483278DD4B5D
:103DF0000078294610444200184616F07FFC88F8E7
:103E00000370D8E701F07CFB72E6FDF7C9FBDDF833
:103E10002404FDF774F8DDF82C0438B1DDF828042B
:103E200010B1FDF7AAFD01E0FDF78FFDDDF81804E4
:103E300030B1CE4880F801B080F802A080F803903D
:103E4000DDF818040DF2344DBDE8F08F10B50024F4
:103E5000FDF772FDC54910F0020F0AD04A78002A1A
:103E600008BF012410F0040F03D08A78002A08BF8D
:103E7000012410F0010F18BF10F0100F03D0C87804
:103E8000002808BF01240020002C08BF10BD00201E
:103E90000870BDE810400BE608B50F2101F0D2FB19
:103EA000012804D1FFF7D2FF009001F021FDAF48B7
:103EB000417800291CBFC178002904D080780028EF
:103EC0001CBF012008BD002008BD08B50F2101F06E
:103ED000B9FB012804D1FFF7B9FF009001F008FDFC
:103EE000A248417800291CBFC178002904D08078FD
:103EF00000281CBF012008BD002008BD70479B4959
:103F0000002048708870C870704710B54FF4806109
:103F1000974816F0EEFBBDE810404FF480619548DD
:103F200016F0E7BB2DE9F047904F814608983978A5
:103F3000002914BF904991490D78A0EB030805FBB7
:103F400008F603FB05F4FEF79BFD41462846FEF705
:103F50000FFE884809EB440500EB4408A0F5806C8F
:103F60000CEB44012B4642460846FEF730FEFEF7B6
:103F70009AFD72002946404616F0C0FB0120787079
:103F8000BDE8F087002818BF0120784948707047C5
:103F900010B5764C002804BF606010BDDFF8E0C1AA
:103FA00075490B7877490A7801465A4352006046B2
:103FB00016F0A4FB7248606010BD734900200860D1
:103FC00048608860C860086148618861C8610862AB
:103FD00048628862C862086348638863C86308648B
:103FE00048648864C864086548658865C86508666B
:103FF00048668866C866704763487047002818BFDF
:1040000001205A498870704710B55821564816F05B
:1040100070FBBDE810405821524816F06ABB0028DA
:1040200018BF01205149C870704710B54F4C002887
:1040300004BFA06010BDDFF854C148490B7848495F
:104040000A7801461A445200604616F057FB4F4862
:10405000A06010BD4549002200284A708A70CA70CD
:1040600018BF0120087023E52DE9F04F87B04FF409
:1040700080613F4816F03DFB4FF480613D4816F0EB
:1040800038FB5821384816F034FB5821354816F0D3
:1040900030FBFDF751FC0446FDF782FA0020FCF7E7
:1040A0002EFF0690FDF769FC00252E4604F0AAFCC1
:1040B000012875D06846FDF719FE002878D06846BB
:1040C00005F0E4F914F0020F1CD02B48DFF8A0B083
:1040D000DDF8049090F800802A48DA460778FEF769
:1040E000CFFC0120FEF75FFD39464046FEF749FD53
:1040F000524649465846FEF7A4FD0020FEF753FD00
:10410000FEF7D1FC14F0010F18BF14F0100F20D0EF
:104110001248DFF854B04FF0020801781048DA4630
:10412000DDF8109000780844401C4708FEF7A8FC12
:104130000120FEF738FD41463846FEF722FD524683
:1041400049465846FEF77DFD0020FEF72CFDFEF7A0
:10415000AAFCFDF701FE1DE012410020A340002053
:10416000A4400020645500200C5500207840002019
:104170009C4800209C4C0020A14000209E40002034
:104180009C500020A24000209C540020BC550020E0
:1041900006E00DE06D1C102D03D2FDF7EEFB85E768
:1041A0000126FDF7FDF90698FCF7A9FE1EB136E0E1
:1041B00001F0A6F97AE714F0020F14D01C481B4B4B
:1041C0004FF0100501781B481A46007848434FF01D
:1041D000000108D032F911C09CFBF5FC23F811C096
:1041E000491C8842F6D814F0010F18BF14F0100FC4
:1041F00015D01248DFF840C04FF010020178104887
:104200006346007809184FF0000008D033F91040D9
:1042100094FBF2F42CF81040401C8142F6D807B011
:104220003046BDE8F08F0120704700009C48002018
:10423000A1400020A24000200C550020A3400020F7
:10424000A4400020FE480078012818BF00207047D5
:104250002DE9FF4FFB4881B0984690F800A0FA483E
:1042600091468B460026057804240E9F06F08DF8B3
:1042700001465FEA0800DFF8C88328D12A1F2046DC
:10428000042AC8BF2A1B09DD31F91030142B01DBC9
:10429000012603E0401C00B29042F5DBB7F1FF3F7E
:1042A00018BF002E13D1B9F1000F10D00198FFF7FD
:1042B0006EFB98F80200052898BF401C08D9281BFF
:1042C00000902346524600215846FFF72BFE00205F
:1042D00088F8020005B0BDE8F08FD948C079012800
:1042E00018BF002070470021D54841720172704705
:1042F0002DE9F05F05468A46408829880024401A47
:1043000001B205EB4A00274630F8042C30F8020CC5
:10431000A046101AA3462646A14600B20829A8BF07
:10432000082807DB08F0DCFA002804BF0123AAF103
:10433000020002D00023AAF1010001B218468B420C
:104340002ADC35F910204245C4BF904600F0FF0931
:1043500098421DDD05EB400C3CF902CCACEB0202AF
:10436000D21D0E2A05D804F1010C0CF0FF0488427E
:104370000ED1A7420BD22746884203D10E2A98BFFE
:1043800046B201D9421E56B2F21B4FFA82FB0024FC
:10439000401C80B28142D4DAAAF10400874205DDD4
:1043A000CB45DEBFB1450020BDE8F09F0120BDE850
:1043B000F09F70B5A64AA54906461478097800EB27
:1043C00044021046FFF794FF054621463046FFF7AA
:1043D0008FFF00229A49002D1CBF00284A7208D185
:1043E000487A401CC0B248720A2882BF4A72002034
:1043F00070BD012070BD2DE9F34F91498BB00020B5
:104400000870DDE90B1202AB009303AB089304AB19
:10441000079305AB06938D4B8046C1461B780993E5
:104420008B4BB1F90050B2F9007093F800A02C4604
:1044300031F91AC032F91A60ADF80C00ADF8140069
:1044400001206346ADF808A0ADF810A0BAF1010F45
:1044500033DD31F910B0AB45C8BF5D4632F910E02D
:10446000BE45B8BF7746A34504DA5C46DDF818B010
:10447000ABF8000001EB400B3BF902BCCDF804B0F7
:1044800031F910E0BBEB0E0B44BFDDF804B0AEEB2E
:104490000B0B0FFA8BFBC3450BDDD846DDF804B0E0
:1044A000F345D4BF8346A0F1010BDDF820E0AEF860
:1044B00000B0401C00B28245CBDCDDF824B00AF12C
:1044C0000100DA44CDF804A082452FDD31F910A0B7
:1044D000E245C8BFD44632F910B0B345B8BF5E4616
:1044E0009A4504DA5346DDF81CA0AAF8000001EB57
:1044F000400A31F910B03AF902ECBEEB0B0A48BFA2
:10450000ABEB0E0A0FFA8AFACA4509DDD146DE4541
:10451000D4BF8246A0F1010ADDF800B0ABF800A0DC
:10452000401CDDF804A000B28245CFDC4FF0010A48
:1045300016F5967FB8BF17F5967F0BDA4049C87914
:1045400060B98879401CC0B288710A2888BF81F898
:1045500007A003E03A4900208871C8713D48ACEBE0
:104560000303006890F81F118B42C4BF2B1B8B42C2
:1045700005DD90F81E114945B8BF414520DB009983
:10458000B0F91C01B1F9001032F91110884217DBA3
:104590000799B1F9001032F9113041428B420FDB1B
:1045A000089BB3F9003032F91330984208DB0698C3
:1045B000B0F9000032F910008142D8BF002400DDBC
:1045C0005446CCB1BDF91410BDF91000CDE900017D
:1045D000BDF90C30BDF90820DDE90B0100F034FE17
:1045E000012808BF4FF0FF340B98FFF7E2FE0028C8
:1045F00008BF4FF0FF3484E0114900204872087270
:1046000010480C9A0678104890F80080002000901E
:10461000B2F90010B2F902C0054602EB4803B1EB53
:104620000C0048BFACEB01000FFA80FC0027012111
:10463000A8F1010BBBF1010F26DD32F911E00BE00F
:10464000844000209E4000209F400020A340002086
:10465000A44000209441002002EB4100B0F90290F8
:10466000BEEB090048BFA9EB0E0000B26045C4BF15
:1046700084464FB2481CC1B25945DEDB002F1CBF37
:10468000A8F10200874203D1BCF1190FC8BF012570
:10469000B3F90010B3F90220881A48BF501A02B2C9
:1046A0000121A6F101094FF00008B9F1010F1ADD4F
:1046B00003EB410033F911C0B0F90270BCEB070005
:1046C00048BFA7EB0C0000B29042C4BF02464FFAAD
:1046D00081F8481CC1B24945EADBB8F1000F1CBFA4
:1046E000B01E804501D1192A04DC0098002808BFBB
:1046F000002D03D0FE4880F801A002E0FC49002014
:1047000048700DB02046BDE8F08F2DE9F04FDFF87E
:10471000E493064685B0D9F8000090F824110029EA
:104720001CBFB0F8380100280AD0FDF74CF9D9F8C1
:10473000001091F82411B0FBF1F201FB120018B146
:1047400005B00120BDE8F08F02F0ACF90546FFF797
:1047500038F90446D9F80000002DB0F93811049159
:10476000B0F93A7168D0E4480078102804BF2846B0
:1047700004F060FDE1484FF00008002C0378E048A9
:1047800002781FBF002113EB020CD9F80000B0F82B
:10479000289109D034F9020B0028B8BF404248459F
:1047A0004CDC491C8C45F5D8CDE90082C64600207A
:1047B000CDE902235DF820A002AA06EB4A0352F8D5
:1047C00020B033F9024B4FF000080121C146A44646
:1047D000BBF1010F0CD933F9022B9442BCBF144634
:1047E00089469445C4BF94468846491C8B45F2D8F7
:1047F000A4EB0C010AB204998A421ADB0AEB090104
:104800000AEB080335F8111035F81330C91A511A9C
:1048100009B20029B4BF4B420B46002AB8BF52422E
:10482000934206DA0029B8BF4942B94201DAF0469C
:1048300004E0401C0228BDD34FF00108B8F1000F7E
:1048400008BF02F039F9404605B0BDE8F08FA8482E
:1048500000214A1E8172C172C2810282418281821C
:104860007047A348C0787047A149C8707047F0B43A
:104870009F4D4FF0000CB5F90E40EE788C420AD1F6
:10488000B5F912409C42B8BF6B8204DBB3EB640FF6
:10489000B8BF4FF0010CB5F910400027844208D191
:1048A000B5F914409442B8BFAA8202DBB2EB640FA0
:1048B00002DBBCF1000F0AD0E87A401CC0B2E872FB
:1048C000B04281BFEF720120F0BC704704E0EF728C
:1048D0006B82AA82E9812882F0BC002070472DE912
:1048E000F04F894685490446B0F900300D78844977
:1048F0004FF0010C0F7800EB47060020B6F90020BE
:10490000014683468246012F0BDD34F91C80984511
:10491000C4BF434661460CF1010C0FFA8CFCBC4548
:10492000F3DB0124012D0BDD36F914C09445C4BF1F
:104930006246204604F1010C0FFA8CF4AC42F3DB22
:10494000DFF8B0C10026002FDCF800C0C8BFBCF9FA
:1049500034400CDD06FB050839F91880A04502DD5E
:104960004FF0010B03E0761C36B2B742F2DC0026B2
:10497000002DC8BFBCF934C00CDD01FB056439F95A
:104980001440644502DD4FF0010A03E0741C26B2B6
:10499000B542F2DC564CBBF1000F1EBFBAF1000F5E
:1049A0004FF0000C84F80AC007D0FFF760FF012821
:1049B00018BF00200CD0BDE8F08F94F80AC00CF1AD
:1049C000010C0CF0FF0C84F80AC0BCF1050FECD907
:1049D000FFF73DFF0120BDE8F08F45490020087337
:1049E0007047434800797047414908717047F0B4F7
:1049F00044493F4F00230A7843493E7991F800C06B
:104A0000194602FB0CF4002C14DD3A4A1268958E0C
:104A100030F91120002AB4BFC2F1000C9446AC4515
:104A200004DD1D323A2A9CBF5A1C93B2491C89B23C
:104A30008C42EDDC0021B3EB640FD8BF397309DD84
:104A4000387B401CC0B23873B04281BF397301203B
:104A5000F0BC70470020F0BC7047F0B5174600244A
:104A6000234D1E460A468446012804BFE8790128E2
:104A700005D0FFF7ECFEBCF1010F07D007E0394687
:104A80001046FFF72CFF002818BF01241EB100209C
:104A900028732046F0BD3846FFF7A9FF002818BF4D
:104AA0000124F6E72DE9F04F97B0054600200F905E
:104AB00014480F46047814480078039000200490AE
:104AC00007F0E3FE18B10EF082FC01282DD0264637
:104AD00000200C900A904FF0060A81460E90804606
:104AE0000590069007904FF00C0B08900EE0000028
:104AF000844000209441002012410020A340002067
:104B0000A44000209E4000209F4000206FF00B003A
:104B10000B90FEF759FF0D9007F0B7FE002844D028
:104B20000EF055FC082806D03FE0FE48006890F8DB
:104B30003D01461CCCE70398A0428CBF401E601E7E
:104B4000C2B20398844234BF601E401EC1B2501EE0
:104B5000C0B20423CDE900300292002309A804F07A
:104B60002BFF9DF825109DF82700884228BF0023C1
:104B700019D39DF824009DF8262082420DD301FB15
:104B80000402DDF834C0401CC0B22CF8123027F803
:104B900012309DF826208242F1D2481CC1B29DF805
:104BA00027008842E5D20220049010A9384605F07B
:104BB000BEFA00B258454ADDDDE90302A0EB020C63
:104BC000944568DD0021002E3CD902FB041083B21D
:104BD00037F913000028B8BF404258452EDD35F99B
:104BE000130058450ADD069B9842C4BF0891CDE9E1
:104BF00006020C9B5B1C1BB20C9306E00B9B9842BD
:104C0000BCBF09F101030FFA83F90E9B5B1C9BB239
:104C10000E930028B4BF43420346DDF828E09E45CA
:104C20000CDA0028ACBF034643429B4506DA002855
:104C3000B8BF404200B2059190460A90481C81B22C
:104C4000B142C2D3501C82B29445BBDC23E0DDE903
:104C50000301A0EB010C8C451DDD0020002E16D9B0
:104C600001FB040293B237F91320002AB8BF524265
:104C70005A4508DD35F913300B9A9A42C4BF09F141
:104C800001020FFA82F9401C80B2B042E8D3481CFE
:104C900081B28C45E1DC0C9850EA09001DD00C98DB
:104CA000002821D040F3478107F0EFFD78B10EF0E6
:104CB0008EFB082824D00EF08AFB012820D00EF0AD
:104CC00086FB09281CD00EF082FB0A2818D09648D3
:104CD0000078012814D000F02EB9934900204873C1
:104CE000487117B0BDE8F08FB9F1000F40F3238190
:104CF0008D4900204873487117B0401EBDE8F08F01
:104D0000601E00F0FF090EF062FB092803D00EF0D0
:104D10005EFB0A280AD10598142807D3484505D810
:104D2000DDE90780059001200F9001E00F98D0B1D8
:104D30000598A6F1010C08FB0400002335F91010BA
:104D400005981FFA8CF288B308FB04091FFA89F949
:104D5000002970DD05EB490939F9029CCA456ADD75
:104D6000401E83B26BE00598A6F1010908FB040020
:104D7000002335F910C005981FFA89F260B308FBCB
:104D8000040189B2BCF1000F11DD35F911B005EB5A
:104D9000410131F9021CBBEB010B04D40029B8BF5F
:104DA0004942514514DA401E83B215E047E00FDA5C
:104DB00035F911B005EB410131F9021CABEB010BE8
:104DC000BBF1000FEFDC0029B8BF49425145EADBD7
:104DD000401E0004000CD2D10598484545DA08FB76
:104DE000040189B2BCF1000F0EDD35F911B005EBFD
:104DF0004101B1F90210BBEB010B2FD40029B8BF60
:104E0000494251452ADB10E00FDA35F911B005EBC4
:104E10004101B1F90210ABEB010BBBF1000F1DDC3E
:104E20000029B8BF4942514518DB401C80B24845B3
:104E3000D5DB1AE0FFE7401E0004000C84D1059882
:104E4000604512DA08FB04091FFA89F9002908DD18
:104E500005EB4909B9F90290CA4502DD401C82B24E
:104E600003E0401C80B26045ECDB059808FB0400C1
:104E700081B208FB043083B208FB04200D9A1FFAAC
:104E800080FC0D9832F9132037F8133030F91100F7
:104E900013441DB20D9B37F8111033F91C3037F84D
:104EA0001CC0014409B29C440FFA8CFCB1EB05080C
:104EB00048BFA5EB0108B1EB0C0548BFACEB010501
:104EC00008EB05010FFA81F8811A48BF111AC21ABE
:104ED00048BF1A1A881805B20F9878B1A8452ADA7F
:104EE00011494879821E032A9CBF401C48716FD922
:104EF0000020487117B0401EBDE8F08F07F0C5FCD8
:104F000018B10EF064FA012813D0A84507DBB8EBFE
:104F1000050048BFA5EB0800B0EB4A0F0BDA4FF0D5
:104F2000FF3003E0944100208440002017B0BDE82A
:104F3000F08FA845F3DB03984FF00009C01E1FFA5D
:104F400080FB06984FEA540CC8464FF4FA65BE2819
:104F50003BDAABF102000CFB00F10E98814234DA2F
:104F6000DDE90302A0EB020E724521DA00231946A7
:104F7000002E13D902FB041080B237F910008245CD
:104F8000BEBF82285B1C9BB24045C8BF8046A8427A
:104F9000B8BF0546481C81B2B142EBD39C453CBF2B
:104FA00009F101001FFA80F9501C82B29645DDDC40
:104FB00007F06BFC48B9B8F1BE0F06DAD94504D347
:104FC00015F11E0FC8BF0320ABDCFF480221417161
:104FD0000120A6E72DE9F05FDFF8F0A38046002668
:104FE000DAF80000374690F8241100291CBFB0F809
:104FF000300100286CD0FCF7E6FCDAF8001091F8DC
:105000002411B0FBF1F201FB1200002860D101F085
:10501000B7FC5FEA00095BD0ED480078102804BFB8
:10502000484603F0F1FFEB484FF0000C444690F87F
:1050300000B0E948634690F800E0BEF1000F19DDCA
:1050400034F9020B0125BBF1010F10DD34F9022BFD
:10505000101A01B20029B8BF494208B2604502DD0A
:1050600084461E462F466D1C10465D45EEDB5B1CDC
:105070007345E5DBDAF80020B2F83001844527DB20
:1050800006FB0B7008EB400338F8101033F8023CB5
:10509000C91A39F8103009EB400009B230F8020C97
:1050A000181A081A00B20028B4BF43420346002968
:1050B000B8BF49428B420BDA0028B8BF4042B2F871
:1050C0003211884204DA01F0F7FC0020BDE8F09FBD
:1050D0000120BDE8F09F70B515460E46044607F066
:1050E0001BFB002C18BF70BD042818BF052806D074
:1050F000B648006890F82400A84288BF70BD3046CA
:10510000BDE8704015F05ABD2DE9F84F1E46DDE9A7
:105110000A7B90460C46054607F0FEFA824607F0E9
:10512000B4FBDFF8A49278B10EF051F908284FD003
:105130000EF04DF901284BD00EF049F9092847D05F
:105140000EF045F90A2843D0002E41D007F09DFB10
:1051500040BB38460C99CDF800B00027234601F03B
:10516000FF0B012C04BF99F80710012904D0FFF7A9
:105170006EFB012B06D008E00099FFF7B0FB00287A
:1051800018BF0127BBF1000F06D0002089F80C00E2
:1051900047B14FF0FF340FE00098FFF728FC0028DC
:1051A000F7D1F5E7012C07D199F8000001281CBFC1
:1051B000002DB5F1FF3F0BD007F067FB80B10EF07B
:1051C00006F9092806D00EF002F90A2802D007E0F5
:1051D0002C46F1E707F089FB012808BF4FF0FF34A8
:1051E000B4F1FF3F0CD0002C18BFBDE8F88FBAF126
:1051F000040F18BFBAF1050F17D00D9878B114E05D
:10520000B8F1000F1CBF4046FEF708FC002E08BF97
:10521000BDE8F88F3046BDE8F84FFEF7B8BB99F807
:105220000700012818BFBDE8F88FB8F1000F1CBFB8
:105230004046FEF7CBFB002E08BFBDE8F88F304696
:10524000BDE8F84F15F09ABC2DE9FF4F0E46044615
:10525000634962488BB091F800B00078002158444F
:105260000690401ECDE904B0ABF10100CDE902107B
:105270000D9888468A4634F9100008900E988946A1
:10528000474634F91000009101910790FEF77DFB2D
:1052900005460020014609904B48407801280AD075
:1052A0000E98814222DC34F91030079AB3EBA20F3A
:1052B00018DA02901AE00E98022102280BDB0E98F1
:1052C000ABF10302824206DB0698C21E0D988242B1
:1052D000A8BF0228E4DA3C48012101700FB0002089
:1052E000BDE8F08F401E00B28142DCDD0E98ABEBD2
:1052F000010282420BDD34F910C0079BBCEBA30F07
:1053000001DA039003E0401C00B29042F3DB0D98F9
:105310000BEB010282420BDC34F910C0089BBCEBA2
:10532000A30F01DA049003E0401E00B28242F3DDD5
:10533000069A0D98511A81420BDD34F91030089A03
:10534000B3EBA20F01DA059003E0401C00B28842E3
:10535000F3DBDDE9042082422ADA06EB420036F96B
:105360001230B0F90210581A48BFC81A01990844FF
:1053700000B2019005EB420035F91210B0F902308D
:10538000C81A48BF581A0099084400B2009004EBAC
:10539000420034F91230B0F90210581A48BFC81A46
:1053A00050440FFA80FA501C02B205988242D4DBB6
:1053B000DDE90201884236DA06EB400136F91030A9
:1053C000B1F90220991A0DE0844000209441002098
:1053D0000D4100209E4000209F400020A34000205F
:1053E000A440002048BFD11A41440FFA81F805EBD0
:1053F000400135F91020B1F90230D11A48BF991A8D
:1054000049440FFA81F904EB400134F91020B1F955
:105410000230D11A48BF991A39440FB2401C03997F
:1054200000B28842C8DBDDE90010081A0024B0EBA6
:105430006A0FDCBFA9EB0800B0EB670F16DC07F0C2
:105440004FFA68B9189835F9101010480068B0F98B
:105450001C0181420ADC199935F91110814205DCE1
:105460000998002804BF0A4804720BD00849087A3A
:10547000401CC0B20872032881BF0C7201200FB01B
:10548000BDE8F08F00200FB0BDE8F08F9441002000
:105490008440002010B505F0BBFB05F045FC002062
:1054A00010BD0000FE4800787047FD4800780228D3
:1054B00005D005281CBF0020704704F05AB907F03A
:1054C0002BB9F7490870704710B50446062C28BF61
:1054D00010BDDFE804F01203070F120B084600F0BE
:1054E00013FA0AE0084607F00CF906E0084604F053
:1054F00035F902E0084606F0A3FEE948047010BD45
:10550000E84900200968B1F8641011F4807F08BFF1
:105510007047FDF756B8E34900200968B1F86410F8
:1055200011F4807F08BF7047FDF760B8DD490020A7
:105530000968B1F8641011F4007F08BF704715F0D6
:105540003DBAD84900200968B1F8641011F4806FA1
:1055500008BF704715F071BAD149487800281CBFC0
:10556000401E4870704770B5CF490868D0F8CC002D
:10557000CB4C10F0030F0BD0096840F4BE0040F094
:105580002040C1F8C8006078002804BF0120607086
:10559000C64800688068C34D10F0020F296807D123
:1055A000C3480068406910F0010F01D0607840B135
:1055B000B1F86410002011F4807F18BFFDF716F8D1
:1055C00007E0B1F86410002011F4806F18BF15F0E7
:1055D00034FAB849084208BF70BD2968496E090C01
:1055E000617070BD10B572B6FEF74EF9BDE810409F
:1055F000FDF7DDBE10B54FF42F30FDF7ABF872B6F6
:10560000FEF742F9BDE81040FDF7D1BEA44800699D
:105610007047A348C0687047A14948617047A048D7
:10562000406970479E49886170479D48806970470E
:105630009C48026802F5B073118A508A02F5A07284
:10564000FCF716BA2DE9F04FDFF8549295B00E46EC
:10565000C9F8100005F042FAC9F80C0000287DD006
:1056600090F800C089F802C0417889F80310837867
:1056700004460CF1010089F8043000F0FE0089F8BE
:105680000500E27889F80620207989F8070060791A
:1056900089F8080009F10A004FF0000B80F800B00B
:1056A00080F801B0207889F809006046FCF7F2FA2A
:1056B00099F8081099F80700FCF707FB694620469F
:1056C00005F029FA608AD9F8145000281CBF6843F5
:1056D000050B678BD9F81880002F08BF4FF480574F
:1056E0004FF4805A002016F0020F18BF112016F058
:1056F000040F18BF40F00A0016F0080F18BF40F062
:10570000040016F0010F18BF40F02000616A01EAA2
:105710000006009810900498119008981290019833
:105720001390CDF850B010A93046FCF720F816F0D1
:10573000020F72D004F0DFFE5FEA000B35D004F0F8
:10574000F1FE6843050B59460020FBF704FC218A53
:1057500000291CBF0020FBF74CFC00E018E004F01F
:1057600001FF08FB00F0000B00F50060020A0820B2
:10577000012101FA00F3134201D1401EF9D5A0F135
:105780000408A07B002818BFA0F1010B17D112E07C
:1057900044480068B0F8640010F4807F18BFFCF73C
:1057A00025FF002015B0BDE8F08FB4F80CB0BBF1B8
:1057B000000FC8D1CBE70020FBF799FC8346E07BC4
:1057C000002814BF401EFBF7C1FC0BEB08010429A5
:1057D00005DDA8EB010101F10408042104E0002922
:1057E000BCBFA8EB010800218044B8F1040F05DD1F
:1057F000A8F10400C5404FF0040807E0B8F1000F1D
:1058000004DAC8F1000085404FF000080020FBF7E3
:1058100084FC41460020FBF7AFFC16F0010F30D0AE
:10582000A18A00291CBF0120FBF795FBB4F8188062
:10583000B8F1000F07D041460120FBF7DAFB4146E3
:105840001120FBF7D6FB94F81680B8F1000F09D0B1
:10585000A8F101010120FBF760FCA8F10101112072
:10586000FBF75BFC94F81780B8F1000F09D0A8F1A2
:1058700001010120FBF780FCA8F101011120FBF7D9
:105880007BFCE07A00281CBF0001FBF7DEFA0298DF
:1058900004F087F8039898B12B4699F803200BE0A1
:1058A0009C400020944100203CE3010040E30100C3
:1058B00034E301000800030099F8021004F0A8F88E
:1058C00052463946284604F058F90598FEF760FB21
:1058D000069800F0D1FF16F0100F05D00998FEF7DA
:1058E000A4FB0A9801F056F815B00120BDE8F08F2E
:1058F00010B5FBF7E4FF04F05CF802490020C86033
:10590000012010BD9C400020FE4948707047FD48B2
:1059100040787047FC4810B4FC4A0168914218D1A5
:105920004168B1F5887F14D80022D0F808C003463A
:105930001146B2EB9C0F24BF10BC704753F82140B6
:10594000491C2244B1EB9C0FF8D3002A04BF10BCC1
:105950007047002010BC7047EB48FCF7FBBEE949DC
:10596000012048707047E7490020087070472DE912
:10597000F34FDDB000208A4646904D904C9072B6B1
:10598000FBF7DAFF0546FDF70EFE48B1FDF7E5FE31
:105990004D90FDF7C2FEFDF7E6FE4C90FDF7CDFE03
:1059A000FBF7D6FEFBF7FAFD5690FBF7C8FF5590C4
:1059B000FBF7F6FDFDF7B7FB5490FDF798FB4FF4AE
:1059C0009350FDF710FB62B60022914630AE46F8C8
:1059D0002290521C062AFAD3CD4F15F0020F4FF039
:1059E000010407D0309438684FF4E76100F5804037
:1059F00014F07FFEC64A15F0010F44F238701268A9
:105A000002EB000510D04FF4E071284614F071FE4F
:105A10000120FAF7F9FD002818BF32941120FAF797
:105A2000F3FD002818BF3394DFF8E8B2DFF8D48222
:105A3000309868B30020FBF74DFB00909BF8000006
:105A40008DF80400B4480078012894BFB348B448E6
:105A500000788DF805000020FBF70AFC002818BF2D
:105A60004FF0FF3003908DF806A0B8F80400ADF8B1
:105A700008000020FBF7D8FAADF80A00386800F5F6
:105A80008040059038680690386800F5005007900F
:105A900031984FF0FF0A48B30020FBF71BFB08903A
:105AA0009BF800008DF824008DF82540CDF82C904F
:105AB0008DF826A0B8F80400ADF828000020FBF708
:105AC000B3FAADF82A009DF805003A68C0EBC001B2
:105AD00002EBC10101F580410D919DF8041048438E
:105AE00002EB40000E9000F500500F90DFF834926A
:105AF000DFF834B2329870B30120FBF7EBFA109064
:105B0000FBF74FF800280CBF9BF8000099F8000045
:105B10008DF844000120FBF7EAFA04FA00F08DF852
:105B200045000120FBF796FBC04313908DF846A07B
:105B3000B8F80600ADF848000120FBF775FAADF89B
:105B40004A001595386842F2204100F584601690AD
:105B5000386808441790339890B31120FBF7BAFACD
:105B60001890FBF71EF800280CBF99F800009BF86E
:105B700000008DF864001120FBF7B9FA04FA00F078
:105B80008DF865001120FBF765FBC0431B908DF875
:105B900066A0B8F80600ADF868001120FBF744FADB
:105BA000ADF86A00386844F2A87108441D9038685E
:105BB00042F2206100F5C4601E90386808441F90CE
:105BC0009DF845100220022988BF8DF845009DF8F8
:105BD0006510022988BF8DF865004FF055301B9085
:105BE0001390FBF731FB57900120FBF71EFB0120C0
:105BF000FBF754FB5A900020FBF717FD599000204B
:105C0000FBF708FD58900020FBF779F95B90FBF754
:105C1000B4FE00204890499037903E904698002866
:105C200040F0D18302F0EEFE012800F0CC834998C9
:105C3000802800F2C88340A8FCF758F8002800F03C
:105C4000BC8340A803F022FC4898401C489000F018
:105C5000AB83002048904998401C4990002038AA06
:105C6000012142F82010401C0628F8D3379800285C
:105C700008BF369013D0012804BF0020369000F0F2
:105C80000181022804BF0020369000F034820328EE
:105C900004BF0120469000F0668300F094BB369963
:105CA00030A850F8210000287CD0369A684600EBD6
:105CB00042100022479207794279D0F800803F9243
:105CC000B0F9086042694B923E998269C068C1F19F
:105CD00004054A90A9B1002D65DB3F984FF00009FB
:105CE00000287DD905F10800012101FA00FBE81D1B
:105CF00001FA00F0509001234A9803FA09F1084094
:105D000014E01EE0B840002000AF020054435246A9
:105D100050E30100A1400020A04000209F4000204F
:105D2000A2400020A3400020A440002018BF012072
:105D3000002151904B98C9EBC9038C4600EBC30A74
:105D400087E03F984FF0000A002849D901214A987E
:105D500001FA0AF3034214BF4FF0010E4FF0000E98
:105D600000204B99CAEBCA03844601EBC30B30E019
:105D70000121814011EA080F28D041084FEA194358
:105D80004E915BF82190C1074FEA0343CC0E29FAEC
:105D900004F132F9023B89B29B1B0CF1010CBEF1FC
:105DA000000F01E066E060E018BF5B42002BC8BF57
:105DB00041F4805141F400614FF6FF73A34029EA9A
:105DC0000303A1400B434E994BF82130401C1C2883
:105DD00001D2BC45CCD33F980AF1010A824500E0CC
:105DE0003FE0B3D33DE00120884010EA080F2DD0FA
:105DF00048084F905AF82000CB07DC0E4E90E04048
:105E000032F9023BDDF844E19B1B80B20CF1010C3E
:105E1000BEF1000F18BF5B4210F4805F02D0002B70
:105E200004DA01E0002B01DD20EA0B00002DC4BFE5
:105E3000509B18434FF6FF7E0EFA04FE4E9BA04087
:105E400023EA0E0303434F984AF82030491C1C29CB
:105E500001D2BC45C7D33F9809F101098145FFF440
:105E60004AAF002D04BF0120479038A9369A4798C1
:105E700041F822003698401C36900628FFF40FAFF8
:105E800000F071BA369930A850F82100002800F0CF
:105E90002A81369A684600EB421000224E9204791D
:105EA0004679837905684793B0F9088042694A9238
:105EB000C368826950934089479B3E991840C1F15D
:105EC00008074F90E9B1002F77DB4FF0000A002E52
:105ED00072D90120B8404B90781E012101FA00F0E0
:105EE00053900123509803FA0AF1084018BF01208B
:105EF00000213F904A98CAEBCA038C4600EBC30BC3
:105F000095E04FF0000A002E56D90123509803FA6D
:105F10000AF1084018BF012000213F904A98CAEBBF
:105F2000CA038C4600EBC30B40E0012088402842A6
:105F300039D0480851905BF82000CB074FEAD3696D
:105F40004B9020FA09F032F9023BDDF8FCE080B218
:105F5000A3EB08030CF1010CBEF1000F18BF5B426C
:105F600010F4805F09D0002B0EDA10F4706018BFB7
:105F7000A0F5807040F4805006E0002B04DD10F4A2
:105F8000706018BFA0F5807040F080004FF6FF7E73
:105F90004B9B0EFA09FE23EA0E0300FA09F00343B5
:105FA00051984BF82030491C1C2901D2A445BCD380
:105FB0000AF1010AB245A8D340E043E0012088403D
:105FC000284231D0480852905BF82000CB074FEAB6
:105FD000D369519020FA09F032F9023BDDF8FCE078
:105FE00080B2A3EB08030CF1010CBEF1000F18BF47
:105FF0005B4210F4805F02D0002B04DA01E0002B3A
:1060000001DD4B9B9843002FC4BF539B18434FF6B1
:10601000FF7E519B0EFA09FE23EA0E0300FA09F0F7
:10602000034352984BF82030491C1C2901D2A44547
:10603000C4D30AF1010AB245FFF453AF002FC8BF21
:106040004E984CDC4FF0000A002E46D94798C0F518
:1060500080703F90479840F4807B4A990020CAEBBB
:10606000CA034FEA174C02464FEA0C4C01EBC30936
:106070002DE001218140294226D04FEA5008C10776
:1060800059F82870CB0E27FA03F11FFA81FCDDF8CE
:10609000FCE00CF0FF0101EB5E01DDF83CE101EA00
:1060A0000B01521C714588BF71462CF0FF0C4CEA65
:1060B00001014FF6FF7C0CFA03FC27EA0C0C994017
:1060C0004CEA010149F82810401C1C2801D2A242C8
:1060D000CFD30AF1010AB245BFD301204E90369AC0
:1060E00038A941F822003698401C36900628FFF463
:1060F000C9AE00F038B9369930A850F82100002810
:1061000000F02B813E985290684600EB4110002130
:106110004E91016850910179479141793F91817980
:10612000B0F9089042695192D0E906844289C0686A
:106130004F905298C1F5807602EA010710F0010FE6
:1061400015D03F984FF0000B00287DD901214F98C2
:1061500001FA0BF2104018BF01204A905199CBEB85
:10616000CB02002001EBC20182464B91E2E000200D
:10617000FBF794F8054647993F984143032000EB0D
:10618000410020F003024146204614F0B7FA2846A9
:10619000FBF784F83F984FF0000B002854D90122F8
:1061A0004F9802FA0BF1084018BF012000214A90D5
:1061B0005198CBEBCB020D4600EBC20E50E0012014
:1061C00000FA01F25098024247D038F9020B6D1CD8
:1061D000A0EB09034A98002818BF5B424808539077
:1061E0005EF82000CA074FEAD26A4B9020FA0AF004
:1061F00082B2C2F3032002F0FF0C12F4805F02D0DF
:10620000002B02DB04E0002B02DDACEB060401E016
:106210000CEB0604BC4205DD0F28AEBF3C46002453
:10622000401C06E0002C04DA0028C6BF3C46401E95
:10623000002402F4805242EA00204FF6FF7220430D
:1062400002FA0AF24B9B00E07DE023EA020200FA28
:106250000AF0024353984EF82020491C1C2902D210
:1062600047988542ABD33F980BF1010B834596D3FA
:1062700069E0012101FA00F250990A4257D034F93D
:10628000021B4A9AA1EB09010AF1010A002A18BF70
:10629000494238F9022BA2EB090218BF52420029E9
:1062A000B4BF4B420B46002AB8BF52429A423ED975
:1062B0004B9B4208539253F82220C3074FEAD36EF8
:1062C0005C9222FA0EF293B2C3F3032203F0FF0CA6
:1062D00013F4805F02D0002902DB04E0002902DD14
:1062E0000CEB060501E0ACEB0605BD4205DD0F2A0F
:1062F000AEBF3D460025521C06E0002D04DA002A00
:10630000C6BF3D46521E002503F4805141EA0221DA
:1063100029434FF6FF735C9A03FA0EF39A4301FA8E
:106320000EF142EA0103539A4B9941F82230401C86
:106330001C2802D247998A459BD33F980BF1010B49
:106340008345FFF403AF5298032826BF01204E90E7
:106350004E9838A9369A41F822003698401C36905B
:106360000628FFF4C8AE0123002038A951F82020E8
:10637000EAB1401C0628F9D3CBB137981F2811D2B7
:10638000401C012101FA00F237905D98024209D1C8
:106390003798401C3790032804D801FA00F25D9822
:1063A0000242F5D000203E90469818B10BE03E988E
:1063B000401CF8E7FBF7E1FA34E4FFF7ACF8469845
:1063C00000283FF42FACFBF7EBF85798FAF72DFFB6
:1063D0005A98FAF763FF5998FBF727F95898FBF793
:1063E00019F95B98FAF78BFD569830B1559810B1B2
:1063F000FBF7C3FA01E0FBF7A8FAFDF7D4F848B1C0
:106400004D98002818BFFDF7D4F84C98002818BF05
:10641000FDF71BF95498002818BFFCF72AFE469890
:1064200000280CBF012000205FB0BDE8F08F2DE9EF
:10643000F04FADF2047D4FF0000807464646CDF818
:106440000087E5E0304604F049FB00287ED0008953
:1064500000EA070424F0CC0030F47C4076D00F2111
:106460003046FFF7EFF8002870D0FBF765FA0546D5
:10647000DDF8000700286AD105F00E00FBF764F98B
:1064800003210020FAF789FEDDF8000700285ED11D
:1064900014F0010F1ED0FF210F20FFF768FACDF88E
:1064A0000007FBF77DF8DDF8000700284FD1FFF764
:1064B000B0F88146EA464FF0040B5046FBF750FC1B
:1064C00099F92C105246584604F047FBDDF80007B6
:1064D00000283CD114F0060F33D0FDF7C5FDCDF8F0
:1064E0000007FBF75DF8DDF8000700282FD114F056
:1064F000020F11D0FDF768FA8146FFF78AF80523ED
:106500005FEA090204D090F92D10184604F025FB2B
:10651000DDF80007002878D114F0040F11D0FDF742
:1065200053FA8146FFF775F806235FEA090204D0A3
:1065300090F92E10184604F010FBDDF80007002833
:1065400063D105F01100FBF7FFF801E05FE04DE0DB
:10655000DDF80007002858D114F0100F1DD0FF21DE
:106560000F20FFF704FACDF80007FBF719F8DDF864
:106570000007D8BBFFF74DF88146EA464FF0080BFD
:1065800051460120FBF730FC99F93010524658462D
:1065900004F0E3FADDF8000740BB14F0600F34D0DC
:1065A000FDF762FDCDF80007FAF7FAFFDDF8000706
:1065B000E0B914F0200F13D015F0100018BFFDF74C
:1065C000E4F98146FFF725F809235FEA090204D0C0
:1065D00090F93110184604F0C0FADDF8000728B928
:1065E00014F0400F11D015F0100000E00DE018BFBE
:1065F000FDF7CBF90446FFF70CF80A23220004D07C
:1066000090F93210184604F0A8FAFFF771F9761CD9
:1066100004F060FAB04204D9DDF8000700283FF426
:1066200011AFFE4880F80080DDF8000700280CBF9D
:10663000012000200DF2047DBDE8F08F2DE9F04F20
:10664000F648CDB04478FEF72DFF012870D1F4480C
:106650000068B0F93610B0F9340003F065FD14F0AD
:10666000020F7CD00DF5807BFFF754F90025ED4F2C
:1066700030264FF488784FF050094FF0FF3A78B148
:10668000B0E80E108BE80E10B0E80E100DF5887B08
:106690008BE80E100FC80DF5907B8BE80F0013E010
:1066A000FF223021584614F02EF8CDE94495CDE96B
:1066B0004265CDF82CA1CDF828A1CDF824A14695AE
:1066C000CDE9475ACDE94078DFF85CB35846FCF78E
:1066D00041F84598401C459040F27770FFF7A7FEBF
:1066E000012803D1FDF79FFD012817D0479800220C
:1066F000401C47901F21CDF81091022005F0DFFCCF
:106700000DF5807904F0CAF998B181694891C169A1
:10671000499141694A91C0684B9012E014F0080F0A
:1067200014BFA220A12044904698401C4690E7E761
:106730004EE0CDF82CA1CDF828A1CDF824A1CDF8BC
:1067400020A1CDE94265CDE940780021D9F8083093
:106750004A46084652F820C0401C614400E01FE051
:10676000B0EB930FF6D34D42FF22511C6846C9F897
:106770000C5013F0C8FFD9F80820F9E804018DE89F
:106780002700B9E80F0004AD85E80F0099E80F0075
:1067900008AD85E80F0058466946FCF744F810E05C
:1067A00014F0010F0DD040F22220FFF740FE012827
:1067B00008BFFDF738FD20B901221F21022005F096
:1067C0007EFCFDF79CFB01212246084605F077FC84
:1067D0004DB0BDE8F04F02F011B990498880704784
:1067E0008E49C880704770B50126FFF793F820B135
:1067F0000069A12818BFA22801D0002070BD002484
:1068000004F068F9002831D9204604F067F900281F
:106810001EBF058925F0CC0030F47C4021D00F212B
:106820002046FEF70FFFE0B115F0010F09D0FBF78E
:10683000A7FA30B944F480721E21022005F03FFC13
:10684000002615F0100F0AD00120FBF72AFB30B903
:1068500044F480521E21022005F031FC0026FFF78F
:1068600047F8641C04F036F9A042CDD8304670BD1C
:1068700000207047002070472DE9F04F674EADF2C1
:106880000C4D0028B06004BF0DF20C4DBDE8F08F38
:10689000317811F0020F6BD16449DFF898810C78E0
:1068A00063490D78C6F80C800090FDF7EBF8CDF841
:1068B0000404614890F8009060480778604890F8B8
:1068C00000A0BAF1010F8CBF0DF1040BC346DDF837
:1068D00004040099002809FB07F04FEA40024BD05E
:1068E00001A813F00BFF4B4601AA00975846DDF8AC
:1068F000041415F0B3FBBAF1010F0FD95946404605
:1069000014F062FC404509D0484A014640461378DD
:10691000474A12785A43520013F0F0FE0027F068FD
:10692000B846002D18D930F9021B0122012C0FD9CD
:1069300030F902CBACEB010109B20029B8BF4942E2
:106940000BB2BB42C8BF1F466146521CA242EFD3E6
:1069500008F10108A845E6D331480068B0F82C01D9
:10696000B842C4BF0020F060307840F002003070C0
:106970000DF20C4DBDE8F08F584613F0BFFEBAE79C
:106980002648816800291BBF017811F0020F002002
:10699000C06870472DE9F84F204E0028306108BFCD
:1069A000BDE8F88F317811F0100F18BFBDE8F88FEF
:1069B000244D824624484FF0000904782348077884
:1069C000FAF7BAFF10F0100F02D0FCF7FAFF814679
:1069D00004EB07084FEA48025146284613F08EFEA2
:1069E000B9F1000F09D00220009008F1010043081E
:1069F0002A464946104615F031FB0020B5F9003013
:106A0000A91C0122012F2AD931F902CBACEB0303D7
:106A10001BB2002BB8BF5B421BB219E0B84000208C
:106A2000944100205443524600AF02009E40002093
:106A30009F40002014560020A1400020A2400020CA
:106A4000A0400020145A0020A3400020A4400020B1
:106A50008342C8BF18466346521CBA42D4D331F9A8
:106A6000023B0122012C0FD931F902CBACEB03031D
:106A70001BB2002BB8BF5B421BB28342C8BF184693
:106A80006346521CA242EFD314490968B1F82E1193
:106A90008142C8BF00257561307840F01000307029
:106AA000BDE8F88F0E48016900291BBF017811F07D
:106AB000100F00204069704708480949006890F8A5
:106AC00025218878401CC0B28870824228BF704758
:106AD0000020887001210846FEF7F6BC9441002092
:106AE000B840002070470020704708B503F0070049
:106AF00001280AD103F088FF38B101208DF8000089
:106B0000024669460C2001F059FF002008BD08B577
:106B100003F0070001280AD103F076FF38B1002006
:106B20008DF80000012269460C2001F047FF00208B
:106B300008BD10B503F00700012808BFFEF752FD9D
:106B4000002010BD08B503F0070001280AD103F0AA
:106B50005BFF38B103208DF8000001226946022056
:106B600001F02CFF002008BD08B503F00700012844
:106B70000AD103F049FF38B10B208DF80000012243
:106B80006946022001F01AFF002008BD08B503F095
:106B9000070001280AD103F037FF38B101208DF832
:106BA000000002466946022001F008FF002008BDEF
:106BB0001FB513F0070F0BD19DF80800F0280AD07D
:106BC00003F022FF20B1012202A9082001F0F6FE05
:106BD00004B0002010BDFEF7BFFEF9E71FB513F0AB
:106BE000070F07D103F010FF20B1012202A90320F3
:106BF00001F0E4FE04B0002010BD2DE9F84F8046FE
:106C000003F007000026F84D0A9C0F46012802D029
:106C1000022806D002E00520A8702E810020BDE8E1
:106C2000F88FA878052832D12889A04227D2FCF70E
:106C300016FC4FF0AC098DF80090010A8DF8011098
:106C40008DF8020003F0E0FE90B1DFF8A0A3DAF8BF
:106C5000000003F0BEFF58B1DAF8000090F8200001
:106C600010F0020F04D08DF8019043208DF802003F
:106C700028891DF8001088F80010401C288180B277
:106C8000A04204D12E81012038700320A870012079
:106C9000BDE8F88F2DE9F04103F00702D44C002540
:106CA000D14EDDF818C0012A02D0022A56D052E097
:106CB000FCF7D5FB0521B170002122685554491C11
:106CC0000E29FADB2268AC2111702268010A51708A
:106CD0002168887003F098FE00283BD0C34F3868C5
:106CE00003F077FF002835D038682168807CC870B1
:106CF00038682268017C1171017E11F0040F0ED0FA
:106D0000C18A2268090A51712268817D9171818A44
:106D10000A0A2168CA712268017D11720DE0818A18
:106D20002268090A51712268017D9171C18A226825
:106D3000090AD1712268817D117222682021517265
:106D40002268022191722168CD7221680D73017E43
:106D50002068417335810020BDE8F081B278052AB2
:106D60000FD13289624504D223689B5C0370501CAA
:106D700030813089604504D13581012008700320BD
:106D8000B0700120BDE8F08130B403F00704984BE7
:106D9000954D029A4FF0000C012C02D0022C3AD0F3
:106DA00036E00220A8704FF42F30A5F808C0016823
:106DB000880A444211EB842418BF401C404201EB76
:106DC0008000C01C20F0030041F6E8710144B0F5DA
:106DD000283F14D8CC78086864F31F60854CA04223
:106DE0000DD10020002A13D901EB000C1C689CF87F
:106DF00004C004F800C0401C8242F5D808E000201E
:106E0000002A05D9196801F800C0401C8242F9D84F
:106E100030BC00207047AC78022C10D12C899442F1
:106E200004D21B681B5D0370601C28812889904276
:106E300005D1A5F808C0012008700320A87030BC57
:106E40000120704730B403F00704694B664D029A85
:106E50004FF0000C012C02D0022C51D04DE002204A
:106E6000A8704FF42F30A5F808C00168880A444282
:106E700011EB842418BF401C404201EB8000C01C71
:106E800020F0030141F6E8700844B1F5283F2BD803
:106E9000C478016864F31F61564CA14224D11A687A
:106EA000017C11701A68417C51701A68817C917064
:106EB0001A68C17CD1701A68017A11711968427A16
:106EC0004A711A68817A91711A68C17AD1711A6807
:106ED000017D11721A68417D51721A68817D91722B
:106EE0001968C07DC87208E00020002A05D9196819
:106EF00001F800C0401C8242F9D830BC0020704725
:106F0000AC78022C10D12C89944204D21B681B5DF2
:106F10000370601C28812889904205D1A5F808C01B
:106F2000012008700320A87030BC012070472DE9B3
:106F3000F04103F0070200262D4D2B4F069C012A3D
:106F400002D0022A3AD036E003F0A8FD40B3D0E9DF
:106F500006212B68C0681A70D5F800C0130A8CF897
:106F60000130D5F800C0130C120E8CF802302B68DB
:106F7000DA702A6811712B680A0A5A712B680A0C98
:106F8000090E9A712A68D171296808722A68010A63
:106F900051722A68010C9172010E2868C17207E0D3
:106FA0000020002C04D929680E54401C8442FAD8D1
:106FB0000220B8703E810020BDE8F081BA78022A34
:106FC0000FD13A89A24204D22B689B5C0370501CFB
:106FD00038813889A04204D13E8101200870032005
:106FE000B8700120BDE8F081D84000209441002015
:106FF00054E3010034CD12AB70B403F00703F84C36
:10700000F84D039A4FF0000C012B02D0022B50D008
:107010004CE00220A8704FF42F30A5F808C001689A
:107020000026880A434211EB832318BF401C4042CC
:1070300001EB8000C01C20F0030101F50050B1F508
:10704000283F98BF10F0030F27D1E74B0168994202
:1070500004BF0023194620D150F82150491C2B446D
:107060000729F9D303B1C6B12268017C11702268E7
:10707000417C51702168827C8A702268C17CD17009
:107080002268017D11712268417D51712268817DE4
:1070900091712168C07DC87108E00020002A05D9DF
:1070A000216801F800C0401C8242F9D870BC002061
:1070B0007047AB78022B10D12B89934204D22468FD
:1070C000E45C0470581C28812889904205D1A5F8F9
:1070D00008C0012008700320A87070BC0120704710
:1070E0002DE9F04103F007040027BE4EDDF818C07B
:1070F000012C05D013F0070F06D0022C43D03FE03F
:107100000220B07037813BE00125002412F0010F0E
:107110001FD04FF42F300168880A434211EB8323BC
:1071200018BF401C404201EB8000C01C20F003034C
:10713000B3F5283F23D800204FF40051B0EB930F54
:1071400007D251F804CB401C6444B0EB930FF8D342
:10715000ADB112F0020F0ED003F0A0FC78B182683E
:107160000021B1EB920F06D250F8043B491C1C449D
:10717000B1EB920FF8D3002D18BF346200D1376203
:107180000020BDE8F081B278022A13D1328962452D
:1071900008D2C2F10303346ADB0024FA03F303705C
:1071A000501C30813089604504D13781012008703E
:1071B0000320B0700120BDE8F08130B403F0070374
:1071C0000024DFF820C2029A012B02D0022B0BD040
:1071D00007E005208CF80200ACF8084020208CF86D
:1071E000030030BC002070479CF80230052B14D1FE
:1071F000BCF80830934205D29CF803500570581C27
:10720000ACF80800BCF80800904206D1ACF8084081
:107210000120087003208CF8020030BC0120704768
:107220002DE9F04383B003F007056D4E6D4FDDF897
:1072300028C04FF00008012D0AD013F0070F3B467D
:107240001B8903F10104A4B211D0022D22D01DE04C
:1072500001A9684601F007FE0520B8703168019861
:107260000870316800984870A7F808800EE0634500
:1072700002D23068C2543C813889604506D1A7F8F3
:10728000088030680178407801F0E4FD03B0002008
:10729000BDE8F083BA78052A0ED1634503D232687F
:1072A000D25C02703C813889604505D1A7F808801E
:1072B000012008700320B87003B00120BDE8F083FE
:1072C00070B503F007000026464C454DDDF810C0B0
:1072D000012803D013F0070F06D024E02681286888
:1072E0000670286846701EE02089604503D22B682E
:1072F0001A54401C208180B2604514D13BA0012269
:10730000006826810A702968C2B2097891420AD1C0
:107310002968C0F307204978814204D10022114630
:10732000052001F04BFB002070BD10B503F00700F5
:10733000012808BF02F076F9002010BD70B503F0F7
:107340000704284D012C09D013F0070F2B46D3F862
:1073500020C01B8908D0022C17D014E000202881FF
:1073600004F0A7FE28620EE0002B04BF1002286282
:1073700006D0012B04D14CEA0200286204F092FEF0
:107380002889401C2881002070BD002B04BF4FEAD3
:107390001C21017005D0012B03D180F800C0012011
:1073A0000870581C2881012070BD70B5064603F096
:1073B00007000C4C0D46012808BF00200DD013F02B
:1073C000070F02D0022813D008E02089002804BF4C
:1073D000104610F016FC2089401C2081002070BD52
:1073E00054E30100D84000205446495355AC0000F6
:1073F00010F004FC307001202870F0E72DE9F04710
:10740000074603F00700DFF8F4938A4601280AD004
:1074100013F0070F4B46DFF8E883FA4DDE7808D00B
:10742000022841D03DE00020A9F80800A9F80A0090
:1074300037E0B9F80800002808BF89F803202BD0EE
:10744000012804BF1002C9F8200025D0022823D14A
:10745000D9F82000104384B2C9F8200003F0D4FA10
:10746000D0B1062E18D2DFE806F00306090C10147E
:10747000A8F80E4010E0A8F80C400DE028688486BB
:107480000AE02868A0F80C4106E02868A0F85040FF
:1074900002E02868A0F85240B9F80800401CA9F89A
:1074A00008000020BDE8F087B9F80A0002282AD2B7
:1074B000002403F0A9FAD0B1062E18D2DFE806F0B6
:1074C0000306090C1014B8F80E4010E0B8F80C4090
:1074D0000DE02868848E0AE02868B0F80C4106E0C8
:1074E0002868B0F8504002E02868B0F85240B9F877
:1074F0000A00002804BF200A387004D0012802D1F5
:107500003C708AF80000B9F80A00401CA9F80A008B
:107510000120BDE8F0872DE9F0411C4615460E46D6
:10752000074603F071FA80B1B54814F0070F04D094
:1075300004F0070102290BD007E0002D1ABF90F8D4
:107540006C00C008002007F0E8FC0020BDE8F081D6
:1075500090F86C00C008387001203070BDE8F081F0
:1075600070B50D46044613F0070F04D003F0070072
:10757000022805D002E010460BF06FFF002070BD1E
:107580000BF06EFF20700120287070BD70B503F005
:10759000070200269C4C994DDDF810C0012A02D04C
:1075A000022A15D012E005F0E4F821680870FDF712
:1075B00079FF2168487002F09BFF21688870FDF711
:1075C00074FF2168C8700520A8702E81002070BD4E
:1075D000AA78052A0FD12A89624504D223689B5CC8
:1075E0000370501C28812889604504D12E81012018
:1075F00008700320A870012070BD70B5064603F026
:1076000007000D4602281CBF002070BD01F0F0F9F4
:10761000002814BF0124002401F0EDF9002814BF54
:1076200002220022224332700120287070BD70B502
:1076300003F00702744C0025704EDDF810C0012ADB
:1076400002D0022A42D03FE0FEF764F9002828D099
:107650004169FF292CBFFF21C9B2226811708169DD
:10766000FF2934BFC9B2FF2122685170C169FF29C7
:1076700034BFC9B2FF21226891702268017CD170A9
:10768000226890F820101171018C0A0A21684A7151
:10769000016A2268090C9171006A2168000EC871A4
:1076A00011E02068057020684570206885702168A9
:1076B0005020C8702168FF20087121684871216836
:1076C00088712168C8713581002070BD328962459A
:1076D00004D223689B5C0370501C30813089604564
:1076E00002D1358101200870012070BD2DE9F047DD
:1076F00003F007020026414D089C0F468046012AF0
:1077000002D0022A06D002E00520A8702E810020B7
:10771000BDE8F087A87805281AD12889DFF8E89015
:10772000002804BFD9F8000013F0FEFA2A89A2420B
:1077300006D2D9F80000805C88F80000501C28812F
:107740002889A04204D12E81012038700320A8701E
:107750000120BDE8F08770B503F007020025274C33
:10776000012A02D0022A11D00EE00520A0700021CB
:107770002581084601F077FB4FF6FF7101EA4000D2
:10778000A08101F07CFB6061002070BDA278052A19
:1077900016D12289B4F80CC0624507D212F0010F4D
:1077A0001CBFE37803700DD0501C208120896045F8
:1077B00006D12581012008700320A07001F06DFB27
:1077C000012070BD666922F00103F35A1E0A06709B
:1077D000E370E9E770B503F007020025074C012AC2
:1077E00002D0022A12D007E00520A0702581D02007
:1077F000A08101F0D5FC6061002070BDD840002060
:10780000848300209441002054E30100A278052ADB
:1078100016D12289B4F80CC0624507D212F0010FCC
:107820001CBFE37803700DD0501C20812089604577
:1078300006D12581012008700320A07001F0BEFC54
:107840000120DAE7666922F00103F35A1E0A067086
:10785000E370E9E77FB51C460E46054613F0070FB7
:1078600008D103F0D1F828B1012202A90B2001F0C0
:10787000A5F803E004F00700022802D004B00020BD
:1078800070BD04F076FF28700120307004B070BD28
:1078900010B503F00702F64C012A02D0022A0DD0DF
:1078A0000AE003F09EFA0021606200281ABF4FF43C
:1078B0000560E081E1812181002010BD2289E389FA
:1078C0009A4207D2D4F824C01CF802C080F800C045
:1078D000501C20812089984204BF0120087001209B
:1078E00010BD10B4DFF88CC313F0070F04D003F001
:1078F0000702022A2ED02AE0012A01D09AB126E0FE
:10790000DCF800004069DCF8001040F0010048613C
:10791000DCF80000006BD84920F440500843DCF844
:107920000010086313E0DCF80000006BDCF80010C6
:1079300020F4405040F4BE0040F020400863DCF8E2
:1079400000004069DCF8001020F00100486110BC24
:1079500000207047DCF80020526902F0010202703A
:107960000120087010BC704770B50D46044613F036
:10797000070F04D003F00700022808D005E0002A12
:1079800014BF0120002001F03FFE002070BD01F077
:1079900042FE002814BF012200222270012028701C
:1079A00070BD70B503F00700B14D1446012808BF43
:1079B000002017D013F0070F15D12889002808BF21
:1079C000EA700DD001280BD1E878FBF703F8AB493A
:1079D000E8780B6800EA04021A630968A043486368
:1079E0002889401C2881002070BD70B50E4603F028
:1079F000070C9F4D04990446BCF1010F04BF002001
:107A0000288118D013F0070F03D0BCF1020F14D057
:107A100011E028899A4B02283CBFD3F800C00CF82B
:107A20000020401C80B22881884204D102220F200D
:107A3000196800F0C3FF002070BD0AF0D3F92A894D
:107A4000002A04BF000A207004D0012A02D120704D
:107A500001203070501C2881012070BD70B50E4689
:107A600003F0070C824D04990446BCF1010F04BFDA
:107A70000020288118D013F0070F03D0BCF1020FAB
:107A800014D011E028897E4B02283CBFD3F800C0F7
:107A90000CF80020401C80B22881884204D10222C8
:107AA0001020196800F08AFF002070BD0AF0AFF9BD
:107AB0002A89002A04BF000A207004D0012A02D1BA
:107AC000207001203070501C2881012070BD2DE9EC
:107AD000F04103F0070C664E069D0F460446BCF1CC
:107AE000010F04BF0020308117D0614913F0070F48
:107AF0000B8903D0BCF1020F12D00EE06049022BBB
:107B00003CBF0868C254581C80B23081A84204D1DE
:107B100002220968112000F051FF0020BDE8F08129
:107B200013B1012B05D009E00AF09AF9000A207080
:107B300004E00AF095F92070012038703089401C6B
:107B400030810120BDE8F0812DE9F04103F0070C00
:107B5000474E069D0F460446BCF1010F04BF0020AE
:107B6000308117D0424913F0070F0B8903D0BCF1C5
:107B7000020F12D00EE04249022B3CBF0868C254EB
:107B8000581C80B23081A84204D102220968122018
:107B900000F014FF0020BDE8F08113B1012B05D0E7
:107BA00009E00AF051F9000A207004E00AF04CF9EB
:107BB0002070012038703089401C30810120BDE8E0
:107BC000F08110B503F00702294C012A02D0022AE5
:107BD00027D024E003F005F90023002804BF6362E6
:107BE000E3811BD000F1500161624168B1F5887FEB
:107BF00090F820100CD390F8212001EB020C01FB2F
:107C000002C190F8222090F823001044084404E0B8
:107C100090F822000A1801FB0020E0812381002057
:107C200010BD2289E3899A4207D2D4F824C01CF8F7
:107C300002C080F800C0501C20812089984204BFF7
:107C400001200870012010BD10B513F0070F04D0FB
:107C500003F00702022A05D002E0104601F02AF9DB
:107C6000002010BD074A127802700120087010BD74
:107C7000D840002034E3010000205FA02CE3010085
:107C800054E301000D41002010B513F0070F04D09C
:107C900003F00702022A05D002E0104601F0B0FA14
:107CA000002010BDF74A127802700120087010BD44
:107CB0001FB513F0070F07D102F0A6FE20B1012275
:107CC00002A90A2000F07AFE04B0002010BD70B5B1
:107CD00003F00700EC4C1646012804BF0020208169
:107CE00028D013F0070F25D102F08EFE10B32089A3
:107CF000E64D03283CBF29680E54401C80B2208109
:107D0000032817D1F9F724FD2868B0F8010046BA16
:107D1000F9F744FC040018BFF9F749FE2868007819
:107D2000002818BF01203146F9F715F9002C18BFBB
:107D3000F9F740FE002070BD70B503F00700D24C8B
:107D40001646012804BF002020812DD013F0070F14
:107D50002AD102F059FE002826D02089CB4D0228D6
:107D60003CBF29680E54401C80B2208102281BD1E0
:107D7000F9F7EEFCF9F712FC040018BFF9F717FE4B
:107D80002868007800282868417808BF002005D0BE
:107D90000120F9F72EF9286841781120F9F729F91F
:107DA000002C18BFF9F706FE002070BD7FB51C46F9
:107DB0000E46054613F0070F08D102F025FE28B144
:107DC000012202A9132000F0F9FD03E004F00700EE
:107DD000022802D004B0002070BD04F08DFC002801
:107DE00014BF012200222A700120307004B070BD3F
:107DF0007FB51C460E46054613F0070F08D102F06A
:107E000003FE28B1012202A9142000F0D7FD03E0EF
:107E100004F00700022802D004B0002070BD04F076
:107E20005CFC28700120307004B070BD70B503F0A8
:107E30000700954D049C1646012804BF00202881A8
:107E40001AD013F0070F17D102F0DEFDA0B1288978
:107E50008E4903283CBF0A681654401C80B2288112
:107E6000A04209D108680968B0F80100097840BA51
:107E700000B219B1FEF7B4FC002070BDFEF7ADFCF6
:107E8000FAE770B503F007007F4D049C1646012801
:107E900004BF0020288118D013F0070F15D102F07D
:107EA000B3FD90B12889794B03283CBF19680E5463
:107EB000401C80B22881A04207D11868B0F80100A8
:107EC00041BA18680078FAF707F9002070BD70B55C
:107ED00003F007026C4CDDF810C0012A02D0022A20
:107EE00007D004E000202081FBF764F92062002025
:107EF00070BD2289624506D2C2F10303256ADB0008
:107F000025FA03F30370501C80B22081604504BF42
:107F100001200870012070BD7FB51C460E46054645
:107F200013F0070F0DD102F06FFD50B19DF808005E
:107F300010F0010F09D0012202A9152000F03EFD2A
:107F400003E004F00700022802D004B0002070BD56
:107F500004F070FC28700120307004B070BD2DE971
:107F6000F0411C4617460E46054613F0070F06D192
:107F700002F04AFD18B138460BF06CFA03E004F049
:107F80000700022802D00020BDE8F0810BF01FFAA4
:107F9000287001203070BDE8F081002070477FB567
:107FA0001C460D46064613F0070F08D102F02CFDC3
:107FB00028B1012202A9072000F000FD03E004F02F
:107FC0000700022802D004B0002070BDFDF76AFA55
:107FD000022808BF00200BD0032808BF022007D0CA
:107FE000042808BF032003D0052814BFFF20012068
:107FF00030700120287004B070BD2DE9F0411C469E
:1080000017460E46054613F0070F0BD102F0FCFC95
:1080100040B1384604F038FB00221146012000F040
:10802000CDFC03E004F00700022802D00020BDE8E8
:10803000F08104F02CFB287001203070BDE8F08145
:1080400010B5104613F0070F08BF04F074FB0020B2
:1080500010BD10B5104613F0070F08BF04F077FBF2
:10806000002010BD70B5044603F007000D4602283D
:108070001CBF002070BD04F077FB20700120287029
:1080800070BD000012410020D840002054E30100E0
:1080900070B403F007020024FE4BDDF80CC0012A87
:1080A00005D0022A04BF9A78022A0AD01BE00220D7
:1080B0009870F9481C816FF07F410068081A1862B7
:1080C00011E01A89624506D21E6AD50026FA05F526
:1080D0000570501C18811889604504D11C8101204D
:1080E00008700320987070BC0120704713F0070FD0
:1080F00004BFEA4802700020704710B5944603F0B0
:108100000700E449029A012804BF0020088112D028
:1081100013F0070F0FD10889E14B90423CBF1C6858
:1081200004F800C0401C80B20881904203D10E20A8
:10813000196800F043FC002010BD2DE9F0471746F8
:1081400003F00702DFF84C834FF0000C012A04BF54
:10815000A8F808C0A8F80AC041D013F0070FCD4B0B
:10816000DFF840939D895E6A02D0022A3AD036E059
:10817000B8F80800002808BFC8F824702AD00128E1
:1081800004D0841EAC4216D28CB909E0781CA8F841
:108190000C003044B0F5807F88BFA8F80CC019E00F
:1081A0004FF480724FF42A31BF4812F09DFABC4957
:1081B000301909680F54601CA8420BD1BA48C0F8A6
:1081C000FC904FF42A30FAF7C5FAB7494FF42A3039
:1081D000FAF729FBB8F80800401CA8F808000020AE
:1081E000BDE8F087FF220270C5B1B8F80A20B318C5
:1081F000521CB3F5807F0FD2AC4C24684C4518BF9D
:1082000080F800C004D103F5283393F800380370D8
:10821000AA4204BF01200870A8F80A200120BDE886
:10822000F08770B503F007009A4D049C16460128AC
:1082300004BF0020288115D013F0070F12D102F0DF
:10824000E3FB78B128899649A0423CBF0A681654DE
:10825000401C80B22881A04204D122460968042033
:1082600000F0ACFB002070BD70B50D46044613F065
:10827000070F04D003F00700022805D002E01046E3
:1082800004F0F6F9002070BD04F0F5F9207001202B
:10829000287070BD1FB513F0070F04D1012202A989
:1082A000162000F08BFB04B0002010BD03F0070186
:1082B000DFF8E0C10098012907D013F0070F04BFD1
:1082C0009CF80210012909D01FE001208CF802005F
:1082D0000020ACF80800CCF81C0014E0BCF8081032
:1082E000814208D2DCF81C30491C42EA0322CCF857
:1082F0001C20ACF8081089B2814206D103208CF80A
:108300000200DCF81C00CCF824000020704703F0C9
:108310000701DFF880C10098012907D013F0070F8B
:1083200004BF9CF80210022909D01FE002208CF83B
:1083300002000020ACF80800CCF8200016E0BCF8E1
:108340000810814208D2DCF82030491C42EA03229E
:10835000CCF82020ACF8081089B2814206D1BCF8D4
:108360002000ACF80E0003208CF8020000207047BB
:1083700070B403F007020025464C012A02D0022AFD
:1083800006D002E00220A070258170BC002070475A
:10839000A278022A1CD12289B4F80EC062450FD2FD
:1083A00012F0030F04D1636A53F8046BC4E9086345
:1083B00094F820300370206A000A2062501C20814B
:1083C0002089604504D12581012008700320A07018
:1083D00070BC0120704770B503F0070000252D4CDC
:1083E0000E46012806D013F0070F04BFA07802281C
:1083F00005D02BE00220A0702581256226E020898F
:10840000E189884219D2216A090A41EA0262401CC4
:108410002262208110F0030F0FD1606AB0F5303F67
:1084200028BF026006D2B0F5005F03D304222049C2
:10843000FAF75EFA606A001D60622089E18988426D
:1084400004D12581012030700320A070002070BD70
:1084500030B403F007040025DFF838C0012C08BF52
:10846000ACF8085046D013F0070F02D0022C44D0CD
:1084700040E0042A08BF4FF42C3039D024DC002A15
:1084800008BF4FF4005033D0012A08BF4FF42F30FB
:108490002ED00FE0D8400020704000201540002072
:1084A00054E30100554E564D6C5A0020FCA80200C2
:1084B000F8400020022A08BF4FF4103018D0032AD9
:1084C00008BFFE4814D010E0052A08BF4FF42A3038
:1084D0000ED0FB48102A00680AD0112A08BFF948BC
:1084E00006D0202A08BFB43002D0CCF81C5001E0DE
:1084F000CCF81C0030BC00207047BCF80820042ACF
:1085000007D2C2F10303DCF81C40DB0024FA03F3BA
:108510000370501C80B2ACF80800042824BF01206E
:108520000870012030BC704710B503F00700012827
:1085300004D1002211460D2000F040FA002010BDA9
:108540002DE9F04703F00704DF4E089F9046894667
:108550000546012C04BF0020308119D013F0070F0D
:1085600014D102F051FA88B13089D84902283CBFB1
:108570000A6802F80080401C80B23081B84207D1FE
:1085800002220968062000F019FA01E0022C02D04C
:108590000020BDE8F087328912B1012A04D009E039
:1085A000FCF780FF287005E0FCF77FFF28700120B2
:1085B00089F800003089401C30810120BDE8F08737
:1085C00070B503F00700C04D012803D013F0070F6A
:1085D00005D024E00020E8612862E8701EE0BA4976
:1085E0002C8991F803C0C8690CEB0201CBB2022CB4
:1085F00003D242EA0020E86106E0B349042C096A8C
:1086000004D242EA01202862EB7005E0052C03D277
:10861000624508BF01F050F82889401C28810020DD
:1086200070BD10B503F007011046012905D013F005
:10863000070F08BF00F080F904E0A3490020C861DB
:10864000C8700881002010BD10B5104613F0070F48
:1086500008BF00F071F9002010BD70B50726002496
:108660004FF4103505EB0430FAF7A9F8022808BFDB
:1086700070BD601CC4B2B442F4D3012070BD30B4EC
:1086800003F007030024DFF840C2029A012B02D056
:10869000022B0CD008E005208CF80200ACF8084052
:1086A0009CF805008CF8030030BC002070479CF853
:1086B0000230052B14D1BCF80830934205D29CF847
:1086C00003500570581CACF80800BCF80800904234
:1086D00006D1ACF808400120087003208CF8020095
:1086E00030BC012070472DE9F04779A0DDF820C0AB
:1086F000006803F007050027734E744C012D03D06A
:1087000013F0070F06D034E0378120680770206827
:1087100047702EE03389634503D22568EA545A1C1A
:1087200032813289624524D137814FF0010881F8C6
:1087300000802168C2B2097891421AD12168C0F341
:1087400007204978814214D1072500244FF41039BD
:1087500009EB0430FAF733F8022804D0601CC4B2E5
:10876000AC42F5D34046012806BF86F80580377134
:1087700077710020BDE8F0872DE9F0414FF0000C43
:1087800003F00700534E504C6546012803D013F008
:10879000070F0CD068E02570E580A56165700020AA
:1087A00046F82050401CC0B24028F9D35CE0207845
:1087B00005283CBF401C2070C0B2012808BF100231
:1087C00022D0414902280B8A08BF98181CD024BF28
:1087D000E1888B4248D9404F01F0030001F10108C4
:1087E0003A54A7F128004FF410328069984502EB03
:1087F000002008BF002109D1491CC9B20429FBD3BC
:108800003449FAF710F826E020822DE0032232EAFC
:10881000010120D17A5CCB009A40491CC9B242EADE
:108820000C0C0429F6D3617801F03F02491CC9B24F
:1088300046F822C0617040290DD12649F9F7F3FFAF
:108840006570A069401CA061002046F82050401CC3
:10885000C0B24028F9D3E088401C80B2E080218A71
:10886000884204BF012020710020BDE8F08110B5CE
:108870000446002003F036FF002000F065FF21468B
:108880000222BDE81040062000F09AB82DE9F04120
:108890001E46174688460546F8F75AFFF8F77EFE4B
:1088A000040018BFF9F783F8012D414623D00120B9
:1088B000F8F767FD3146012010E0000000AF02002C
:1088C0009441002084830020D840002054E301001C
:1088D00055AC00006C5A002000410020F8F789FBDD
:1088E0003846F8F70CFB002C08BFBDE8F081BDE866
:1088F000F041F9F75FB80020F8F743FD314600205A
:10890000F8F777FB3846F8F7FAFAECE72DE9F0418B
:108910001F4616460D4601280CBF002401242046A0
:10892000F8F778FD28802046F8F754FB3880F8F7F0
:10893000FDFA3080BDE8F08110B5114C2146238945
:10894000CA78D1F81CC01118C9B2022B03D240EA70
:108950000C20E06107E0B3F5817F06D2094A126876
:108960001A4402F8020CE17006E008BF904203D1FD
:108970000549604600F0C2FE2089401C208110BDE0
:10898000D840002054E301006C5A0020FE48002229
:1089900002704270827002714271C270DFF8ECC3E3
:1089A000114601EB410300200CEB43031A54401C19
:1089B0000628FBD3491C0829F3D3704712F026B9C7
:1089C0002DE9F04115460E460746FAF708FB00F080
:1089D00008040820FAF7FEFA2A463146384612F013
:1089E00015F905462046FAF7F1FA2846BDE8F08168
:1089F000E54880787047E44840787047E2490020B5
:108A0000487070472DE9F84F0024FAF758FFDE4F01
:108A1000B878002800F0D381E9464FF0FF38FAF724
:108A2000DEFA00F0080A0820FAF7D4FAF8780025F0
:108A3000F0B17879D54900EB4002401CC0B201EB9F
:108A400042017871082828BF7D71F878401EF870BF
:108A500091F801800E780020B8F1000F06DD0A18A9
:108A6000927809F80020401C8045F8DC0D704D70AC
:108A70005046FAF7ABFAB8F1000FC0F29281F0B2AB
:108A80000024172880F05081DFE800F083230F19BD
:108A9000260C32FC3783696F74B4FBFAF9F8F78758
:108AA000969BA000FCF7A6FD13E09DF800100120A6
:108AB000FCF70AFD01207870044600F035B99DF8F6
:108AC000000002F08BF901210320FCF7FDFC0120DE
:108AD0007870012400F028B9BDF8000040BA03F016
:108AE000CDFD02210320FCF7EFFC01207870F0E7B8
:108AF0009DF801109DF800004CE04FF0010987F847
:108B00000190387848BBF8F70FFF30B39DF800802C
:108B100087F8009018F0040F18BFFDF7A9FE18F0B1
:108B2000020F05D0FF210F20FCF721FF48F00108BC
:108B300018F0010F10D0FCF7B5FC022802D103F0A9
:108B4000EBFD48B1FCF7AEFC052802D100F011FEA8
:108B500010B10020FBF77EFA3D707D70E4E09DF8D7
:108B60000000401E01F05AFDB3E79DF8000003F03D
:108B700005FEAEE79DF8000000287DD0FCF792FCD2
:108B8000022818BF012403F0D0FD01460220FCF7A3
:108B90009BFCC9E0FCF798FC9BE79DF800000028CF
:108BA00018BF012003F09EFD9DF80000002818BFAB
:108BB000012000F0C9FDB7E09DF8000003F083FD3F
:108BC00087E79DF8000003F0F2FD82E79DF80000C2
:108BD00020B1012872D0022805D0A5E04FF42F3033
:108BE000F9F7B8FDA0E001F052FF00210420FCF7E6
:108BF0006BFC6EE7FAF7F3F900F008080820FAF7C3
:108C0000E9F9F878002808BFBD704046FAF7DEF9A8
:108C10004FF00009C84672B6FAF7C5FC48B1FAF73A
:108C20009CFD8146FAF779FDFAF79DFD8046FAF73B
:108C300084FDF8F78DFDF8F7B1FC8346F8F720FEC8
:108C4000FAF771FA5FEA000A18BFFAF750FA4FF420
:108C50009350FAF7C8F962B64D4805604D4801686F
:108C6000D1F8CC10006841F4BE0141F02041C0F8B9
:108C7000C81011F0E2FE06E032E050E049E042E0C8
:108C80003BE030E01BE0BBF1000F72B603D0F8F719
:108C90005FFDF8F75AFEFAF786FC48B1B9F1000F0C
:108CA00018BFFAF786FCB8F1000F18BFFAF7CDFC31
:108CB000BAF1000F18BFFAF7DCF962B634E09DF89C
:108CC0000000012804BF042105203FF463AF0228FF
:108CD00006D0032807BF002104200221084659E7D7
:108CE0000021032056E79DF80300009A1E2160F33F
:108CF0001F62012003F0E3F916E0BDF8000040BA5E
:108D000009F076F810E0BDF8000040BA09F085F8E7
:108D10000AE0BDF8000040BA09F0A5F804E0BDF88B
:108D2000000040BA09F093F8B4BBE9464FF0FF38B1
:108D3000FAF755F900F0080A0820FAF74BF9F87825
:108D4000F0B17879114900EB4002401CC0B201EB50
:108D500042017871082828BF7D71F878401EF870AC
:108D600091F801800E780020B8F1000F06DD0A1896
:108D7000927809F80020401C8045F8DC0D704D7099
:108D80005046FAF723F908E0044100206C5B00200C
:108D9000444000203CE3010003E0B8F1000FBFF6BF
:108DA0006EAEFAF71CF900F008060820FAF712F97F
:108DB000F978002908BFBD703046FAF707F9FCF7CB
:108DC00071FB022802D101F0EAFD20B9002C04BF9A
:108DD0000020BDE8F88F0120BDE8F88F0246002092
:108DE000022928BF704752B1012A18BF704701EB12
:108DF000810000EBC100F84901EB00107047C1EBA6
:108E0000C100F64900EB800001EB4010704770B5DF
:108E1000FAF7E5F800F008060820FAF7DBF8F04C5E
:108E200000256078302806D24FF40C61EB4811F031
:108E300060FCA570E570A079302806D24FF4D0719F
:108E4000E54811F056FCE57125723046BDE87040EA
:108E5000FAF7BCB800FB01F2B2F50C7F9CBFE04A08
:108E6000C2E9030170470028DD4AD26818BF0260DA
:108E7000DB480029006918BF086050437047D84894
:108E8000012101710078D54980F00100C0EBC000DC
:108E900000EB800001EB40107047D1488278002140
:108EA00032B1C27822B9027882F001020270817078
:108EB00001717047CA491E284A78487008BF0020CF
:108EC00003D01F2808BF012000D10870104670474A
:108ED000C3480078C14980F00100C0EBC00000EB3E
:108EE000800001EB40107047F0B4BD4E96F800C012
:108EF000BA4CCCEBCC0CF5680CEB8C0C04EB4C1C9A
:108F000003FB05F40CEB440C8D4234BF2C460C469D
:108F10003669F31A934238BF1A460026002A9CBFCE
:108F2000F0BC70470023002C06D930F813702CF8E1
:108F300013705B1C9C42F8D8761C0CEB450C00EBC4
:108F400041009642EED3F0BC70472DE9F041A44FAA
:108F500014468C4601467A7806981D468A4218BF08
:108F6000BDE8F0810121F970012802D0022825D046
:108F70002AE038789949C0EBC000FE6800EB800019
:108F800001EB4011A64234BF324622463869A8425E
:108F900038BF05460023002D16D90020002A06D927
:108FA0001CF8007021F81070401C8242F8D85B1C3D
:108FB00001EB4601A444AB42EFD305E000232A466F
:108FC00021466046FFF790FFBDE8F04100F0A7BAE8
:108FD000002808BF70478249824B4A7882491B7833
:108FE000002A097818BF022A05D0042A18BF092AC6
:108FF00001D0012278E77D4A1278012A84BF7C4A99
:109000001378012200F0A5BA2DE9F04F744983B01E
:109010000122CA70774A49781778724A232992F850
:1090200000A024BF03B0BDE8F08FDFE801F01223F9
:10903000122312232323231223232323B6B6232B05
:109040002B2BB6B6B6B6B6B6B6B6B623B6B6B6AA75
:10905000AA0066490978012904D967490F7864494B
:1090600091F800A000287DD000235246394600F038
:1090700070FA8DE0002875D0002352463946FFF77C
:1090800033FF85E0F8F764FBF8F788FA00900028D2
:1090900018BFF8F78CFC55480078012884BF544865
:1090A00090F800A0F8F748FC10F0040F18BF0AF180
:1090B000010A52484A4C006800F5804001906078EF
:1090C000A0F1110920784549C0EBC00000EB8000F9
:1090D00001EB4015E068B84238BF074620695045AB
:1090E00038BF8246F8F7B9FC83460020F9F773F8D9
:1090F0000026BAF1000F37DD0024002F2BDD019987
:10910000C6EBC60001EBC0081BF904001C2824BFF5
:10911000002025F814001BD200EBD0714910C007C5
:1091200058F82110C00E21FA00F081B24FF0FF3044
:10913000B9F1000F1ED0B9F1010F08BFC8B205D0B8
:10914000B9F1020F04BF0846F9F74BF825F81400EF
:10915000641CBC42D8DB2248761C5645C06805EB2F
:10916000400500E014E0C7DB0098002818BFF8F7BE
:1091700021FC0DE011F4805FC1F3032018BF4042D1
:10918000E4E728B100230AF102023946FFF7ACFEFA
:1091900003B0BDE8F04F00F0C2B903B0BDE8F08FF6
:1091A0000F4801214172407980F0010000EB8001FD
:1091B00001EBC000084901EB001070470848C27974
:1091C000002132B1027A22B9427982F00102427161
:1091D000C1714172704700005C6400209C5B0020FC
:1091E0000C4100209F400020A5400020A04000200E
:1091F000A24000209E400020A140002050E301003A
:10920000F6491E288A79887108BF002003D01F28DC
:1092100008BF012000D1487110467047EF484079DF
:1092200080F0010000EB800101EBC000EC4901EB94
:10923000001070472DE9F04FEA4985B0012291F8FE
:109240000080E94991F80090E4490A728979E44C78
:1092500011291CBF1229132939D008B3DF494979D4
:1092600001EB810202EBC10104EB01120021B9F113
:10927000000F06D930F8113022F81130491C894509
:10928000F8D80021B8F1000F0AD909EB010302EB6D
:10929000410C30F81330491CACF868308845F4D8DC
:1092A000F9F79DFE00F008050820F9F793FECB4C76
:1092B000607A002818BF012100F0B980E1712846CA
:1092C000F9F784FE0020207205B0BDE8F08FF8F7B2
:1092D0003FFAF8F763F90190002818BFF8F767FB29
:1092E000BE488179A1F11106817A0091407900EBA5
:1092F000800101EBC00004EB0015F7F752FCBB49FD
:109300004FF0110B0028096801F5804101F5F56760
:1093100001F5E76104BF8A46012004D0BA465846E9
:109320000F464FF0010BF8F756FFF8F794FB0024B7
:109330000390B9F1000F2FD90098C0EBC000C00016
:109340000290039800570828B4BF143008381C282E
:1093500024BF002025F814001BD200EBD072029924
:10936000521001EB8201C00751F80A10C00E21FA19
:1093700000F081B24FF0FF30002E4AD0012E08BF1E
:10938000C8B204D0022E04BF0846F8F72AFF25F819
:109390001400641C4C45D4D35846F8F71CFFF8F76A
:1093A0005CFB00248246B8F1000F2CD90098A3463C
:1093B000C0EBC0004FEAC0091AF904001C2824BF02
:1093C00005EB4400A0F868B01AD200EBD071491048
:1093D00009EB8101C007C959C00E21FA00F081B222
:1093E0004FF0FF30E6B1012E08BFC8B204D0022E04
:1093F00004BF0846F8F7F5FE05EB4401A1F8680044
:10940000641C4445D8D30198002818BFF8F7D2FA55
:1094100046E711F4805FC1F3032018BF4042B6E76E
:1094200011F4805FC1F3032018BF4042E4E7607984
:1094300080F001006071002140E770B50D4667497A
:109440000122CA706A4A497816786A4A2129147832
:109450001EBF2229232970BD002818BF002D11D05E
:10946000002322463146FFF73FFD631C01222146BF
:109470002846FFF739FD05EB4400A31C01223146C5
:10948000FFF732FDBDE8704000F049B870B5534DAC
:109490000446687890B9A06868B1574909780129ED
:1094A00094BF544955490B7855490122097800F079
:1094B00050F8687810B96068FFF7A6FD6878112841
:1094C00004BF0020FFF7A0FD6878122804BF002029
:1094D000FFF79AFD6878132804BF0020FFF794FD7A
:1094E000E06810B1A97921B105E0206918B1A97926
:1094F00009B9FFF79FFEA879112804BF0020FFF7E4
:1095000099FEA879122804BF0020FFF793FEA879DE
:10951000132818BF70BD0020BDE870408AE670B502
:10952000F9F75DFD00F008060820F9F753FD2B4C14
:1095300020790025002801BF207880F001002070EC
:10954000A5701CBF0120A0703046F9F73FFDE57003
:1095500070BD2DE9F047994616460D460446F8F7CA
:1095600081FA5FEA000C1DD01C490878254AC0EB3F
:10957000C000D1F80C8000EB800002EB401009FB2A
:1095800008F200EB4200454594BF2F464746096963
:10959000A1EB0901B14238BF0E460021002E08D8C8
:1095A000BDE8F0874B46324629462046BDE8F047E5
:1095B0009AE40023002F08D91CF9032034F8122064
:1095C00020F813205B1C9F42F6D8491C00EB480092
:1095D00004EB4504B142ECD3BDE8F0870C41002018
:1095E0005C640020A3400020A440002050E3010060
:1095F0009E4000209F400020A0400020A24000206C
:10960000A54000209C5B00202849002814BF0020B2
:109610000120087070472548007800280CBF012001
:10962000002070472148017871B121490A685269C8
:109630000B6842F001025A610A68126B1D4B0968FF
:1096400022F440521A430A63002141608160C160E4
:10965000016141617047E5E700B50178C27983B0E7
:10966000114341F040018DF8001041788DF8011050
:10967000418809098DF80210818809098DF80310C5
:10968000817801F00F02017962F31F118DF8041047
:1096900081798DF80510017A8DF80610407A8DF8E1
:1096A0000700684611F0D1FB03B000BD2041002047
:1096B00034E3010000205FA070B50E460446FBF7BE
:1096C000F1FE042811D1A4F5107080280DD2A01944
:1096D000A0F24120802808D225020024002E04D9BF
:1096E0002846F9F737F8012801D0002070BD641C26
:1096F00005F58075B442F3D3012070BD70B50D46F9
:109700000446FBF7CFFE04280AD1A4F51070802888
:1097100006D220022946F9F786F8012808BF70BD55
:10972000002070BD10B5074CFFF76CF9012808BF89
:1097300010BD206801F04DFA002818BFFBF7EBFEC2
:10974000F2E70000944100208E4A0028516814BFBF
:1097500041F0010021F0010050607047894B5968C9
:109760000A0E120721F07F4142EA00600843586068
:10977000704784484068C0F3036070478148406880
:10978000000F70477F48006970477E4901200861DB
:1097900070477C490020086170472DE9F04F7A4FEF
:1097A00087B03868B0F90E11B0F90C0100F0BCFCBC
:1097B0000EF018FA3868D0F8F800C0F30340FAF752
:1097C00084FBFBF76FFE052839D1DFF8C091DFF885
:1097D000C0B16C4D4FF000084FF47A7A6868C0F35E
:1097E00003643868A100D0F8F800C5F80880C840C4
:1097F00000F00F0621460520C5F80C8002F0E0FCC1
:1098000021460520F6F766FD002C7DD0022C1DD0E8
:10981000042C7AD068680A2C4FEA106120F07F404F
:109820004FEA017118BF41F0007108436860FFF70B
:10983000E9F8012803D0FBF735FE0528CED0FAF76A
:109840005DFB07B0BDE8F04F0EF0D1B90F213046F7
:10985000FBF7F8FE0028EAD000F005FE00F0F9FD65
:10986000FAF7F4FA06460020F7F749FB4948F7F7FC
:10987000DCFE0120F7F7CEFEF9F7D8FB4648F9F7F2
:1098800083FCF9F768FCF9F795FC3968B1F8062113
:10989000504300F5FA70B0FBFAF082B26A8091F89A
:1098A0000801287050B1F9F785FC3968B1F8041146
:1098B000484300F5FA70B0FBFAF082B21046F9F7AF
:1098C000FDFBD9F8001035488861F7F741FFF8F73C
:1098D00054F8287838B1401E10F0FF00287004BFFB
:1098E0006888F9F7EBFB6868C0F30364FFF78AF850
:1098F000012806D06868C0F30360A04208BF002EAC
:109900001DD0D9F8000001E034E037E0C0F818B00D
:10991000F9F7EDFBF9F72BFC0020F9F735FCF9F727
:1099200092FBF7F715FFF7F73BFE0020F7F77DFEF8
:1099300000F08FFD00F0B8FDFBF7DAFF77E768462F
:10994000F8F7D4F958B16846FFF7A0FD684611F062
:10995000A2FB0646F8F700FAFBF7FEFDC6E73868FB
:10996000406E10F0704F02D0FBF7D5FDBEE7FBF75D
:10997000FAFDBBE7304612F049FA58E7304602F0EC
:10998000BEFF54E7384100209441002034E3010039
:1099900000005FA07BDD01003FD1010007005FA058
:1099A0007047002808BF704780220146014810F028
:1099B0009BBE70479C660020F0B4F84EDDE905C4FC
:1099C0003668049DB66916F0010F04D01F464B1B84
:1099D000CD1BDBB2EDB216F0020F06D06746A2EB4C
:1099E000040CD21B0CF0FF0CD4B216F0040F08D0FC
:1099F00080F800C04A1B84704270C91AC170F0BC64
:109A000070470370857080F801C0C470F0BC704767
:109A10002DE9F043164601FB06F90D46014685B0D7
:109A20001F464A46DE4810F069FEDD4C02F02DFF6D
:109A30004FF0000818B109F0CAFC01281AD002F052
:109A400024FF18B109F0C3FC082842D0B7F5805FA5
:109A50001CBF0020B9F1000FDCBF05B0BDE8F083EA
:109A60002156794309132154401C8145F8DC05B087
:109A7000BDE8F08300210B46002ECEBFDFF81CC3EB
:109A800005B0BDE8F0830020002D1CDDDCF80020CF
:109A900092F83E919945DCBF92F83F914B450CDC22
:109AA00092F83C918145DCBF92F83D21904204DC64
:109AB00062567A431213625401E004F80180401C9C
:109AC000491CA842E2DB5B1CB342DCDB05B0BDE80D
:109AD000F083AE428CBF701E681EC2B2B54234BF66
:109AE000681E701EC1B2501EC0B20423CDE9003002
:109AF0000292002303A8FFF75FFF00210A46002E11
:109B0000DCBF05B0BDE8F0830020002D19DD9DF815
:109B10000D309342DCBF9DF80F309A4209DC9DF86E
:109B20000C308342DEBF9DF80E30984204F801806D
:109B300003DD63567B431B136354401C491CA8423E
:109B4000E5DB521CB242DFDB05B0BDE8F0832DE956
:109B5000F0411C4615460E460746F8F791FF214690
:109B60002846F9F70EF806238D4A31463846F9F7AC
:109B70005AF9BDE8F041F8F796BF8A4AC2E90301F5
:109B800070472DE9FF4F884891B04FF000090678E3
:109B9000864890F800A08148006890F8ABE0B0F9E2
:109BA000A810109190F8AA00CDF80090CDF814906C
:109BB000CDF828900F900020CDF80490CDF80890B3
:109BC000CDF80C90CDF81090CDF81890CDF81C90F1
:109BD000CDF82090CDF82490CDF82C90CDF8309091
:109BE000CDF8349001460746844602460E90BAF1FD
:109BF000000F54D94FF0000845464446002E34D992
:109C000002FB064B129830F91B000028B4BFC0F1CC
:109C1000000B8346DE4524DAA8EB00080FFA88F82B
:109C20000028ACBF8346C0F1000B5944A8BF844450
:109C300005DA05F10105C0F1000BEDB25F44DDF876
:109C40004CB0BBF1010F0CD10028B8BF4042DDF889
:109C500040B0584505DA3DF812B00BF1010B2DF874
:109C600012B0601CC4B2B442CAD3B9F1000F07D11C
:109C7000B8F1000F04DD0F98A842D8BF4FF00109DA
:109C8000B54208BF4FF002093DF91200B0EB5A0F80
:109C9000C4BF01200E90501CC2B25245AAD3414C01
:109CA000E06A421A48BF0A1A414DA5FB0165EE0859
:109CB0000125964287BF1F9A157000221F9E98BFEC
:109CC0003270B9F1010F2CD0B9F1020F08D21A7815
:109CD000032A01BFC4E90B1C022015B0BDE8F08FB8
:109CE000B9F1020F25D0B9F1010F2AD0002808BF21
:109CF000C4E90B1C0FD01A78002A1CBF1E9A002A38
:109D000009D000EB400088423FBFC4E90B1C032090
:109D100015B0BDE8F08F139878B30E9801282DD0B8
:109D200035E0226B002A1CBFBCF1000FB2EB470FDD
:109D3000CDD202201870C4E90B1C15B00320BDE879
:109D4000F08F1878022838BF1D70C4E90B1C1878F2
:109D500002280ED01E9830B1BCF1000F18BFBCEB2A
:109D6000470F06D901E0674503D215B00220BDE8D0
:109D7000F08F15B00320BDE8F08F08E018780028B8
:109D80001FBFC4E90B1C052015B0BDE8F08FC4E966
:109D90000B1C15B00020BDE8F08F0000944100209E
:109DA000546700204C4100209E4000209F4000202E
:109DB000CDCCCCCCFE4900200A7A12F0060F18BF99
:109DC000486970470020FA49097A11F0060F18BF58
:109DD000F84870472DE9F00700248FB0002B9EBF94
:109DE0000FB0BDE8F0077047561E4FF000086F46F1
:109DF0004FF0000C002E16D904FB02C531F8159067
:109E000001EB45056D88A9EB05052DB227F81C501F
:109E10000E351C2D98BF27F81C800CF1010C1FFA81
:109E20008CFCB445E8D304FB02FC012A20F81C801A
:109E30004FF0010C13D904FB02C507EB4C0A00EBF1
:109E400045093AF802AC39F8029C0CF1010CA9EB77
:109E50000A091FFA8CFC20F815906245EBD804F132
:109E6000010C1FFA8CF49C42C2D30FB0BDE8F0077E
:109E700070472DE9F04FADF2246D03FB02FA4FF06D
:109E8000000CE946BAF1000F84BF0026CA4D13D971
:109E900031F91C4004F10F071E2F98BF29F81C60F0
:109EA00004D935F81C70E41B29F81C400CF1010C96
:109EB0000FFA8CFCE245EBD84FF0000C002B59D97F
:109EC0000CFB02F44FF0000B39F9148008F119046F
:109ED000322C3CD901252C46012A38D90CFB0246EC
:109EE00039F9167007F10A0EBEF1140F14D907FBE9
:109EF00008FEBEF1000F0FDD09EB460E3EF902EC45
:109F0000A7EB0E071837302F06D831F916600F3639
:109F10001E2E84BF6D1CEDB2641C24B2A242DDD89B
:109F2000142D11D900244FF0010B002A1CD90CFB71
:109F30000245641C31F8156039F8157024B2F61B1F
:109F400020F81560A242F2D8BBF1000F0CD100241A
:109F5000002A09D90CFB0245641C31F8156024B2B3
:109F600020F81560A242F5D80CF1010C0FFA8CFC18
:109F70006345A5D80021BAF1000F8EBF8E4A0DF2BD
:109F8000246DBDE8F08F30F8113022F81130491CF3
:109F900009B28A45F7D80DF2246DBDE8F08F2DE99E
:109FA000F04FDFF818C29DB00DF11008BCE8F000CA
:109FB0008DE8F000BCE8F00088E8F000BCE8F000B4
:109FC0000DF1200888E8F000DCE9004CCDE90C4CEC
:109FD0000026002B9CBF1DB0BDE8F08F0DF1380BA3
:109FE000A2F1010AEE464FF0000C65466746644652
:109FF000BAF1000F31D906FB024831F8189001EB95
:10A000004808B8F80280A9EB08080FFA88F82BF87E
:10A01000148008F10F08B8F11E0F9CBF0CF1010C61
:10A020001FFA8CFC0BD9AC4507D9BCF1000F04D04A
:10A030006546A4F1010C0CF0FF074FF0000C641C06
:10A04000A4B25445D7D3AC4507D9BCF1000F04D016
:10A050006546A4EB550C0CF0FF07052D23D906FB34
:10A06000027C31F91CC00CF10F041E2C1BD93EF8E8
:10A070001740002AA4EB0C0C0FFA8CF54FF0000CE3
:10A0800011D906FB02C43EF81C8031F81470A8EB0D
:10A0900005080CF1010CA7EB08071FFA8CFC20F84F
:10A0A00014706245EDD806F1010C1FFA8CF69E4241
:10A0B00099D31DB0BDE8F08F2DE9F0410746404827
:10A0C0003B4EDFF8088105783E48B26904783E4887
:10A0D000A0FB02304308A3EB8300831805FB04F0C8
:10A0E0004200C3EBC30008EBC01010F007FBB069DF
:10A0F000421CB261002F08BFBDE8F081032A38BFBF
:10A10000BDE8F081F8F7BCFC21462846F8F730FDA1
:10A1100008F5E06308F560722C493846F8F757FDFA
:10A12000BDE8F041F8F7BFBC2149488070472DE9F0
:10A13000F041274E8AB005461D48CDE90056A6F1EC
:10A1400070080C46CDF80880B0F9021003913F2941
:10A15000C8BF3F2005DC11F1400FB8BF6FF03F00D2
:10A1600000DA039000200490F8F78AFC1548144F99
:10A1700001783878F8F7FCFC6846F8F792FD08900B
:10A18000F8F791FCC4E90068BDF814002081BDF81F
:10A1900016006081BDF81800A081BDF81A00E081AA
:10A1A000BDF81C002082BDF81E00608212E0000095
:10A1B0004C4100201C6700201469002058E3010076
:10A1C0009E4000209F400020ABAAAAAA346F002026
:10A1D000247A0020BDF81C00BDF81E103A7801FB5F
:10A1E000020035F910000AB0BDE8F0812DE9FF4FFB
:10A1F000AE4FAF4E83B005002FD0F9F7E5FBAD4A67
:10A2000097F800C03178126800240223B2F91A715D
:10A2100000EB8C02A1F1020826461846B8F1020FA5
:10A2200077DDACF10109C7F10008A1EB030A0021B9
:10A23000BCF1000F7DD9494577D002EB410B32F8D4
:10A240001130BBF802B0A3EB0B031BB24345B4BF04
:10A25000A7421C4669DA012673E002924FF000091A
:10A26000307897F800C04FF0FF364A4640F2E738A2
:10A270004FF00A0E4C4635464F46002837DDACF10C
:10A280000103801ACDE90003CEF1000A0020BCF1E1
:10A29000000F88BF0FFA87FB1AD931F91020424509
:10A2A00002DA904606B25D46019B98420CD001EB63
:10A2B00040035B88D31A1BB25345B8BFCE4502DAC0
:10A2C0005245B8BF01249946401C80B26045E4D392
:10A2D000781C87B2009801EB4C01B842D6DC012C07
:10A2E00005D1029858B102F0FBFA012807D0724854
:10A2F000012C8680C58018BF00203CD10CE06E4840
:10A30000B0F904108E4206BFB0F906008542002461
:10A31000EDE716E00DE008E002F0E2FA012805BFE3
:10A32000069800280220012025E0491C89B26145D9
:10A3300081D336B9401C80B202EB4C0282453FF714
:10A3400076AF022D18BFB5F1FF3F07D136B1012519
:10A350002A460521032001F0B2FE0BE0012D14BFB7
:10A36000B5F1FF3F002E05D100252A460521032027
:10A3700001F0A5FE68B207B0C0B2BDE8F08F4E484C
:10A38000C06970474C48006A70474C4870474C4859
:10A390007047B0F900300122012908DD30F912C000
:10A3A0009C45B8BF6346521C12B28A42F6DB0022BB
:10A3B0000029D8BF704730F812C0ACEB030C20F86E
:10A3C00012C0521C12B29142F5DC704770B4D4B284
:10A3D000B0F900C001230646012C08DD30F9135006
:10A3E0006545B8BFAC465B1C1BB2A342F6DB00233D
:10A3F000002C09DD30F81350A5EB0C0520F81350A4
:10A400005B1C1BB29C42F5DC00EB4202CBB2B2F902
:10A4100000100120012B08DD32F910C08C45B8BFB7
:10A420006146401C00B29842F6DB0020002BDCBFE6
:10A4300070BC704732F810C0ACEB010C22F810C0B1
:10A44000401C00B28342F5DC70BC70471A48806A39
:10A450007047194800214162816170471648002108
:10A46000416281617047134810B50068124C008E3C
:10A47000A060FBF717F802280DD0052818BF10BD03
:10A48000A06810F0060F1ABF20F0060040F002008E
:10A4900010BDA06010BD02F03FF9002804BFA06805
:10A4A00020F00600F5D010BD704700009E4000204F
:10A4B0009F400020944100204C410020D482002085
:10A4C00094810020704708283CBFFE4908707047FF
:10A4D0000020FC4988604860FB48006890F88100D3
:10A4E000082838BF087070470020F6494860704758
:10A4F000F4480078704770B5F34D0024286890F850
:10A500006C0010F0020F0BD0FAF7CCFF022807D135
:10A51000EC482968007801EB8000B0F8840084B230
:10A52000204670BD70B5E84D4FF48054286890F80F
:10A530006C0010F0020F0DD0FAF7B4FF022809D119
:10A54000E0482968007801EB8000D0F88400000C16
:10A55000C0F31304204670BDDA488078002818BF85
:10A56000012070472DE9F041FAF79CFF022803D142
:10A5700002F0D2F8022803D04FF48050BDE8F081F9
:10A580004FF480552E4602F0F4F8DFF83C83044681
:10A59000CC4FD8F8000090F86C1011F0010F0CD0DF
:10A5A000B0F87600B9684042814206DC2CB1002048
:10A5B000641EB860204602F0E1F8D8F8001091F867
:10A5C0006C0010F0040F18BF002C0AD0B1F87C000A
:10A5D000621E9040B1F87E20824238BF1046C0F320
:10A5E0001306D1F8A40010F0020F1CBFB97800299F
:10A5F00002D0000CC0F31305B54298BF354602F0F7
:10A6000044F940B108F0E3FE012804D14003B5F558
:10A61000005F38BF05462846BDE8F0812DE9F04FC0
:10A62000DFF8A4A287B0DAF8001091F86C2012F0DD
:10A63000020F0DD0A34A91F88090DFF890B21778FE
:10A64000002809DB484503D2B84218BF06463DD171
:10A6500007B00020BDE8F08F3E464FF0FF38F6F718
:10A660009FFFF7F745FE0025B9F1000F2ED9DAF864
:10A670000000002400EB8500B0F8840081B2204681
:10A68000F6F769FCF7F779F96846F7F72FFB00282A
:10A690005FD0019878B101468D489BF80020007882
:10A6A0005043421E07D331F9020B0028B8BF404285
:10A6B0000444521EF7D2F7F74FFBF6F771FFA0459F
:10A6C00084BF2E46A0466D1C4D45D0D3B74243D023
:10A6D000082E3CBF7B490E70DAF80000B0F88210FB
:10A6E00039B300EB870200EB8600B2F88420B0F8A3
:10A6F000840092B280B2801A484340F30F34F9F7D5
:10A7000063F9744B9BF80020002193F800C002FB12
:10A710000CF2002A0DD930F81120224420F8112023
:10A720009BF8002093F800C0491C02FB0CF28A42FF
:10A73000F1D84FF0806002F0CBF8DAF80000022187
:10A7400000EB8600B0F8840082B2032001F0B7FC71
:10A7500009E0FAF7E0FE97E702F00BF803283CBFA8
:10A76000401C02F00BF8012007B0BDE8F08F5648FE
:10A7700054490068B0F87600424288688242BCBF03
:10A78000401E886070472DE9F04F8FB093460E460B
:10A7900004464FF0000A01F0ECFFDFF82C81494F2E
:10A7A0000500D14610D1FFF705FBD8F80010B1F82D
:10A7B0007810884208D30120C7F8089001F0DEFF26
:10A7C0000FB00120BDE8F08F002E1FDDB868002813
:10A7D000B8BFC7F8089007DBD8F80010B1F87410BC
:10A7E0008842BCBF401CB860D8F80000B968B0F817
:10A7F0007400884215DC032D13D2681CC7F808903A
:10A8000001F0BCFF0FB00120BDE8F08F09D1D8F8EE
:10A810000000B0F876004142B8688842C4BF401ECC
:10A82000B860B87850B1D8F8000090F8A40010F0E3
:10A83000040F1EBF00200FB0BDE8F08FD8F8000055
:10A84000B0F972108C420EDD796821447960B0F85D
:10A850006E00884210DC4FF0FF30C7F80490FFF71D
:10A86000DDFE824608E07868002805DD002CD4BFB4
:10A8700001212146401A7860DFF85C9099F80000C9
:10A8800007283AD1154859460078420068460FF02B
:10A8900035FFADF80040ADF80260ADF804503889DE
:10A8A000ADF80600B888ADF80800D8F80000B0F898
:10A8B0007210ADF80A10B0F87410ADF80C10B0F8C2
:10A8C0006E100DE080410020944100209E40002049
:10A8D000A24000209F4000200D410020A540002004
:10A8E000ADF80E10B0F87600ADF8100099F8000041
:10A8F000072804BF6846FEF76BFB50460FB0BDE863
:10A90000F08F3E4810B50068D0F8A40010F4807FA6
:10A9100006D0C0F30330012101FA00F0F8F761F826
:10A92000374900204870887010BD70B5344D002440
:10A93000A878002814BF01260026687828B901F0FD
:10A9400031FF002808BF002100D001218E4224D011
:10A950000A1C18BF0122AA7028480068D0F8A43049
:10A9600013F0040F0ED021B1C3F30310082808D24E
:10A9700006E00021A960696090F88100082800D2F3
:10A980002870012413F0020F18BF0124002A18BFF9
:10A9900001220421032001F092FB204670BD1749DB
:10A9A00000200968D1F8A41011F4807F08BF704717
:10A9B000DFF84CC09CF80120131C18BF012330B4F1
:10A9C000104CC1F303322468E46B012505FA02F24E
:10A9D000224011F4007F01D00AB102E00AB1002147
:10A9E00000E001218B4204BF30BC7047081C18BF37
:10A9F00001208CF8010030BC97E700009441002052
:10AA0000804100202CE301005F48007870475E48D9
:10AA1000406800F5407070475B48406800F5807002
:10AA2000704770B5584C4FF4103258496260106846
:10AA3000884204BF5068B0F5087F26D1D2F808C01C
:10AA4000BCF5D04F21D85249D06888420DD00023A0
:10AA500011461846B3EB9C0F07D251F8045B401C1B
:10AA60006B40B0EB9C0FF8D37BB9012502F58070E9
:10AA700000F0AFF848B1606800F5407000F0B8F839
:10AA800000281EBF2570012070BD002070BD3E490A
:10AA9000002008704FF41030F7F75CBE3A48017898
:10AAA00041B14068394A0168914202BF4168B1F53D
:10AAB000087F704700207047334B5B6803F5807355
:10AAC0001844F7F715BF304B5B6803F54073184423
:10AAD000F7F70EBF2C484068006970472A4949685B
:10AAE0000A6982429CBF00207047C0EBC00001EBA6
:10AAF000C00000F580607047234A526802EB800373
:10AB00005B6A1A44234B53F82000FF3020F0FF000B
:10AB100000FB01207047F0B41B4B00221D4E5C6807
:10AB20001746831893F928C0BCF1000FB8BF41F84D
:10AB300022700DDBD3B204EB830556F823306D6A27
:10AB4000FF33254423F0FF0303FB0C5341F822306D
:10AB5000521C102AE5D3F0BC704794460029B8BFB8
:10AB60007047094A526802EB80035B6A1344094A42
:10AB700052F8202002F1FF0020F0FF0001FB00301E
:10AB80006146F7F7B5BE00008C4100205446505393
:10AB9000EFBEADDE90E3010010B5FFF742FFA8B1B4
:10ABA000FFF735FF0146D02216480FF09DFDFFF755
:10ABB00033FF154C01464FF4C27220680FF094FD2C
:10ABC0002068406DBDE8104001F064BDFAF712FD49
:10ABD000E3E758B10D4A0168914207D1406820F07F
:10ABE0000F00B0F5087F04BF0120704700207047B8
:10ABF00030B1006820F00F00602804BF01207047CA
:10AC0000002070478483002094410020415053521B
:10AC100010B572B60120F7F7A7FCF8F7A9FBF8F713
:10AC2000D7FB4FF0FF30F8F7D5F9664880234FF493
:10AC30000052002152F821C040F821C0491CB1EB5C
:10AC4000930FF7D3F8F7D8F9F8F7F2FDF8F71CFEF1
:10AC50000120F8F7EEFDF7F749FD1E20F8F7DCFDBF
:10AC6000F8F7E2FBF7F7CCFEF8F792FDF8F736FCC1
:10AC7000F8F7D8F9F7F737FFF6F7A5FCFFF78CFFE1
:10AC8000F8F752F9F8F70CF9FDF780FEFBF72AFF09
:10AC9000FEF7E1FC62B64C480CF058FE4B4C2068C5
:10ACA000B0F90C010CF09CFFF5F7FBFAFFF70AFC7A
:10ACB000F8F720FEFAF753FE2068418A008AFEF773
:10ACC000C9F82068806EC0F34E0161F35F0001F0A7
:10ACD000E9F9FEF765FEFFF7C1FBFAF7A9FC20686A
:10ACE00090F8640000F00F00F7F750FB206890F830
:10ACF000200010F0010F04BF0021032003D001F059
:10AD000014FD01460220FAF7DFFB314800680069B4
:10AD10000C2100F07002012001F0D1F9F5F7B8FA2A
:10AD2000FFF7EFFD002010BD2A4CFDF76BFE012858
:10AD300006D0FAF7B7FB032802D101F084FAC8B1B4
:10AD4000002C05DC01F0F1FC01460220FAF7BCFB07
:10AD50000126214DFAF7A6FB0446FAF7A6FB0146A9
:10AD60002046F5F7B7FA062C29D2DFE804F02818B8
:10AD700007222515641E002CD7DCE3E7287840B9AC
:10AD8000FBF731FD28B900221E21022001F097F9BE
:10AD90002E7001F052FFDDE7FEF7FFFCDAE7FBF76C
:10ADA0004DFCFAF77FFB012804BF0220FAF789FB6C
:10ADB000D0E701F051FACDE7FEF7B4FCCAE7FAF7A5
:10ADC00011FCC7E700860020848300209441002006
:10ADD00034E30100FF70020098410020FE49087032
:10ADE000704710B44FF42C30FC4A016891421CD1DA
:10ADF0004168B1F5007F18D3836800228446B3F51B
:10AE0000056F88BF4FF405630021B1EB930F24BF9A
:10AE100010BC70475CF82140491C2244B1EB930FF1
:10AE2000F8D3002A04BF10BC7047002010BC704744
:10AE300070B54FF42C310446E84D0868A84217D18C
:10AE40004868B0F5007F13D38B6800228C46B3F5B9
:10AE5000056F88BF4FF405630020B0EB930F08D255
:10AE60005CF82060401C3244B0EB930FF8D302B181
:10AE7000002149B18A68B2F5056F88BF4FF40562B9
:10AE800020460FF031FC1CE0FF224FF40561204604
:10AE90000FF039FC4FF40070C4E900504FF4056026
:10AEA000A0600020E06084F8200084F8210084F88D
:10AEB000220084F8230040F2FF71C4E90410A0616D
:10AEC000E061012070BD70B50021C160D0F808C0FC
:10AED0000B460446BCF5056F88BF4FF4056C002295
:10AEE000B2EB9C0F06D254F82250521C2B44B2EB0A
:10AEF0009C0FF8D35942C1604FF42C304FF40562D7
:10AF00002146F7F7F5FC012818BF002070BD4FF46B
:10AF1000007170B402685160016801F1500291F84B
:10AF200021C091F820300CFB03F102EB410100221B
:10AF3000BCF1000F08D900EB4204521CB4F88A405F
:10AF400021F8024B9445F6D80022002B08D900EBDB
:10AF50004204521CB4F8CA4021F8024B9342F6D87E
:10AF60000022BCF1000F07D900EB4204521CA48858
:10AF700021F8024B9445F7D80022002B08D900EBAA
:10AF80004204521CB4F8444021F8024B9342F6D8D4
:10AF9000B0F8862021F8022BB0F8882021F8022B87
:10AFA000B0F8842021F8022B00240022BCF1000F0D
:10AFB00088BF00EB841508D905EB4206521CB6F891
:10AFC0000A6121F8026B9445F6D80022002B88BF55
:10AFD00000EB841508D905EB4206521CB6F8CA618D
:10AFE00021F8026B9342F6D8641C032CDDD370BCAD
:10AFF00070472DE9F74F88B000250A992C462E4658
:10B000000968049101F150030999002984BF74492A
:10B01000D1F800801CD90022002888BFB8F9CE7072
:10B020000DD933F9021B0029B4BFC1F1000C8C46C5
:10B03000BC45BCBF0D44641C521C8242F1D309992B
:10B04000761C8E42E7D3002CC8BF95FBF4FA08DCCF
:10B050004908414301EB5002049901EB4201B1F967
:10B0600050A00021029101910499503100910021DA
:10B070000391099900296CD95949009E06960968DF
:10B080004FF0000B4FF00109B1F9C0E0D1F8B41056
:10B090005F46C1F30741D846CDF814B007910028A8
:10B0A00029D9B6F900204FF0000C06999344634665
:10B0B00000280DD9B1F90040A51A48BF151B7545E8
:10B0C000B8BF0CF1010C01EB49015B1C8342F1D3C9
:10B0D00007998C4503D305997F1C1144059108F10C
:10B0E000010806EB49068045DBD3002FC4BF059954
:10B0F00091FBF7F101DC9BFBF0F1039B0A9A09B28B
:10B1000002EB43029180364A1268B2F9BA30AAEBD8
:10B11000030399420ADDB2F9B82052448A4205DDA0
:10B12000019A114401910299491C02910099099ACE
:10B1300001EB400100910399491C039191429BD37B
:10B140000299002905DDDDE9011291FBF2F101917F
:10B1500002E05146CDF804A00A9AA2F88610002118
:10B16000029103910499503100910021049100282B
:10B170006FD91B49009F069709684FF0000B099E85
:10B18000B1F9BCE0D1F8B410D846090ED946CDF8D3
:10B1900014B00791002E32D9B7F900204FF0000CFF
:10B1A000069993446346002E0DD9B1F90040A51AC3
:10B1B00048BF151B7545B8BF0CF1010C01EB4001F0
:10B1C0005B1CB342F1D307998C4504D3059908F170
:10B1D00001081144059105E09941002053454C4672
:10B1E0009441002009F1010907EB4007B145D3D391
:10B1F000B8F1000FC4BF059991FBF8F101DC9BFB8E
:10B20000F6F1049B0A9A09B202EB4302A2F8441039
:10B21000FE4A1268B2F9BA30AAEB030399420ADD7A
:10B22000B2F9B82052448A4205DD039A11440391D1
:10B230000299491C02910099891C00910499491CAA
:10B240000491814295D302980028C4BF039991FBD1
:10B25000F0FA0A98A0F888A001980A99504400B220
:10B2600000EBD0704010A1F884000BB0BDE8F08F67
:10B270002DE9F74F84B0E5490698DDE904430268FB
:10B280000546002000935063009B0968002B88BF8F
:10B2900001262AD905EB4003B3F90430002BB4BFD3
:10B2A000C3F1000C9C460FFA8CFCB1F9CC706745D9
:10B2B00010DCB5F986C0BCF1000FB8BFCCF1000CB2
:10B2C000002BB8BF5B42ACEB0303B1F9C6C01BB2A5
:10B2D0009C4506DA536B06FA00FC43EA0C0CC2F8F4
:10B2E00034C0009B401C9842D4D391F8CA30002B44
:10B2F0007BD091F8CB00834288BF18460023DDF84D
:10B3000000C0BCF1000F84BF401C019073D94FF006
:10B31000010EDDF804C04FF000090120CA46BCF15F
:10B32000010F4BD903FB0445B1F9CEC003950EFBC9
:10B330000445029503FB040602EB4605B5F950806F
:10B34000B8F1000FB4BFC8F100054546AC4535DB88
:10B350000EFB040602EB4605B5F95060002EB4BFA3
:10B3600075423546AC4529DB039D2F1A02EB470594
:10B37000B5F94E50002DB4BF6F422F46BC451DDBC2
:10B38000029F3F1A02EB4707B7F94E70002FB4BF78
:10B39000C7F1000BBB46E34510DCA6EB0808B1F98A
:10B3A000C8604645B8BF09F101097D1BB542C8BF59
:10B3B0000AF1010A401C019DA842BBD3BAEB090067
:10B3C00048BFA9EB0A0091F8CAC0604507DB01201D
:10B3D000D2F834C098404CEA000CC2F834C000984F
:10B3E0005B1C834207D2002B00E004E018BFA3F1EE
:10B3F000010E8ED18BE7069C049D4FF0000C206857
:10B400006346002DC0F830C088BF012714D904EB73
:10B410004306B6F94460002EB8BF764236B2B1F9A1
:10B42000CC80B04505DD066B07FA03F846EA08064E
:10B4300006635B1CAB42EAD300236E1E1CBFB14601
:10B440004FF0010A27D004EB4305B5F94670B5F972
:10B450004460BD1B48BFF51B2DB2B1F9C480A8459F
:10B4600016DAB4F98850B6EB050848BFA5EB060814
:10B470000FFA88F87E1B48BFEE1B35B2A845056B56
:10B48000AEBF0AFA03F65E1C0AFA06F635430563F8
:10B490005B1C4B45D7D3DDE9056500202B68002EEA
:10B4A000C3F83CC088BF012714D905EB4004B1F9AB
:10B4B000D880B4F90A41A04503DCB1F9DA80A0458F
:10B4C00005DADC6B07FA00F844EA0804DC63401C88
:10B4D000B042EAD3069D049E00202B68002EC3F8DC
:10B4E00038C088BF012714D905EB4004B1F9D880D2
:10B4F000B4F9CA41A04503DCB1F9DA80A04505DA08
:10B500009C6B07FA00F844EA08049C63401CB042B4
:10B51000EAD3DDE9056500202B68002EC3F844C09E
:10B5200088BF012714D905EB4004B1F9DC80B4F9D8
:10B530004A41A04503DCB1F9DE80A04505DA5C6C28
:10B5400007FA00F844EA08045C64401CB042EAD3FD
:10B55000069D049E00202B68002EC3F840C088BFC3
:10B56000012714D905EB4004B1F9DC80B4F90A4293
:10B57000A04503DCB1F9DE80A04505DA1C6C07FAB2
:10B5800000F844EA08041C64401CB042EAD3DDE938
:10B590000574049E20680023002FC0F84CC0C0F83A
:10B5A00048C088BF4FF0010814D904EB4305B1F936
:10B5B000E090B5F98A51A94503DCB1F9E290A945BB
:10B5C00005DAC56C08FA03F945EA0905C5645B1C90
:10B5D000BB42EAD30023002E88BF012714D904EB15
:10B5E0004305B1F9E080B5F94A52A84503DCB1F949
:10B5F000E280A84505DA856C07FA03F845EA0805F4
:10B6000085645B1CB342EAD302E000009441002051
:10B61000D2F83880106C30EA08031364916C43EA66
:10B62000080021EA00049464116B44EA000021EA56
:10B630000005156316D00021049E0846002E88BF21
:10B6400001260FD906FA00F73B4218BF491C401CDF
:10B65000049FB842F6D3012904D148EA0300C2F896
:10B6600040C0906324B1D06C002808BFC2F848C025
:10B67000D2F83C80506C30EA08035364D16C43EA42
:10B68000080021EA0004D464516B44EA000021EA76
:10B690000009C2F8349016D00021059E0846002EFD
:10B6A00088BF01260FD906FA00F73B4218BF491C94
:10B6B000401C059FB842F6D3012904D148EA030093
:10B6C000C2F844C0D06324B1906C002808BFC2F80F
:10B6D0004CC01DB1106940F010001061B9F1000FAD
:10B6E00003D0106940F020001061906B18B1106910
:10B6F00040F040001061D06B18B1106940F080003C
:10B700001061106C18B1106940F480701061506CB9
:10B7100018B1106940F400701061906C18B1106994
:10B7200040F480601061D06C18B1106940F4806002
:10B73000106107B00120BDE8F08F2DE9F04FB1B0E6
:10B7400016460D460446F5F72BFFF5F72AFA0100D9
:10B750004FF011001DBF029001200390012108BF8E
:10B76000CDE90210CDE91A54F6F775F900220DF172
:10B77000100B002D09D98356082BB4BF1433083B96
:10B780000BF80230521CAA42F5D3F6F766F90021F5
:10B79000002C07D9425C0BEB0103491C83F82020E5
:10B7A0008C42F7D8F6F7C8F82D900120F5F7CCFFBA
:10B7B000FE48007810F0200F4AD0F5F7F2F9FC4966
:10B7C00044F2A87244F23873096800280A44194404
:10B7D0000CBFCDE90012CDE9002106F18A001C90D2
:10B7E00040301D90FF210F20FAF7C1F8F5F7D8FE81
:10B7F0000025E9460DF1700A1AA850F8257002A834
:10B8000050F82500F6F7E7FC0024002F88BF0BEB6B
:10B8100045181AD918F904001C2828BF00200DD299
:10B8200059F8251000EBD072521051F82210C007C1
:10B83000C00E21FA00F080B2F6F7D3FC5AF82510BA
:10B8400021F81400641CBC42E4D36D1C022DD3D338
:10B85000D648007810F0010F00F0A181F5F7A1F9AA
:10B86000D3490028096801F5C46201F584610CBF61
:10B87000CDE91C12CDE91C210120F5F75DFB3090CC
:10B880000120F5F7F6FD2E900298F5F7A3FB28901E
:10B890000398F5F79FFB279024A8009022AB20AADD
:10B8A0001EA90298F5F740FD25A8009023AB21AA18
:10B8B0001FA90398F5F738FD0298F5F7ABFD269020
:10B8C0000298F5F7A7FDBB4D01902868B0F8E41089
:10B8D0000120F5F740FB00210120F5F7B5FD2868B0
:10B8E00090F8E6100298F5F784FB286890F8E610C7
:10B8F0000398F5F77EFB2868B0F8E8100298F5F792
:10B9000040FD2868B0F8E8100398F5F73AFD0020EC
:10B91000F5F7C1FD2F902868B0F8EC10009190F871
:10B92000EB3090F8EA2001210298F5F7CAFC28686C
:10B93000B0F8EC10009190F8EB3090F8EA2001217B
:10B940000398F5F7BEFC0020F5F7A5FD14ACF6F75B
:10B9500014F8FDF757F8012805D02046F6F7C6F988
:10B96000002800F02981F5F71BFE179900221AAC78
:10B97000002054F822C0BCF1000F84BF02EB420348
:10B9800006EB831308D931F8027B03EB4008401C17
:10B99000A8F80A718445F6D8521C022AE8D3029806
:10B9A000F4F732FE2A900398F4F72EFE29900298BD
:10B9B000F5F790FB2C900398F5F78CFB7D4D2B90C1
:10B9C0002868B0F8EE10009190F8EB3090F8EA207B
:10B9D00001210298F5F775FC2868B0F8EE10009187
:10B9E00090F8EB3090F8EA2001210398F5F769FC14
:10B9F00000250020F5F74FFD00210298F4F7EFFD38
:10BA000000210398F4F7EBFD0DF10808012158F827
:10BA10002500F4F7E4FD1AA8002450F825701CA8AE
:10BA2000002F50F825A032D904A800EB451905EBEA
:10BA3000450006EB8018002119F804B00846F5F718
:10BA400043FD012000FA0BF102A88B4650F82500B7
:10BA5000F5F733FB6FEA0B010920F5F735FD0DF122
:10BA6000500BF5F78AFFFCF7CDFF012804D05846AC
:10BA7000F6F73CF900287CD0F5F792FDBAF8000003
:10BA800008EB4401641CA1F84A01BC42D3D3002155
:10BA90000846F5F719FD6D1C022DAAD32A990298C4
:10BAA000F4F79DFD29990398F4F799FD2C990298D4
:10BAB000F5F703FB2B990398F5F7FFFA3D4C206847
:10BAC000B0F8F010009190F8EB3090F8EA200121E6
:10BAD0000298F5F7F6FB2068B0F8F010009190F8A6
:10BAE000EB3090F8EA2001210398F5F7EAFB0120FA
:10BAF000F5F7D1FC14ACF5F740FFFCF783FF012804
:10BB000004D02046F6F7F2F800285BD0F5F748FDA0
:10BB1000179900221AAC002054F822C0BCF1000F83
:10BB200084BF02EB420306EB831308D931F8025BB2
:10BB300003EB4007401CA7F88A518445F6D8521CF5
:10BB4000022AE8D301203099F5F705FA01202E9951
:10BB5000F5F77AFC28990298F5F74BFA279903989C
:10BB6000F5F747FA24980090229B209A1E99029894
:10BB700000E024E0F5F7A5FB25980090239B219A8F
:10BB80001F990398F5F79DFB26990298F5F7F9FBA5
:10BB900001990398F5F7F5FB2F98F5F77CFC2D98A4
:10BBA000F5F7D2FD31B0BDE8F08F000099410020DB
:10BBB00050E3010094410020F9F7ADFCC9E6F9F724
:10BBC000AAFC50E7F9F7A7FC97E72DE9F04FADF68F
:10BBD000F42DFF224FF4056102A80EF094FDFF2220
:10BBE0004FF423710DF658000EF08DFD02A8CDF82C
:10BBF0005808FFF71DF9FE4D4FF0000495F800A01E
:10BC00001AF0800F73D0DDF858080DF6580290F83E
:10BC100020C090F82110503001FB0CF300EB4300E2
:10BC20000023002908D902EB430730F8026B5B1CA4
:10BC3000A7F88A609942F6D80023BCF1000F08D912
:10BC400002EB430730F8026B5B1CA7F8CA609C4507
:10BC5000F6D80023002907D902EB430730F8026B1E
:10BC60005B1CBE809942F7D80023BCF1000F08D9B5
:10BC700002EB430730F8026B5B1CA7F844609C455D
:10BC8000F6D830F8023BA2F8863030F8023BA2F832
:10BC9000883030F8023BA2F88430002600230029C7
:10BCA00088BF02EB861708D907EB430930F8028BEF
:10BCB0005B1CA9F80A819942F6D80023BCF1000F59
:10BCC00088BF02EB861708D907EB430930F8028BCF
:10BCD0005B1CA9F8CA819C45F6D8761C032EDDD3DF
:10BCE0006046FFF786F94FF0010887E0FFE7C1489B
:10BCF0000DF658064FF00008006890F8B40000F008
:10BD00000F0700F0A6FA012809D00F213846F9F7ED
:10BD100099FC012808D0002000F098FA6EE000217C
:10BD20000846F5F724FD02E0012000F08FFAB24842
:10BD300090F80090B1480778002F18BFB9F1000FB4
:10BD40005AD0DDF858084FF4006180F8209080F850
:10BD5000217080F8224080F8234050300EF0C9FC5A
:10BD6000F6F76DFA1AF0210F04D0324639464846EC
:10BD7000FFF7E3FC1AF0030F3CD0BA460196F5F743
:10BD8000DBFD06460220F5F7DFFCFF210F20F9F767
:10BD9000EEFDF5F705FC3046F5F7D6FCDDF85888E2
:10BDA000002108F15000009053464A460846F6F735
:10BDB0004EF90020F6F70FFA00260AFB09FBBBF14B
:10BDC000000F0AD908EB4607B7F85000F6F709FA52
:10BDD000761CA7F85000B345F4D8894800781D2890
:10BDE00004BF08F15000FDF70FF951464846019A8B
:10BDF000FFF7FFF84FF00108F5F761FD9DF8280007
:10BE00009DF82910CDF8E40AB8F1000F19BF0028F9
:10BE100000290DF6F42DBDE8F08F0020069074483F
:10BE20000078CDF8EC0A10F0020F00F0D38000206B
:10BE3000DDF8586847F6FF7ADDF8E42A06F1500885
:10BE40006FEA0A09009005460190002947D9694820
:10BE50000068CDF8E80A05FB02F0012438F910303B
:10BE60004FF0000B1F46BC46012A17D905FB0240C4
:10BE700038F910006045C8BF84469842B8BF0346F1
:10BE8000B0EB070E48BFA7EB000E0FFA8EF75F4529
:10BE9000C8BFBB460746641C9442E7D3CC45C8BF25
:10BEA000E1465345B8BF9A46BCEB030048BFA3EB3D
:10BEB0000C0000B2DDF8E83AB3F9C030834205DB8C
:10BEC000DDF8E80AB0F9C200834505DD012000FA7B
:10BED00005F30198184301906D1C8D42BBD30025DA
:10BEE000002A45D943480068CDF8E80A38F91530EA
:10BEF00001241F46BC464FF0000B012917D904FB53
:10BF0000025038F910006045C8BF84469842B8BF57
:10BF10000346B0EB070E48BFA7EB000E0FFA8EF7F3
:10BF20005F45C8BFBB460746641C8C42E7D3CC457F
:10BF3000C8BFE1465345B8BF9A46BCEB030048BFB3
:10BF4000A3EB0C0000B2DDF8E83AB3F9BC30834251
:10BF500005DBDDF8E80AB0F9BE00834505DD012008
:10BF600000FA05F30098184300906D1C9542BDD36C
:10BF70000198F06218B1306940F008003061009813
:10BF8000B06218B1306940F004003061A6F824A016
:10BF9000A6F82690BDF9DC28B9EB020048BFA2EB59
:10BFA0000900144A1368B3F9B820904203DD3069E0
:10BFB00040F002003061BDF9DC28B2EB0A0048BF56
:10BFC000AAEB0200B3F9BA20904203DD306940F0D9
:10BFD00001003061DDF8EC0A054C10F0010F05D0CE
:10BFE0000DF65802DDF8E40AFFF742F9207809E07F
:10BFF00099410020944100209E4000209F40002055
:10C000000D41002010F0400F2FD10798401C0790E1
:10C010000698002814BF0998089800F1010014BF81
:10C02000099008900DF65800FEF771FF00200246B7
:10C030000590049802A98C46B0F5056F94BF03469D
:10C040004FF405630020B0EB930F06D25CF820405C
:10C05000401C2244B0EB930FF8D35042C8604FF419
:10C060002C304FF40562F6F743FC0A208DF80000EF
:10C070009DF818008DF801009DF819008DF8020058
:10C080009DF81A008DF803009DF81B008DF8040040
:10C0900005226946012000F039F80DF6F42DBDE8BF
:10C0A000F08F00006549C2B2C0F307200A804880C3
:10C0B000704762484188008861F31F207047DFF8AD
:10C0C0007CC101238340BCF800C013EA0C0F08BFF9
:10C0D000704700B583B000F03F008DF800008DF888
:10C0E00001108DF80220100A8DF80300100C8DF855
:10C0F0000400100E8DF8050000208DF806008DF864
:10C10000070068460EF0B6FD03B000BDDFF82CC195
:10C1100001238340BCF800C013EA0C0F08BF70472E
:10C1200010B582B000F03F008DF80000072A88BFEC
:10C13000072200206B46002A09D911F800C01C18FC
:10C14000401C84F801C09042F7D3072805D2002193
:10C150001A18401C51700728FAD318460EF08AFDB1
:10C1600002B010BDDFF8D4C001238340BCF802C088
:10C1700013EA0C0F08BF704710B582B000F03F0003
:10C1800040F080008DF80000072A88BF07220020B9
:10C190006B46002A09D911F800C01C18401C84F80D
:10C1A00001C09042F7D3072805D200211A18401C7D
:10C1B00051700728FAD318460EF05CFD02B010BD8E
:10C1C00070B51E4D82B040EA0122AC880228234699
:10C1D00002D0052805D009E0002918BF022905D1A1
:10C1E00003E0002918BF022900D11446A34204BF6E
:10C1F00002B070BD0126F6F7DDFF297844EA004061
:10C2000011F0080F17D003218DF800108DF8016090
:10C210008DF80200010A8DF80310010C8DF804104E
:10C22000000E8DF8050000208DF806008DF807003F
:10C2300068460EF01FFDAC8002B070BD9A41002030
:10C24000FE4908707047FD4800787047FB49487008
:10C250007047FA48407870472DE9F04FF74891B0A1
:10C2600000214170FCF7CEFB012806D1F9F71AF93D
:10C2700003281CBF11B0BDE8F08FF04C207810F0FF
:10C28000010F07D0FFF7A1FC207820F001002070FB
:10C29000FCF7B4FB207810F0020F00F0DF81E848D3
:10C2A000E64900684978B0F858000229C0F3032035
:10C2B0000DD0E24CA17801F00F01F9F7C3F9012884
:10C2C0000CBF02200020607005D000F0AEB9002144
:10C2D0000846F5F74CFAF5F72FFBDFF860A30E9050
:10C2E0009AF8020010F0100F18BFF5F7A5FFFF2114
:10C2F0000F20F9F73CFBD34800780490D24800782F
:10C300000590D24890F800B0D14800780D9005987B
:10C3100000281CBF0498002813D0FEF7A4F8FEF7ED
:10C3200098F80020F7F734FE0020F7F77EFE9AF821
:10C33000020010F0100F0CD00120F7F78BFE012047
:10C340000BE00D98002818BFBBF1000FE5D100F0FD
:10C350006CB90020F7F77EFE0020F7F77BFE012086
:10C36000F4F7CDFDF5F7F1FA1E20FCF7A3FD00214F
:10C370000846FCF733FD814601210020FCF72EFD25
:10C38000DDE904128046002001FB02F7002F84BF84
:10C39000B0494A0C06D929F8101028F81020401C82
:10C3A0008742F8D81E20FCF72BFF00210120FCF764
:10C3B00015FD054601210846FCF710FD04460D99C0
:10C3C00000201BEB01061CBFA2494A0C06D025F831
:10C3D000101024F81020401C8642F8D800200C9041
:10C3E0009648808800287DD9701C40080F90FCF783
:10C3F00009FB012876D006A8F5F778FC002872D052
:10C400000798E8B38D48807810F0100F08D0DDF859
:10C410001CA0FDF7B4FF51460FF0EEFD824614E07C
:10C420000020002300900190029003901A461946C4
:10C4300007980EF00DFF82468048807810F0200F9C
:10C4400003D0FDF79CFF824609E0F7F7BDFA059A95
:10C450000092524601461046049B0FF0FFFDBAF1D0
:10C46000000F1CBF0020002F12D93AF9101039F923
:10C4700010208A42B8BF29F8101038F9102000E0C7
:10C4800006E08A42C8BF28F81010401C8742ECD84A
:10C490000E9810F0010F1CBF0A98002831D0674891
:10C4A000807810F0200F09D000210A980FF080F951
:10C4B000FDF76BFF5FEA000A23D00BE0DDF828A050
:10C4C000F7F763FA022200925246014610460F9B8C
:10C4D0000FF0C4FD0020002E13D93AF9101035F9E1
:10C4E000102001E01BE012E08A42B8BF25F81010CE
:10C4F00034F910208A42C8BF24F81010401C86422C
:10C50000EBD8F5F729FC0C98401C0C9002E0F9F7E9
:10C5100002F80C98494989888842FFF468AFF5F71A
:10C520003FF8FDF796FFFDF7BFFF44490C98898857
:10C53000884274D30E9810F0020F26D000224FF6D6
:10C54000FF731046002F0ED939F9101038F910C0BA
:10C55000A1EB0C019142C8BF0A469942B8BF0B46F5
:10C56000401C8742F0D80B208DF80000100A8DF88F
:10C5700001008DF80220180A8DF803008DF80430B0
:10C58000052269460120FFF7C1FD0E9810F0010F4A
:10C5900045D000224FF6FF731046002E0ED935F914
:10C5A000101034F910C0A1EB0C019142C8BF0A462B
:10C5B0009942B8BF0B46401C8642F0D80020BBF120
:10C5C000000F84BF0D9901EB0B0616D9A6EB000CEA
:10C5D00005EB4C0104EB4C0C31F8027CABEB000199
:10C5E00005EB410804EB4101A8F866703CF802CC69
:10C5F000401CA1F866C08345E8D80D208DF80000E6
:10C60000100A8DF801008DF80220180A8DF8030039
:10C610008DF80430052269460120FFF777FD3020B0
:10C62000FCF748FC3020FCF7EBFDF5F748F9034830
:10C63000017821F0020101700EE00000A04100200D
:10C64000944100209E4000209F400020A3400020F5
:10C65000A44000200080FFFFFCF7D0F9F8F722FF8C
:10C6600003281CBF11B0BDE8F08FF8F754FFF9E5BF
:10C670000449887070470348807870470149888072
:10C6800070470000A0410020FB4908707047FA483D
:10C6900000787047F84982B26FF30F00C1E90402D5
:10C6A0007047F54880787047F34A0028516914BFF5
:10C6B00041F0020021F0020050617047EE48007D19
:10C6C000C0F340007047EC4AF02303EA00105169C0
:10C6D00021F0F001084350617047E748007DC0F346
:10C6E00003107047E44A0028516914BF41F001006B
:10C6F00021F0010050617047DF48007D00F001002B
:10C700007047DD4B19690A0E120721F07F4142EA9A
:10C710000060084318617047D7480069C0F30360A0
:10C720007047D5480069000F7047D4480068406DD5
:10C73000C0F303607047012101FA00F04FF47F015C
:10C7400001EA0041CC4802691143016170470121AF
:10C7500001FA00F04FF47F0101EA0041C648026986
:10C7600022EA010101617047C3480069C0F3074034
:10C770007047C148008AC0F303307047BE4910B506
:10C78000024608694FF47043C0F3033420F470404C
:10C7900003EA02331843086103210846FFF78FFCC0
:10C7A000204610BDB448808AC0F38020704770B521
:10C7B000B14E0446C0F380007569C5F3002188427C
:10C7C00010D0F7F79CFB14F0040F05D006F0FFFD26
:10C7D000012808BF002003D0A94890F86C00C008C9
:10C7E00002F09BFB14F0010F14BF45F0400025F050
:10C7F000400014F0040F14BF40F4807020F48070E7
:10C8000014F0080F14BF40F4007020F4007014F00E
:10C81000100F14BF40F4806020F4806014F0200FEB
:10C8200014BF40F4006020F400607061BDE8704007
:10C83000FEF77BB890484169002011F0400F18BF07
:10C84000012011F0200F18BF40F0020011F4807F8A
:10C8500018BF40F0040011F4007F18BF40F008003A
:10C8600011F4806F18BF40F0100011F4006F18BF72
:10C8700040F0200070478048007DC0F38010704772
:10C880007D48007DC0F3401070477B48808AC0F32C
:10C89000002070477848808AC0F340207047FDF739
:10C8A0005BBE7548808AC0F3C02070477248808A9A
:10C8B000C0F30030704770484069C0F3003129B1BF
:10C8C000C0F34010002804BF0120704700207047CB
:10C8D00069498A691043886170476749C861704730
:10C8E0006548007F00F0010070476348007FC0F397
:10C8F000400070476048007FC0F3800070472DE91A
:10C90000F04387B00546F8F7CDFD0446F8F7CDFDB6
:10C91000594F8046052C0CBF5A4E5B4E387DC0F3F4
:10C92000031218BFB8F1050F05D1FFF7C4FF0028A7
:10C9300018BF42F0020211462846F8F783FE00288D
:10C9400004BF07B0BDE8F083FDF78DFDF7F77EFA71
:10C950000546F6F732FC0020F4F7D1FAF5F70DF8AA
:10C960004FF00009FCF74EF8012809D0F8F79AFDBE
:10C97000A04205D1F8F799FD404508BF002D0AD027
:10C98000F4F70EFEFDF790FDF8F7B2FFF6F751FC55
:10C9900007B0BDE8F0836846F5F7A8F9C0B1052CEB
:10C9A0000CD0B889401C81B2B981142906D9022261
:10C9B00032210120FFF783FBA7F80C906846FCF7B3
:10C9C00065FD6846B047050008BFF4F7D6FFC9E724
:10C9D000F8F796FDC6E7284AD080118170472DE907
:10C9E000F04385B0294A002104911578284A0B4666
:10C9F00016780091019102910A46039104A90EF064
:10CA000027FCFDF7BCFC81464FF000084A4647462C
:10CA1000002E25D932F9021B00234FF0010C012D05
:10CA200011D932F9024B611A09B220F8021B002910
:10CA3000B8BF494209B29942C8BF0B4621460CF122
:10CA4000010CAC45EDD320F8023B4345C8BF9846E6
:10CA50007F1CB742DED3B8F10F0FC4BF0120049092
:10CA60000C480078012804BF4846FCF7CDFA04982A
:10CA700005B0BDE8F0830000A841002094410020EB
:10CA80008483002047D0010037DA01009E40002057
:10CA90009F4000200D4100202DE9F84FDFF800B441
:10CAA00004460026BBF90690FE48FF490096007830
:10CAB000097837464518F8F7F5FCF6F782FF824605
:10CAC000F6F763FF9BF8041000EB4108F748007885
:10CAD000032804BF4046FCF7ADFBBAF1000F7DD040
:10CAE0009BF804000AEB400AF0480078022804BFD3
:10CAF0005046FCF79FFB0020002D0CD93AF810108F
:10CB000038F81020114434F81020511A24F810106D
:10CB1000401C8542F2D8DFF8948398F8000006287C
:10CB200004BF2046FCF786FB0020691E1CBFBBF932
:10CB300008C00B4613D004EB400134F8102049889C
:10CB4000891A09B224F810100029B4BF4A420A46D3
:10CB50006245BCBF0E447F1C401C9842EBD3002FA3
:10CB6000C8BF96FBF7F60FFA86FA04EB450727F8DD
:10CB700002AC98F80000072804BF2046FCF75AFBD7
:10CB800000263046691E18BF0A4610D034F810102F
:10CB9000A1EB0A0109B224F810100029B8BF4942DC
:10CBA00009B28E42B8BF0E46401C9042EED327F821
:10CBB000026CB4F9000010F11E0F03DB37F9040C0E
:10CBC0001E2805DD0BF01AF8002818BFFCF7E1FD60
:10CBD000BBF81400C0F30020D0B100E008E006F07C
:10CBE000F6FB012812D006F0F2FB08280ED00FE069
:10CBF0000020002D8FD934F8101038F81020891A31
:10CC000024F81010401C8542F5D884E74FF0050940
:10CC10004E4508DD0120009098F80000142804BF5C
:10CC20002046FCF707FB98F80000012804BF2046C7
:10CC3000FCF700FB0098BDE8F88F2DE9F04F87B0B6
:10CC4000FDF746FCDFF868B2DBF80000B0F93610FB
:10CC5000B0F93400FDF768FAF7F751F9042000F055
:10CC60003EF9DFF83C9280B199F81400C0F340100F
:10CC700010B9FFF720FE40B9DBF80000806DC0F36B
:10CC800003400F2818BFF7F720F9052000F027F917
:10CC900058B1FFF710FE40B1DBF80000806DC0F323
:10CCA00003500F2818BFF7F710F9FF2089F8030089
:10CCB000F8F7F8FB022804BFDFF8F8A14FF00008EE
:10CCC0007DD1D9F81000C0F30364DBF80000A100A7
:10CCD000806DC9F82080C84000F00F05C9F8248095
:10CCE00021460220C9F82880FFF76AFA062C4DD2A7
:10CCF000DFE804F0690303036D6DD9F81000C0F399
:10CD0000036499F81400022CC0F3031212D01146E8
:10CD10002846F8F797FC002838D002210846F3F798
:10CD2000D9FAFDF7A0FBFDF794FBF7F78FF80500A4
:10CD300009D029E0FFF7BFFD002814BF42F002022E
:10CD400022F00202E3E799F8000000281CBF00016E
:10CD5000F4F77BF8F4F7F9FD89F80180564E574F48
:10CD6000FBF750FE01280BD0F8F79CFB022807D1F7
:10CD7000D9F81000C0F30360A04208BF002D06D010
:10CD8000FDF767FBFDF790FBF8F7B2FD5DE0684645
:10CD9000F4F7ACFFA0B16846FCF778FB68460EF0EC
:10CDA00072FE0546307838B1DAF8000080683860E5
:10CDB000DAF80000C0F80080F4F7CEFFD0E74DE0CD
:10CDC000F8F7A9FBCCE728460FF020F83DE0F8F78C
:10CDD00069FB0446F8F769FB0746052C0CBF384E83
:10CDE000384E99F81400C0F3031218BF052F05D16F
:10CDF000FFF761FD002818BF42F0020211462846E5
:10CE0000F8F720FC08B3FDF72EFBF7F71FF80546EF
:10CE1000F6F7D3F90020F4F772F8F4F7AEFDFBF75C
:10CE2000F1FD012809D0F8F73DFBA04205D1F8F744
:10CE30003CFBB84208BF002D19D0F4F7B1FBFDF759
:10CE400033FBF8F755FDF6F7F4F9FBF7DBFD0128A6
:10CE500004D0F8F727FB02283FF433AF0AF092FD25
:10CE6000F7F74CF807B0BDE8F04FFDF731BB684667
:10CE7000F4F73CFF40B3052C0ED0B9F80C00401C71
:10CE800080B2A9F80C00142806D902223221012010
:10CE9000FFF715F9A9F80C806846FCF7F7FA14E0DB
:10CEA000A8410020A4400020A340002012410020FF
:10CEB0009441002018E3010015400020704000203C
:10CEC00047D0010037DA010006E06846B0470500A8
:10CED00008BFF4F752FDA2E7F8F712FB9FE70D4AEF
:10CEE0000228117D1269C1F30311C2F3074205D074
:10CEF000012808BF11F0020F0AD002E011F0040F60
:10CF000006D0012101FA00F0104018BF012070473F
:10CF100000207047A8410020394A30B4146894F8C2
:10CF20006CC01CF0040F1ABF012222EA0C050CF0A1
:10CF30000105B0F90030B1F900201DB1E58AAA1A47
:10CF4000521E12B21CF0020F03D0A48AE31A5B1E19
:10CF50001BB21CF0040F19BF02800B8003800A80F3
:10CF600030BC70474FF6FF71A0F8B010A0F8B210B7
:10CF7000A0F8B410A0F8B61070472DE9F0470E469F
:10CF8000824606F0F7F9074606F0ECF900F1380999
:10CF9000002E18BF002588BF4FF6FF7811D098BF2C
:10CFA000BDE8F08705EB4500C0EB451007EBC0047A
:10CFB00094F8DE00012804BF94F89500002811D1F0
:10CFC00003E0BDE8F04701F0FBBEA4F8B080A4F890
:10CFD000B280A4F8B480A4F8B680224649465046F0
:10CFE00003F00AFA94F8E500022812BF032820464D
:10CFF00001F03AFD681CC5B2B542D3D3BDE8F08755
:10D000009842002000230028B4BF42420246002973
:10D01000B4BFC1F1000C8C4642B9BCF1000F05D081
:10D020000029ACBF4FF487705A2070474FEA0C4C70
:10D03000BCFBF2FC30B4FF4C002254F82250654592
:10D040001ED804EB82056D68AC4519D202EB420292
:10D0500013B200FB01F2002ABCBF5A4213B20028EF
:10D06000B8BFC3F1B40008DB0029BBBF584200B20F
:10D07000C3F5B47030BCB8BF704700B230BC704765
:10D0800004EB82056D68654598BF5A23521C12B2A5
:10D090001D2AD2DBDDE72DE9F001E7491025402606
:10D0A0008024E64A09684FF0200C670010B301287D
:10D0B00050D002281CBFBDE8F0017047488A3223D7
:10D0C00000FB03F84B8BB8FBF3F808FB08F8C2F839
:10D0D000148000EB001808EB4010B0FBF3F0404365
:10D0E0009061486F000F062823D2DFE800F0221E6F
:10D0F00022272B2F488A00EB80034FEA83084B8BB3
:10D10000C000B8FBF3F8B0FBF3F008FB08F84043AD
:10D11000C2E90580B1F87400C0F30330062808D2D4
:10D12000DFE800F00703070C10149580BDE8F0015C
:10D130007047A2F804C0BDE8F00170479680BDE8D2
:10D14000F00170479480BDE8F00170479780BDE81A
:10D15000F0017047488A498BC0EB00135B00B3FBBA
:10D16000F1F35B43536100EB4003C3EB4010B0FBB2
:10D17000F1F0404390619480BDE8F0017047AE4803
:10D1800000B5006890F87C10428A01FB02F3418BE5
:10D19000B3FBF1FCA94BC3F80CC090F87D005043E1
:10D1A000B0FBF1F0186102EB82008000B0FBF1F0FF
:10D1B0004043D8610020FFF76EFFA1484FF6FF7192
:10D1C0000180418000BD2DE9F04F8DB09846DDE92A
:10D1D00016760D46044606F0C5F8079006F0DEF810
:10D1E0000C900020009095484FF4A051B0F804A096
:10D1F0000B970191D0E905B004908F4801684B8AE4
:10D200004A8B9800B0FBF2F040430A9064205843E8
:10D21000B0FBF2F04043089003EB8300B0FBF2F068
:10D220004043099094F899C086481CF800700A3071
:10D2300047B1012F0AD0032F04BF1CF800000328B8
:10D2400050D007E01CF8000020B904E01CF80000F2
:10D2500001282FD00120DFF8F09194F8E520A9F102
:10D260000A07A7F10A0C022A1CBF94F8BB20012A66
:10D2700067D094F89930754A02EBC30252F8083C23
:10D28000039352F8042C02922A8806926A88059227
:10D2900094F8CC20002A76D094F89A2002EB42032E
:10D2A000C3EB42130C9A02EBC30292F8CC20002A83
:10D2B0006BD095E0DDF81CC001209CF80CC0BCF1DF
:10D2C000000FC8D003EBC30C0CEB031CBCFBF2FC3F
:10D2D00003EB4303DB00B3FBF2F252430CFB0CFB0A
:10D2E0000492B8E7079F01203F7B002FB3D003EBE8
:10D2F000C30707EB0317B7FBF2F703EB4303DB00AE
:10D30000B3FBF2F2524307FB07FB0492D845A2D3CA
:10D310004F4F07EB4C0333F8022CB2F5807F9AD9BC
:10D32000A2F5807292B223F8022C94F89930B2F5EB
:10D33000807F07EB43033CBF4FF4807223F8022C3D
:10D3400089E72A8803926A88029294F89930002229
:10D3500003F80C2094F89930DA5594F8993003F8D2
:10D36000092094F899E03A4B019A03EB4E0323F815
:10D37000022C94F89920012A86D1304A0023137098
:10D380005370937080E70EE0FFE794F89930304ACD
:10D3900002EB430232F8023CB34221D922F8026C7C
:10D3A00094F8CC20E2B9089A904594F8E52012D37D
:10D3B000022A10D0089A904512D394F899E0244B91
:10D3C00094F8CC2003EB4E0333F802ECB64588BF4B
:10D3D00023F8026C06E04FF4A0630222019301E0FF
:10D3E00094F8CC200A9B984538BF0222134B9B78B7
:10D3F000002B01BF94F89930012B94F8CC30032B0B
:10D400000AD1DFF838E001238EF80230104B1B8878
:10D41000B34284BF0E4B1E80D84529D3022A18BFC1
:10D42000002825D094F899300020D85594F89930E8
:10D4300010E0000090E6010098420020D441002056
:10D44000F44100203587002017870020B486002093
:10D450002287002003F8090094F8990010F80C3096
:10D46000642B3CBF5B1C00F80C30032000901AE0DA
:10D47000049B984501D2022A03D110B1022A21D07F
:10D4800011E094F89930002003F80C0094F89930DA
:10D4900003F8090094F89900C35D642B3CBF5B1C42
:10D4A000C3550220009094F899B0DFF8ECE50EEB3C
:10D4B0004B031BF8077033F8020CBFB1B04237D3EF
:10D4C0004AD946E094F899304FF0000003F80C0078
:10D4D00094F89930D85594F8993013F809006428D5
:10D4E0003CBF401C03F809000120DBE71BF80CC01F
:10D4F000BCF1000F23D0864216D2A0EB060CA0EBA5
:10D500006C0080B223F8020C94F89930000A0EEBFC
:10D5100043034FF6FF7C23F8020C94F899300CEA91
:10D5200000200EEB430307E0DDF82CC0604501D27C
:10D53000504401E010D90CE023F8020C0CE01BF879
:10D5400009C0BCF1010F07D9DDF804C06045EFD375
:10D5500002D9A0EB0A00EFE794F899700EEB4700B0
:10D56000012F30F8020C04D1DFF830C5009B8CF895
:10D570000030002808BF002163D0022A1CBF099A8E
:10D5800090455FD8079A000A92F82A20022A1DD3F4
:10D59000B1F81890069A0B8A09FB02F2B2FBF3F677
:10D5A000DDF80CA04A8BDDF814C009FB0AF9B9FBC1
:10D5B000F3F302FB0CFCB1F81280DDF80890BCFB21
:10D5C000F8FC02FB09F2B2FBF8F21BE0B1F8149090
:10D5D000069A0B8A09FB02F2B2FBF3F6B1F8168049
:10D5E000059ADDF80CA008FB02FC09FB0AF9B9FB5F
:10D5F000F3F34A8ADDF80890BCFBF2FC08FB09F85B
:10D60000B8FBF2F2A0F1010808FB036608FB02C2B6
:10D61000B6FBF0F3B2FBF0F2088A00FB03F007D38D
:10D620000B8BB0FBF3F04B8A498B03FB02F206E055
:10D630008B8AB0FBF3F04B8AC98A03FB02F2B2FB80
:10D64000F1F130E0B1F814C0069A0B8A0CFB02F23B
:10D65000B2FBF3FACA8A059E498A02FB06F6B6FBBC
:10D66000F1FB039E4FEA10100CFB06F6B6FBF3F835
:10D67000029E02FB06F6B6FBF1F9A0F1100606FBCE
:10D6800008F806FB09F606EB0B16B6FBF0F608EBFE
:10D690000A18B8FBF0F803FB08F001FB06F1B0FB39
:10D6A000FCF0B1FBF2F1FE4A02EBC70343F8080CB1
:10D6B00094F8993002EBC30242F8041CA880E98078
:10D6C0000DB0BDE8F08F2DE9F84FF649F64B014457
:10D6D0004FF0000E01F801EC0344012103F8011C96
:10D6E000F249744601EB40110091F149724601EB99
:10D6F000401B01F5A07101EB4019009800210BEBD4
:10D70000041809EB041700EB0416002008EBC10312
:10D7100007EBC10C06EBC10503EB800A4AF8202C8D
:10D720000CEB800A4AF8202C05EB800A401C00B262
:10D730004AF8202C0228EFDB481C01B20229E4DB66
:10D74000601C04B2022CD8DBDA48DB4E0021D0F892
:10D7500000C0A6F110070BEB0E1809EB0E1A002003
:10D7600006EBC10908EBC1050AEBC10407EBC103D5
:10D77000814207D1BCF87A2043F82020BCF87820F9
:10D7800049F8202053F8202005EB800B02EB8202A1
:10D7900052004BF8202C04EB800B401C00B24BF8DD
:10D7A000202C0228E4DB481C01B20229D7DBBDE8AB
:10D7B000F88F10B490F899C0C04C00230CF80430D6
:10D7C00090F899C00A340CF80430BA4B90F899C01C
:10D7D0001B6893F87430C3F303131B02153404EB76
:10D7E0004C0C2CF8023C90F899C0A4F16E0303EBAA
:10D7F000CC0C4CF8081C90F8991003EBC10141F8CF
:10D80000042C90F8990010BC5DE710B5044605F0B3
:10D81000C5FD014694F8E500022804BFB4F8B40041
:10D82000B4F8B6100BD094F89A0000EB4002C2EBAB
:10D83000401001EBC001B1F8B400B1F8B61094F893
:10D84000CC20022A04BFA4F8B400A4F8B61010BD7E
:10D850002DE9F041044605F0A1FD94F8E500984E4D
:10D86000022835D09348B4F8B650B4F8B410006824
:10D87000038B028AB0F81AC0478A05FB0CF595FBAA
:10D88000F7F05943B6F9005091FBF2F16B4393FB6B
:10D89000F2F3B6F9022002FB0CF292FBF7F2B1EBC5
:10D8A000030C48BFA3EB010CBCF10A0F16DA811A76
:10D8B00048BF111A0A2911DAA5F57F40FF380DD0AB
:10D8C0003088A4F8B4007088A4F8B600BDE8F081F0
:10D8D000B4F8B4003080B4F8B60002E04FF0FF3086
:10D8E00030807080BDE8F0812DE9F041044605F0FC
:10D8F00055FD01466948DFF8CCC100690CF10B0702
:10D9000000FB00F694F8E500022844D094F89A0051
:10D9100000EB4002C2EB401001EBC000B0F8B410C5
:10D92000B0F8B600B4F8B430B4F8B6205D1A05FB10
:10D9300005F8151A05FB0585B5420ADA94F89950E1
:10D9400015F80C50012D04BFA4F8B410A4F8B600CB
:10D9500013D094F8995007EB850636F8048CA3EBA6
:10D9600008084144A4F8B41036F8021C511A0844BF
:10D97000A4F8B600002005F80C0094F8990007EB15
:10D98000800020F8043C94F8990007EB800020F810
:10D99000022CBDE8F08194F89920B4F8B41007EB9C
:10D9A0008202B4F8B60022F8041C94F8992007EB20
:10D9B000820222F8020C94F89930012203F80C201C
:10D9C000B0E72DE9F04F90F899C08FB04FF4806325
:10D9D00000290CBF364C3C4C04EB4C14334D0292E6
:10D9E00005EB4C1705F5A5756544203C15F8015C61
:10D9F00007EB051606EBC10858F8206C921B039242
:10DA000090F8E520022A1CBF90F8BB00012842D004
:10DA100058F81C8C04EB051206EB0809CDF8389079
:10DA2000D2F80490D6689568106809EB0602DFF812
:10DA30009C9028441044D9F800A035445044D9F8AB
:10DA400004A0DFF874B05244D9F808A0D9F80C90BB
:10DA500055444E44DDF808A0DDF83890AAEB0909DA
:10DA6000CDF82090DDF80C90A9EB0809CDF82C90AA
:10DA7000DBF800908144CDF82890DBF8049009EBA6
:10DA8000020ADBF80890DBF80CB0A9440BEB060E99
:10DA9000DDF828B01CE0B2E022870020D44100204D
:10DAA000B4860020548C00205E8C0020148B002053
:10DAB00094880020984200203442002003870020F0
:10DAC000F84100207F860020D489002024420020D5
:10DAD0000BFB0EFB0AFB19BB9BFBF3FBBBF1000F1F
:10DAE00008BF4FF0010B4FEA8E2E4FEA8A2A9AFBAD
:10DAF000FBFA4FEA892999FBFBF99EFBFBFECAF171
:10DB0000000ACDF834A0DDF828A0C9F100094FEAD9
:10DB10008A2A9AFBFBFB00FB0EFA02FB09AA9AFB7E
:10DB2000F3FACDF828A0DDF834A000FB0AFA02FBD6
:10DB30000BAA9AFBF3FACDF824A005FB0EFA06FB1C
:10DB400009A999FBF3F9DDF834A0CDF8309005FB75
:10DB50000AF906FB0B9999FBF3FBDDF828A0DDF829
:10DB600020900AFB09FEDDF824A0DDF82C900AFBCA
:10DB700009EEDDF820A0DDF830909EFBF3FE09FBF6
:10DB80000AFADDF82C900BFB09A999FBF3F9DDF8F3
:10DB900038A0C844F244CDE900A8DDF828A0CBF5B0
:10DBA000806ECAF5806808FB00FBDDF824A0DDF874
:10DBB0003090CAF1000AC9F100090AFB05BB08FB55
:10DBC00002F809FB00F00AFB06880EFB05009BFB30
:10DBD000F3FB98FBF3F890FBF3F0CDF810B0CDE930
:10DBE000058009FB02F00EFB060090FBF3F00790A6
:10DBF000FF480022E84604AE00EB0C0315E0FC4AA7
:10DC000000206244039012F8012C02AB07EB0212D1
:10DC100002EBC10253F8204002EB8005401C00B229
:10DC200045F8204C0228F5DB20E013F8015C58F899
:10DC3000220007EB051505EBC10505EB820545F84C
:10DC4000200C002006EBC20513F801AC55F820901B
:10DC500004EB0A1A0AEBC20A4AF82090401C00B2F0
:10DC60000228F1DB501C02B2022ADEDBE0486044ED
:10DC700010F8010C07EB001000EBC10050F8200C6D
:10DC80000FB0BDE8F08F0288438862F30F018088EF
:10DC900063F31F419A4284BF63F30F0162F31F4194
:10DCA0000A0C824288BF60F31F4188B20A0C90427E
:10DCB00084BF62F30F0160F31F41080C704770B519
:10DCC0000146154691F8E560CA4B91F8991090F815
:10DCD00099202C88688801EB4101A3F1780C0CEBAA
:10DCE000810C022E19D03CF80A1C2CF8081C3CF8B8
:10DCF0000C1C2CF80A1C2CF80C4C3CF8041C2CF8BE
:10DD0000021C3CF8061C2CF8041C99182CF8060C74
:10DD100011F8011C012911D019E02CF8084C2CF83D
:10DD20000A4C2CF80C4C2CF8020C2CF8040C1A445D
:10DD30002CF8060C012102F8011C08E0ACF10C00E3
:10DD4000FFF7A1FF0446ACF10600FFF79CFFAC8093
:10DD5000E88070BD30B4002488B0A44601EB001107
:10DD600001EB4C0030F8100C04440CF101001FFAD8
:10DD700080FCBCF1080FF3D3E4081C6000231846B4
:10DD80006D4601EB400C3CF810CCACEB040C0CFBEA
:10DD90000CFC45F820C0401C80B263440828F0D336
:10DDA000D80831F80A3C31F8101C591A494311605F
:10DDB00008B030BC7047904A0021024402F8011CB0
:10DDC0008E4A024402F8011C8D4A024402F8011CEA
:10DDD0008C4A02EB800242F8041C8B4A02EB800260
:10DDE00042F8041C894A02EB800242F8041C884A6B
:10DDF00002EB800242F8041C864A02EB400020F845
:10DE0000021C418070472DE9FF4FE1B053B2002260
:10DE10005792814A1F461268B2F812C0528BCCEB5F
:10DE20000C1CBCFBF2F25092754ADFF8D0C10244E0
:10DE300012F8016C0CF10202844402441CF8015CEB
:10DE400012F8014C00EB800C01EB0C1C002E7DD075
:10DE50000CEB450131F8505C5495B1F850105391DA
:10DE600012F8011C143949B20029BCBF283149B24B
:10DE70000CEB410131F8502C5292B1F850101E2297
:10DE800051910CEB4401052A31F8504C5994B1F8EA
:10DE90005010589140F2E7815A49EE4601EB80015B
:10DEA00051F8044C58495E9401EB8000012150F870
:10DEB000040C5B90844268DD649800885A90501E80
:10DEC00058BF744612D40CEB430544F8201004EB01
:10DED00080065B1E35F8505C5BB2C6F8A050002B84
:10DEE000B8BF2723401E00B20028ECDA00210C4600
:10DEF000B846501E58BF754616D40CEB480355F86B
:10DF00002060B3F850307343A8F1010659184FFA56
:10DF100086F844EBE374B8F1000FB8BF4FF0270860
:10DF2000401E00B20028E8DA00252E46501E58BFD9
:10DF3000F1465CD40CEB470309EB8008B3F8503092
:10DF4000D8F8A0807F1E03FB08F300E00BE05D190A
:10DF50007FB246EBE376002FB8BF2727401E00B202
:10DF60000028E7DA7DE0611CCAB23CF8501C5491ED
:10DF7000BCF85010539125F00101614431F8505C18
:10DF80005295B1F8501051917BE76E9800885A90E5
:10DF9000501E58BF744612D40CEB430544F82010B1
:10DFA00004EB80065B1EB5F850505BB2C6F8A0507B
:10DFB000002BB8BF2723401E00B20028ECDA002156
:10DFC0000C46B946501E58BF75462ED40CEB49037B
:10DFD00055F8206033F8503C7343A9F101065918F5
:10DFE0004FFA86F944EBE374B9F1000F16E038E01C
:10DFF000548C0020E08C0020DC410020DA4100201D
:10E00000DE410020144200201C420020FC41002080
:10E01000044200200C42002098420020B8BF4FF07C
:10E020002709401E00B20028D0DA00252E46501ED7
:10E0300058BFF14615D40CEB470309EB800833F8C1
:10E04000503CD8F8A0807F1E03FB08F35D197FB217
:10E0500046EBE376002FB8BF2727401E00B200280A
:10E06000E9DA0027B8463846002AC8BFF4460ADD78
:10E070005CF8203000F101005B43DF1948EBE378E6
:10E0800000B28242F4DC0023CDE955331846002A61
:10E09000C8BFF44615DD0CEB80095CF82030D9F8D8
:10E0A000A09003FB09F3DDE955A94FEAE37B13EBED
:10E0B00009034BEB0A09401CCDE9559300B282429B
:10E0C000E9DC4FF0000AD1465046002AC8BFF346AB
:10E0D00010DD0BEB80035BF820C0D3F8A03000F11B
:10E0E000010003FB0CF313EB0A0A49EBE37900B2DE
:10E0F0008242EEDC4FF0000CE3466046002A0EDD63
:10E100006B4603EB800300F10100D3F8A03000B2AE
:10E110005B4313EB0C0C4BEBE37B8242F0DCA7FB85
:10E120000C32CDE95CCB08FB0C2207FB0B2CDDE9A4
:10E130005520A0FB0ABECDE95F2002FB0AE200FBEE
:10E140000922B3EB0B006CEB0202CDE95520104322
:10E1500004BF4FF0000B594632D0DDE95C03A0FB51
:10E16000012C5C9103FB01C100FB0411DDE95F3070
:10E17000A0FB05CB03FB05B300FB0633B2EB0C00A1
:10E1800061EB0301DDE955320CF0C2FA8346A7FBCF
:10E19000050108FB051107FB06125C99AAFB013C6F
:10E1A00009FB01C10AFB0411C01A62EB0101090459
:10E1B000DDE9553241EA104100040CF0A9FA0146AC
:10E1C0005A9848431BEB204048BF00205B9B5E9A57
:10E1D0009A4224DD549A539B4A430BEB2242D31AB2
:10E1E00044BF539B9B1A509A93423CD2529A51433C
:10E1F000519A0BEB21418A1A44BF519A521A5099F5
:10E200008A4230D25899091A44BF5899411A509AF3
:10E21000914228D26E9908800120579023E0539AAA
:10E22000549B4A430BEB2242D31A44BF549B9B1A84
:10E23000509A934217D2519A5143529A0BEB214173
:10E240008A1A44BF529A521A50998A420BD259994B
:10E25000091A44BF5999411A509A914203D26499BC
:10E26000088001205790579865B0BDE8F08F2DE9E0
:10E27000FF4F8DB09A468B46054605F073F8009027
:10E2800090F82A0002282CBF03200A20049095F859
:10E290009940022C94BF4FF001094FF0000995F806
:10E2A0007B0001281CBFFE48C06908D0019095F88A
:10E2B000E500FC4B4FF0000802283AD109E0FA488B
:10E2C00064220068418A408B5143B1FBF0F0404327
:10E2D000ECE71819B9F1000F00F8018CF34820445D
:10E2E00000F8018C80F80980F148204400F8018C86
:10E2F00080F80980EF4800EB440020F8028CA0F879
:10E300001280ED488BF8CC80204485F8CC8000F852
:10E31000018CEA48204400F8018CE948204400F8C8
:10E32000018CE848204400F8018C1CBF2046FFF710
:10E3300042FD0F981919B9F1000F0288E2480391C4
:10E3400000EB0410079011F8011C029100EB410052
:10E3500020F8102CBAF80010DC4AA0F8901076D003
:10E36000A2F122002044A2F120010590214410F8DE
:10E37000010C01F8010CA2F11E012144069111F8D3
:10E38000011C01B3411CC9B2282926D3D04904EB92
:10E39000840301EB031101EB400331F850EC33F837
:10E3A00050CCAEEB0C0C02EB840E4EF804CCB3F860
:10E3B0005030B1F85010CB1A02F1080101EB840182
:10E3C00041F8043C24E002EB840141F8048CC1498B
:10E3D00001EB840141F8048C1AE0BD4B04EB840C82
:10E3E00003EB0C1303EB410131F8503C31F852CCF4
:10E3F000A3EB0C0302EB840C4CF8043CB1F8503056
:10E40000B1F84E105B1AB34901EB840141F8043CAA
:10E410000F9904EB840C27280B88AD4901EB0C11F4
:10E4200001EB400121F8503CBAF80030A1F850301F
:10E4300003D1069B012103F8011C401C0599C0B2C1
:10E44000282801F8010C24BF059800F8018C95F8E4
:10E45000E500022800F080810020069005900298D7
:10E460000799C01D00F007000F9B01EB400030F83A
:10E47000101C1B88B0F89000591ABAF80030181A0E
:10E48000B9F1000F34D0944B234413F801CC934BD3
:10E49000BCF1000F03F1080648D003EB840C0029FF
:10E4A0005CF8047CACBF0B464B421F4406EB840374
:10E4B0004CF8047C53F804EC0028B4BF46420646EE
:10E4C000764402EB840243F8046C52F8042C002AD0
:10E4D000B8BF5242BA1A4CF8042C7E4A02EB8402AE
:10E4E00052F8042C002AB8BF5242B21A43F8042C46
:10E4F0006D4A1268138B5943138A91FBF3F6518BC3
:10E500004843518AB9F1000F90FBF1F704D07248EB
:10E51000204410F8010C00B3002E3CDD65484FF09C
:10E52000020100EB440020F8028C4CE003EB840273
:10E53000002952F804CCB4BF4B420B46634442F866
:10E54000043C06EB8402002852F804CCB4BF4342DA
:10E550000346634442F8043CCAE76148002E00EBDE
:10E56000440030F8022CB4BF714231468A4205DAC9
:10E57000002EACBF3146714220F8021C4288002FA9
:10E58000B4BF794239468A42C6DA002FACBF394659
:10E5900079424180C0E706DA4648012100EB440099
:10E5A00020F8028C0FE04248204410F8011C41483A
:10E5B00000EB440030F8022C642A04D2521C20F8EC
:10E5C000022C01200690002F07DD3A4A4FF004008C
:10E5D00002EB4402A2F8128015E007DA354A4FF048
:10E5E000030002EB4402A2F812800CE0314A3048EA
:10E5F00002EB44022044538A407A642B03D25B1C12
:10E600005382012205922A4A224412F8013C1BB38C
:10E610008B4222D1274B03EB440333F8023C3C2BC3
:10E62000224B234496BF13F801CC03F8018CBCF1B4
:10E63000640F2BD2DDF818E0BEF1000F26D10CF1EB
:10E64000010C0CF0FF0C03F801CCBCF10A0F1DD338
:10E65000194B234403F8018C18E0144B234413F89E
:10E6600001CCBCF1050FDFF850C0A44436BF1CF844
:10E6700001EC0CF8018CBEF1640F05D2062EA4BF8C
:10E680000EF1010E0CF801EC03F8018C537A4BB338
:10E69000834245D1074B03EB44035B8A3C2B22E0CA
:10E6A000D44100202A8E002098420020488E00206D
:10E6B000348E00205C8E0020848E00208E8E002000
:10E6C000988E00208A880020EA8C0020FC410020DF
:10E6D0004A87002004420020DE410020144200202E
:10E6E0000C42002035E0FE4B234496BF93F809C04E
:10E6F00083F80980BCF1640F2BD2DDF814E0BEF181
:10E70000000F26D10CF1010C0CF0FF0C83F809C0AE
:10E71000BCF10A0F1DD3F34B234403F8018C18E01E
:10E72000EF4B234493F809C0BCF1050FDFF8B4C3E5
:10E73000A44436BF1CF801EC0CF8018CBEF1640F48
:10E7400005D2062FA4BF0EF1010E0CF801EC83F8E0
:10E75000098002F8011C507202980399401CC0B253
:10E7600001F8010C08280AD3039800F8018C9BF8E3
:10E77000CC00002804BF01208BF8CC0006E09BF8F9
:10E78000CC00002808BF85F8CC8053D00AAB08AA7B
:10E79000D5492046FFF7DEFA83460BAB09AAD349D9
:10E7A0002046FFF7D7FA01998B4598BF88420CD9CC
:10E7B000032085F8CC00CE48CE492044214400F8FF
:10E7C000018C012001F8010C14E0C548204410F828
:10E7D000011C08299CBF407A082810D9032085F81D
:10E7E000CC00C3480121204400F8018CC1482044DA
:10E7F00000F8011C95F8CC00032839D01AE0BC4879
:10E80000204410F8011CC8293CBF491C00F8011C19
:10E81000B849214411F8011C012908D110F8011C44
:10E82000049881429CBF032085F8CC0020D90220A7
:10E8300085F8CC00B048204400F8018CA948204459
:10E8400000F8018CAD4802212044019000F8011C21
:10E85000AB48B9F1000F00EB040B0BF8011C04BF2F
:10E8600011B0BDE8F08F95F8CC00032810D012E06D
:10E87000A148204410F8010C042805D299482044EE
:10E8800010F8010C0428DDD3009902200873D9E7A1
:10E8900004F0A0FD28B12046FFF78DFA11B0BDE8C5
:10E8A000F08F9848204410F8010C01280ED0002861
:10E8B0001CBF11B0BDE8F08F9348204410F8010C44
:10E8C000401C07283CBF11B0BDE8F08F282ED8BFF0
:10E8D000282F09DC8D4800EB440030F8021C282961
:10E8E0009CBF408828280FD90098007B002804BFCF
:10E8F00011B0BDE8F08F0320019901F8010C0BF86D
:10E90000010C11B0BDE8F08F7F48CDF800A0204485
:10E910007F4910F8012C20460F9BFFF774FA01285D
:10E9200007D0019800F8018C0BF8018C11B0BDE8FC
:10E93000F08F0199012001F8010C0BF8010C11B0C6
:10E94000BDE8F08FB0F8B030B1F8B0C0B3EB0C0256
:10E9500048BFACEB0302B0F8B230B1F8B210581AAD
:10E9600048BFC81A02FB02F100FB0010704770B5E7
:10E970000D46044604F0F6FC94F8E500654E0228C6
:10E980001DBF94F8BB000128012DB4F8B4000FBFDF
:10E99000B4F8B62094F8990006EBC00151E90202E0
:10E9A00032213125B4F8B4C0B4F8B63005FB00C04C
:10E9B000B0FBF1F005FB0232B2FBF1F194F89920C3
:10E9C00006EBC20242F8080C94F8992006EBC2024A
:10E9D00042F8041CA4F8B400A4F8B61070BD2DE9E8
:10E9E000F0074D4A0F88B0F800801268DFF82CA1BC
:10E9F000B2F81890158AB2F81AC0568A07FB0CF4C0
:10EA000094FBF6F208FB09F393FBF5F314B2BAF8A2
:10EA100000201BB202FB09F999FBF5F5BAF8029048
:10EA20002DB209FB0CFC9CFBF6FC0FFA8CFC5E1B68
:10EA300048BFEE1A0A2E10DAB4EB0C0348BFACEB59
:10EA400004030A2B09DAA2F57F43FF3B1FBF0280B4
:10EA5000A1F80090BDE8F0077047AAF80080AAF876
:10EA60000270BDE8F00770472DE9F04F87B004460B
:10EA700000F0A0F9824600F0A0F9814604F08EFC77
:10EA8000059004F06FFCDFF890B08046007B94F8AE
:10EA90009950DBF80010002866D0086FC0F3C04220
:10EAA0000192C0F34042C0F3804004920090486F4E
:10EAB000C0F303410F021149294411F8011C022936
:10EAC0000EBF4FF44076C0F3035006020220FEF75B
:10EAD000E2FA1148006890F8700010F0010F1FE092
:10EAE000488E00208E8E0020EA8C00208A8D002027
:10EAF000988E00208A880020848E0020368700208F
:10EB000040870020DE410020DC4100200C42002034
:10EB10004A870020A48E002098420020F441002063
:10EB200000F02D8194F89A00B4F8B010ADF80810F8
:10EB3000B4F8B210ADF80A1000EB4001C1EB40117F
:10EB4000059802AA00EBC10B59462046FFF7B7F81B
:10EB50000198002841D0BDF80C00ADF80800BDF8C0
:10EB60000E00ADF80A003DE091F87000C0F3C0025D
:10EB70000192C0F34002C0F380000492009098F824
:10EB80001400012815D004F025FC38B104F01FFC56
:10EB9000012815D004F01BFC082811D0DBF8000078
:10EBA00090F8740001070F0DC0F303100602002057
:10EBB0008DE7B1F87400C0F3032007023E46F6E784
:10EBC000DBF80000B0F8740001070F0DC0F303205C
:10EBD000000200F58076012079E76E490020294483
:10EBE00001F8010C94F8E500022819BF94F8BB0065
:10EBF00001282846FEF767FDBDF8082000212046C1
:10EC0000FEF7DFFE0190BDF80A2001212046FEF745
:10EC1000D8FE01990029B8BF00210028B8BF002004
:10EC2000DFF874C1DCF80020B2F91030A3F1010E56
:10EC30008E45B8BF7146B2F91220531E8342B8BF49
:10EC4000184689B282B25548554BADF80C10ADF854
:10EC50000E2028442B4410F801CC13F801EC00F8E6
:10EC600001EC03F801CC009800281CBFADF8081097
:10EC7000ADF80A200DF10E0303AA59462046FFF70E
:10EC8000F6FAB4F8B020BBF8B000111A48BF811AE8
:10EC9000B4F8B220BBF8B230D01A48BF981A494332
:10ECA00000FB001398F80C00A8B93E48284410F85F
:10ECB000010C012807D070B93B48284410F8010C1A
:10ECC000401C282807D9BDF80C00ADF80800BDF895
:10ECD0000E00ADF80A00CDE9007698F82A2002A9C6
:10ECE0002046FEF770FA049838B1BDF80C00ADF874
:10ECF0000800BDF80E00ADF80A00BDF80800BDF828
:10ED00000A105045B8BF50464945B8BF4946224D44
:10ED10002A68B2F91030A3EB0A03A3F1010C844571
:10ED2000B8BF6046B2F91220A2EB0902531E8B4213
:10ED3000B8BF1946A4F8B400A4F8B61004F04AFB12
:10ED4000012804BF94F8E300012807D1B4F8B0000B
:10ED5000A4F8B400B4F8B200A4F8B600286890F89B
:10ED6000700010F0100F04BF07B0BDE8F08F98F8E6
:10ED70002A102046FEF7B8FD07B0BDE8F08FB4F8C2
:10ED8000B000A4F8B400B4F8B200A4F8B60007B01C
:10ED9000BDE8F08FE08C002098420020548C0020C9
:10EDA0005E8C0020DE410020DC410020FE487047E0
:10EDB000FE487047FE4800787047FD48407870472D
:10EDC000FB480E2181801221C180E02101814FF496
:10EDD0009071418170470346002002460029D8BF48
:10EDE000704753F822C0521C60449142F9DC7047CE
:10EDF0002DE9F05F0E46054604F0E0FA044604F003
:10EE0000D9FA310291FBF0FC290291FBF4F3DFF80F
:10EE1000A0E3E64D5E12BEF80490BEF80680002125
:10EE20004FEA6C2705F1E00A002C0BDD01FB03F231
:10EE300006EB222245F821204AF82120491C09B27C
:10EE40008C42F3DCD84E002106F1E00B00280BDDEC
:10EE500001FB0CF207EB222246F821204BF821207F
:10EE6000491C09B28842F3DC0CFB09FC03FB08F3E4
:10EE70004FEA6C315A135F13CEF80C102B684FEA2F
:10EE80006C3C9B1A2B6005EB840353F8045C15441F
:10EE900043F8045C33685B1A336006EB800353F875
:10EEA000045C0D4443F8045C9EF80330002BDAF850
:10EEB000003017D09B1ACAF800300AEB84030BEB22
:10EEC000800053F804CC624443F8042CDBF80020A3
:10EED000521ACBF8002050F8042C114440F8041CBE
:10EEE000BDE8F09F9A1ACAF800200AEB84020BEBE7
:10EEF000800052F8043C3B4442F8043CDBF800201C
:10EF0000511ACBF8001050F8041C6144E6E7A848F9
:10EF1000C078012818BF002070472DE9F047A54EA2
:10EF20000446A34D30684FF01209478AB0F81080AC
:10EF30000E20142C03D2A4F10F01052903D2A880BE
:10EF4000A5F806901EE0A4F10A01052903D21420B9
:10EF5000A880E88016E0611F052903D21620A8804A
:10EF6000E8800FE0052C28BFA88009D204F032FA0F
:10EF700000281DBF1820A880E880A5F8049001D1C2
:10EF8000A5F806900021FCB13068428A408BC2EBA4
:10EF90000212B2FBF0F0A870E970AA884FF6FF7079
:10EFA00000EA02122A81EA8800EA021068813068C9
:10EFB000428A408B6243B2FBF0F028706970414690
:10EFC0003846BDE8F04713E7A9700120E870E4E790
:10EFD00070B578480E24E025026892F86C30508AAB
:10EFE000DB0803FB00FC538B118ABCFBF3FC704A6B
:10EFF00082F800C04FF0000C82F801C09480122407
:10F00000D48015814FF490755581C0EB0015B5FB88
:10F01000F3F393704FF6FF7482F803C0FFF7E8FE36
:10F020006549002001EB800221F82040401C80B29D
:10F0300054800A28F6D370BD2DE9F04FB3B00D46C9
:10F040000446CC225D4968460BF04EFB5948B5F9A1
:10F0500002200068012A90F807C090F80680478ACD
:10F06000068A687800FB0CF109B2D8BF01222B7820
:10F07000DFF84CE1EB4683B1ACF101094B45194493
:10F0800017D104EB410131F9021C0129D8BF01213C
:10F09000C902494291FBF2F140E004EB4101B1F9B0
:10F0A00002100129D8BF0121C90291FBF2F109B276
:10F0B00035E004EB410939F9021C0129D8BF0121CF
:10F0C000B9F90290B9F1010FD8BF4FF001094FF023
:10F0D000640A01FB0AF109FB0AF901EB620109EB81
:10F0E000620991FBF2F199FBF2F93BF911103BF93E
:10F0F0001990494508BF002111D001EB090A1AF502
:10F10000004FB8BFF24604DBBAF5004FA8BF47F680
:10F11000FF7AA1EB0901C90291FBFAF109B2A0B192
:10F12000A8F101094845A0F1010909FB0CF90FFA02
:10F1300089F9994415D134F91940012CD8BF01241B
:10F14000E402644294FBF2F255E003EB0C0934F95B
:10F150001940012CD8BF0124E40294FBF2F212B250
:10F160004AE034F91990B9F1010FD8BF4FF0010905
:10F1700000F1010A0AFB0CFA0FFA8AFA9A4434F9F0
:10F180001AA0BAF1010FD8BF4FF0010A642409FB9D
:10F1900004F404EB620494FBF2F44FF064093BF9CD
:10F1A00014400AFB09F90DE0F48E0020648F002062
:10F1B0004442002098420020B490002008E701005B
:10F1C0000080FFFF09EB620999FBF2F23BF9122084
:10F1D000944208BF00220FD004EB020919F5004F3A
:10F1E00005DBB9F5004FB4BFCE4647F6FF7EA21A45
:10F1F000D20292FBFEF212B21B04000403EB0111D7
:10F2000000EB021201F5004002F5004190FBFCF01A
:10F2100091FBF8F1704301FB07F100144FEA214123
:10F220004CBF00220246B242C8BF304602DC002872
:10F23000B8BF00200029B4BF00220A46BA42C8BFA6
:10F24000394602DC0029B8BF0021A5F8B000A5F8B6
:10F25000B21033B0BDE8F08F2DE9FF4FFFB00E467E
:10F260009146702168460BF044FA70211CA80BF0FF
:10F2700040FA702138A80BF03CFA702154A80BF02A
:10F2800038FA04F08BF8044604F06CF87B9004F034
:10F290007BF800F13808739004F094F8789004F04B
:10F2A00089F8054604F08AF80746FE480068418A56
:10F2B0007091008A719004F08DF8012812D104F049
:10F2C00086F801280ED1DFF8E0A31820AAF8040080
:10F2D000DDE97001FFF78CFDF448DAF80C20016BD2
:10F2E00011440163F2487A907038799099F80000DF
:10F2F00099F8011099F8993001FB050099F89A10D6
:10F30000305C01EB4102C2EB411104EBC102E9495F
:10F3100000F03F0001EB830C3CF8041C7291A1F556
:10F320007F43FF3B1DBF3CF8021CA1F57F43B3F1B7
:10F33000FF0393880CBFD188729BB9F80440749482
:10F3400004F1050ADC4CA4FB0ABACAF3CF0ACDF8D3
:10F35000F0A1B9F806A00AF1050BA4FB0BEBCBF367
:10F36000CF0BCDF8DCB103F1050BA4FB0BEB01F1E6
:10F37000050EA4FB0EE4C4F3CF047694749C4CF603
:10F38000CD4E04FB0EF4E40C75940AFB0EF4E40C71
:10F390007D9403FB0EF4E40C7494DDF8F0A1CBF340
:10F3A000CF0B01FB0EF44FEAD44EDA4504BFDDE982
:10F3B000764AA24506D0DDE9744AA24504BF7D9C89
:10F3C00074450FD17B9C94F82A40022C0AD3DDF8B7
:10F3D000CCA19AF82AA0A24504BF99F89840022C23
:10F3E00000F0C9804FF6FF712CF8041CB14A99F85F
:10F3F000993002EB830222F8021C99F80AA099F8CE
:10F400000B10729199F80C4099F80D10729AE94618
:10F410000DF1700E8A4228D802FB05F31FFA83FB18
:10F420005346A2451DD8DDF8FCC10BEB03083CF99F
:10F4300018C016F8088008F03F0880450DD1DDF8A7
:10F44000E081C44509DB59F82380E04449F8238072
:10F450005EF82280C4444EF822C05B1C9BB2A342DB
:10F46000E1D9521C92B28A42D6D900214A460846B6
:10F47000002D40F3E48052F82030401C1944A8428B
:10F48000F9DB002940F3DB80002172460846002F9B
:10F4900040F3D58052F82030401C19448742F9DCF3
:10F4A000002940F3CC800020002D88BF38A90BD95B
:10F4B000799A59F8203052F820205A4341F82020F8
:10F4C000401C80B28542F3D80020002F88BF54A989
:10F4D0000BD97A9A5EF8203052F820205A4341F82E
:10F4E0002020401C80B28742F3D8002138AA084669
:10F4F000002D05DD52F82030401C19448542F9DC0E
:10F5000000224B461046002D05DD53F820C0401C5C
:10F5100062448542F9DC91FBF2FC002154AA0846C2
:10F52000002F05DD52F82030401C19448742F9DCD9
:10F53000002273461046002F05DD53F82040401C82
:10F5400022448742F9DC91FBF2F0BCF1000FB8BF16
:10F550004FF0000C0028B8BF00207199491E8C455F
:10F56000C4BF7199A1F1010C7099491E8842C4BFB2
:10F570007098401E66E0DDF8C8B14E4C4FF6FF7A39
:10F58000D34504BF3CF802BCD34507D12CF8043C5A
:10F5900099F8993004EB830323F8021C917A99F8C7
:10F5A0000A30994238BF89F80A10D17A99F80B309D
:10F5B000994238BF89F80B10117B99F80C309942A9
:10F5C00088BF89F80C10517B99F80D30994288BF9B
:10F5D00089F80D1099F80AA099F80BB0CDF8C8B1C8
:10F5E0001378527899F80D1002FB053299F80C4007
:10F5F00018F802208B4502F03F093FF607AF0BFBDE
:10F6000005F292B273925246A24511D8739B1344ED
:10F6100018F803C00CF03F0ECE4505D12CF03F0C7E
:10F620004CEA000C06F803C0521C92B2A242EDD97B
:10F630000BF101021FFA82FB8B45E0D9E6E64FF0A1
:10F64000000C60468299A1F800C08C9908800DF5E5
:10F65000037DBDE8F08F2DE9F34FF9B00546CC22CC
:10F66000164968460BF040F8CC22154933A80BF038
:10F670003BF8002076906D904FF4947078900020C5
:10F6800077907A98027841780648D0F800C09CF8C4
:10F6900007309CF806007490BCF812006E90BCF81D
:10F6A00010000FE09842002044420020D48F002038
:10F6B00044900020B4900020CDCCCCCCD4E7010005
:10F6C000A0E80100709074984FEA40086E98B0FB73
:10F6D000F8F970984FEA4308B0FBF8F84FF6FF705E
:10F6E00000EA490A00EA48007190002075907A9873
:10F6F000CDF8BCA19CF807B090F800A04078002A93
:10F7000000FB0BA00FFA80FA7CD0581E904278DDE7
:10F7100001206C90501E01FB03000FFA80FB501C6F
:10F7200001FB030000B235F91AE035F91BA035F9E9
:10F7300010006EF31F445045C4BF60F30F046AF31A
:10F740000F0605DC60F30F0601206AF30F047690C4
:10F7500020B20028BCBF002060F30F0430B20028A4
:10F76000BCBF002060F30F060FFA84FB0EEB0B000A
:10F770004FEA0E3ABAFBF0FACDF8CCA14FEA0B3AB9
:10F78000BAFBF0F0DDF8CCA17290AAEB000041F6D4
:10F79000333B75900FFA86FA00FB0BF00AFB00F082
:10F7A000B0FBFEF0DDF8CCA1000B0AFB00F0CDF8B9
:10F7B0009CA100F50060DDF8D8A1000BBAF1000FA4
:10F7C000DDF8C8A114BFCDF898A1CDF8A0A145D00F
:10F7D00068900020824672906C98012808BF002033
:10F7E0006BD002287DD0DDE966A0A0EB0A0ABAF54D
:10F7F000406F9ABF0120EB4608F1020072D9C5E0C4
:10F8000000E02DE002206C90012001FB030000B21B
:10F8100035F91AA035F910006AF31F4460F30F069A
:10F82000BAF1000FBCBF4FF0000A6AF31F44002872
:10F83000BCBF002060F30F064FEA244A0FFA86FB94
:10F840000AEB0B004FEA0A3ABAFBF0FACDF89CA19A
:10F850004FEA0B3ABAFBF0F0689000206690B8E7E8
:10F8600003206C90501E01FB030000B235F91AA072
:10F8700035F910006AF31F4460F30F04BAF1000F6A
:10F88000BCBF4FF0000A6AF31F440028BCBF002031
:10F8900060F30F044FEA244A0FFA84FB0AEB0B00D3
:10F8A0004FEA0A3ABAFBF0FACDF89CA14FEA0B3ABC
:10F8B000BAFBF0F0669000208AE70DF5CC7BDDF80E
:10F8C000C8E15BF820B0DE44CDF8C8E102EB000EE1
:10F8D000AEF1010E401C0BFB0EAAC0B20328ECD304
:10F8E00001E011E03AE0DDE9700BA0EB0B0000FB5A
:10F8F0000AFA7298BAFBF0F00001A3F1010AB0FB1A
:10F90000FAF000EB081047E0DDE9670AA0EB0A0A0D
:10F91000BAF5406F8EBF08F101000120EB4617D801
:10F920003BF810E0F24502D2A0F1010A03E0401CCE
:10F93000C0B26628F4D34FEA083000F5805000FBCF
:10F940000AF8DFF828A80020D346E8FB0AB0400CEC
:10F95000DDF8C481A8EB0000401C1DE03BF810E07E
:10F96000F24502D2A0F1010A03E0401CC0B26628B1
:10F97000F4D34FEA083000F5005000FB0AF8DFF836
:10F98000ECA70020D346E8FB0AB0400CDDE9708A02
:10F99000A8EB0A084044801EDDF8B081B8F1010FE1
:10F9A00041D1DDF8D48141F2545A08FB0AF84FEAFC
:10F9B000183ABAF5805F88BF4FF4805A4FF00108BB
:10F9C000EB463BF818E0F24506D20DF1CC0A0AEB03
:10F9D000480838F802AC06E008F1010808F0FF0812
:10F9E000B8F1660FEDD30FFA84F836B218EB0604BF
:10F9F00017D04FEA0838B8FBF4F83603B6FBF4F436
:10FA0000A8EB040404FB0AF4E40A544588BF5446F6
:10FA100004EB4404769EC4F3D714002E0CBF20449C
:10FA2000001B083000094FF00008002975D0749CB5
:10FA3000641E8C4270DD01FB0324A1F1010808FB68
:10FA4000032801F1010A24B20AFB03230FFA88F804
:10FA50000FFA83FA35F914402B4635F9188035F939
:10FA60001A50012664F31F43A845A3BF68F30F0390
:10FA700065F30F07012565F30F03BCBF68F30F079C
:10FA800000256D951DB2002DBCBF002565F30F0349
:10FA90003DB2002DBCBF002565F30F070FFA83F8B8
:10FAA00004EB08054FEA043ABAFBF5FA4FEA0838C6
:10FAB000B8FBF5F5AAEB050841F6333E0FFA87FBD4
:10FAC00008FB0EFE0BFB0EFBBBFBF4F4240B0AFB46
:10FAD00004F4CDF8A8A104F50064DDF8B4A1240B6A
:10FAE000BAF1000F14BF69956B9540D06B94002557
:10FAF000AA46012E08BF002469D0022E7DD0DDE980
:10FB00006954651BB5F5406F9ABF0124EA4609F1B7
:10FB1000020473D9B8E000E02BE001FB032424B217
:10FB20004FF0010A0AFB032A35F914402B4635F938
:10FB30001A50022664F31F4365F30F07002CBCBF65
:10FB4000002464F31F43002DBCBF002464F30F079F
:10FB50001D140FFA87FA05EB0A042D03B5FBF4F523
:10FB60006A954FEA0A35B5FBF4F46B940024699466
:10FB7000BDE701FB0324A1F1010A24B20AFB032320
:10FB80000FFA83FA35F914402B4635F91AA00326EB
:10FB900064F31F436AF30F03002CBCBF002464F31B
:10FBA0001F43BAF1000FBCBF002464F30F031D1400
:10FBB0000FFA83FA05EB0A042D03B5FBF4F56A95F9
:10FBC0004FEA0A35B5FBF4F4699400248EE70DF58D
:10FBD000D27B01EB040E5BF824B0AEF1010E641C85
:10FBE0000BFB0EAAE4B25D44032CF0D3DDE96E4BAF
:10FBF000A4EB0B0404FB0AF401E00AE02EE0B4FBE2
:10FC0000F5F42501749C641EB5FBF4F404EB0914AF
:10FC100040E0DDE96A45651BB5F5406F8EBF09F12F
:10FC200001040124EA4615D83AF814B05D4501D222
:10FC3000651E03E0641CE4B2662CF5D34FEA093478
:10FC400004F58054DFF824956543CA460024E5FB9B
:10FC500009A4640C6F9D2C1B641C1BE03AF814B0C3
:10FC60005D4501D2651E03E0641CE4B2662CF5D349
:10FC70004FEA093404F50054DFF8F0946543CA46AE
:10FC80000024E5FB09A4640CDDE96E59A5EB090528
:10FC90002C44A41E012E3AD141F2545508FB05F51F
:10FCA0002E0BB6F5805F88BF4FF480560125E846DD
:10FCB00038F815904E4505D233AE06EB450535F8BC
:10FCC000026C03E06D1CEDB2662DF1D30FFA83F8E0
:10FCD0003DB218EB050308BF04F1080316D04FEA44
:10FCE0000837B7FBF3F72D03B5FBF3F3FB1A7343A8
:10FCF000DB0AB34288BF334603EB43036D9DC3F376
:10FD0000D713002D0CBF2344E31A08331C09012923
:10FD100008BF002A06D178998C4201D3814201D9CB
:10FD2000012177919CF86E109CF86D50CB0901F081
:10FD30007F024FEAD51C05F07F0113D0002B18BFBE
:10FD40001044BCF1000F12D0BCF1000F18BF0C44DE
:10FD50007A99A1F8B0007A98A0F8B24077987BB071
:10FD6000BDE8F08F904234BF0020801AE9E78C4252
:10FD700034BF0024641AEBE72DE9F04716460F461E
:10FD8000044603F00BFB8146F948857894F872002D
:10FD9000012804D194F8E500012818BF002503F0DC
:10FDA00009FB804603F00AFB0246F24894F898A04B
:10FDB0000068BAF1010F438A018A94F89A0000EBB7
:10FDC000400CCCEB401009EBC0004FF001094FF0A4
:10FDD000000C34D090F87A00012808BF84F87A909B
:10FDE000607800281CBF521E904208DA2078002854
:10FDF0001CBFA8F10102904201DA84F87AC0002DFC
:10FE0000D8BFBDE8F087BD420BDC481B401E8742CF
:10FE1000D8BFB54205DC581B401EB042A8BFBDE8A4
:10FE2000F08794F87A00012818BFBDE8F08784F8BD
:10FE3000E29084F8DEC084F8E5C0BDE8F087607821
:10FE400000281CBF521E904206D0207800281CBFFC
:10FE5000A8F101029042D0D184F87AC0AF4209DB08
:10FE6000481B401EB842A8BFAE4203DB581B401ED1
:10FE70008642C4DD84F87A90C1E72DE9F84F1D462B
:10FE800016460C46834603F089FA014694F89A0018
:10FE900000EB4002C2EB401001EBC003B54800226A
:10FEA000BBF1010F03D0BBF1080F26D043E000687F
:10FEB000162140F29C4A078AB0F818C07943B1FB7A
:10FEC000FCF11FFA81F9418A4FF0B40807FB0AF7E9
:10FED00001FB08F8408BB7FBFCFCB8FBF0F840F2E4
:10FEE000EC477943B1FBF0F087B21FFA8CF01FFAB0
:10FEF00088F81FFA8CFA00901DE0016840F6A11AFC
:10FF0000488A0F8BC0EB401C0CEB8018B1F81AC06C
:10FF1000098AB2FBF7F901FB0AF1B1FBF7F11FFA0D
:10FF200081FA40F241514843B8FBFCF8B0FBFCF0C9
:10FF30001FFA88F887B24E4534BF48463046A4F8C9
:10FF4000B00056458CBF50463046A4F8B000454539
:10FF500034BF40462846A4F8B200BD428CBF3846A4
:10FF60002846A4F8B2000120BBF1080F15D0BBF160
:10FF7000010F18BFBDE8F88F4E4522BF0099B1426E
:10FF8000454503D3BD4298BFBDE8F88F94F8E5100E
:10FF9000022918BFBDE8F88F1CE04E4528BFB245C6
:10FFA00004D3454524BFAF42BDE8F88F94F8E5106F
:10FFB00002290FD084F8E30093F8E310012918BF59
:10FFC000BDE8F88F84F8E20084F8DE2084F8E520AC
:10FFD000BDE8F88F84F8E20084F8DE2084F8E5209C
:10FFE00084F8E320BDE8F88F2DE9F74F86B014467A
:10FFF00003F0B8F9064603F0C7F9009003F0CEF914
:020000021000EC
:1000000001465C480068428A0492008A039094F892
:100010009A0000EB4002C2EB401001EBC00503F078
:10002000CDF9DFF84C8182460DF1040998F8030000
:10003000D8B10020FEF771FFDDE9060102AB2246D0
:10004000CDF80090FFF708F9BDF80800A4F8B0005B
:10005000BDF80400A4F8B20003F0B9F901287DD07E
:1000600003F0B5F9082879D092E096F83804002713
:1000700020B121460698FFF7EEFA0746B8F80800C7
:10008000B8F80410B0EB011F0DD298F8031051B965
:10009000401C80B2A8F808000009A8F80400DDE9B7
:1000A0000310FEF7A5FEB8F80A00B8F80610B0EB8A
:1000B000011F0DD298F8031051B9401C80B2A8F866
:1000C0000A000009A8F80600DDE90310FEF790FE1B
:1000D00096F838044FF0000BA0B9009890F8380457
:1000E00001280FD994F8E50003280BD1A8F808B02F
:1000F000A8F80AB0A8F804B0A8F806B0DDE9031023
:10010000FEF776FEDDE9060102AB2246CDF800904F
:10011000FFF7A2F896F8380420B1012808BF012F94
:100120000BD016E084F872B0BDF80800A4F8B00057
:10013000BDF80400A4F8B2000BE084F872B086F8B1
:1001400038B4BDF80800A4F8B000BDF80400A4F865
:10015000B2000E20A8F80400122000E00CE0A8F87D
:100160000600DDE90310FEF743FE75E74F09F29440
:10017000444200209842002003F02CF940B103F0E3
:1001800026F9BDF80430BDF808202146FFF775FEBA
:1001900095F8BB00032807BF2878002809B0BDE800
:1001A000F08F687800281CBFAAF101018842A4BF23
:1001B00009B0BDE8F08F94F8BB0001281CBF09B05E
:1001C000BDE8F08FB5F8B000A4F8B000B5F8B20003
:1001D000A4F8B20009B0BDE8F08F2DE9F05F044645
:1001E00003F0DCF801468848DFF820B2D0F8009030
:1001F0009BF800C0B9F81260B9F81A007200B2FB9F
:10020000F0F202EB0C031FFA83F89BF801309BF825
:1002100003B01A4497B264227243B2FBF0F594F82B
:100220009A00B9F810A000EB4002C2EB401001EBBD
:10023000C002B4F8B000B4F8B210BBF1000F19D08E
:10024000604538BF6046994238BF1946AAEB0C0298
:10025000A2F1010C8445B8BF604680B2F21A531E69
:100260008B42B8BF194689B2A4F8B000A4F8B21006
:10027000BDE8F09F94F898B0BBF1010F2AD194F833
:1002800001B0BBF1000F10D099F806E0AEF1010EFD
:10029000F3451CBF94F800B0BBF1000F05D099F8EE
:1002A0000790A9F10109CB450AD194F899E0DFF84C
:1002B00060B14FF005090BEB4E0B2BF8029C09E0E7
:1002C00094F899E0DFF848914FF0000B09EB4E09E4
:1002D00029F802BC40451ED294F8E500032819D144
:1002E00094F899904A4800EB490B3BF8020C05281A
:1002F00010D2B2F8B2904046B1EB0909B2F8B6108C
:1003000048BFC9F10009A94584BF4FF005092BF882
:10031000029C00E06046B9421ED294F8E510032921
:1003200019D194F899903A4901EB490B3BF8021C1A
:10033000052910D2B2F8B0903946B0EB0909B2F8ED
:10034000B40048BFC9F10009A94584BF4FF00509B1
:100350002BF8029C00E01946AAEB0808A8F1010955
:10036000814522DA94F8E50003281AD194F899809F
:10037000274800EB480838F8020C052811D2B2F8DB
:10038000B2C01FFA89F0B1EB0C0CB2F8B61048BF3E
:10039000CCF1000CAC4584BF4FF0050C28F802CC22
:1003A00003E0AAEB0C00401E80B2A6EB070CACF1F8
:1003B000010C8C45BFF658AF94F8E510032917D10E
:1003C00094F89970124901EB470737F8021C052988
:1003D0000ED2B2F8B0301FFA8CF1C31AB2F8B400E2
:1003E00048BF5B42AB4284BF052227F8022C3BE7A3
:1003F000F11A491E89B237E710B51446FFF7F4FD2C
:100400002046BDE81040E8E6984200204442002023
:10041000DC90002070B514460D46064602F0CAFF77
:100420008446D5E905202969002904BF002319461F
:100430000AD002EB820292004900B2FBF1F300EB1A
:1004400080008000B0FBF1F12380FF486180A0FBB9
:100450000332A0FB0110D208C00800FB0C2036F8C4
:100460001000A08070BD2DE9F0410446DDE90606CC
:10047000089F0D4600281CBF002081F8250002D0EF
:100480000020BDE8F081286820606868C4F80A0090
:1004900010686060908820818422194604F114005D
:1004A0000AF022F9A868C4F80E002869A061A8899A
:1004B000A082A88BA4F8740095F8240084F8DF00CB
:1004C00095F8260084F8E000012084F8DE0084F826
:1004D000E1703078401CC0B230700A2828BF01207B
:1004E000CED3BDE8F0812DE9FF5F1F4616460546D5
:1004F00002F038FFB0F902004FEAE00A02F06FFFA5
:10050000504502DD02F06BFF824600229346904682
:1005100091463046BE4221DCB0420CBF0146411E2E
:10052000CBB2B8420CBF0146411C01F0FF0C08F1F0
:1005300001011FFA81F835F9101051450ADD49B162
:1005400035F913309942A4BF35F91C30994201DBCB
:1005500082B203E0401C00B28742DDDA3C46B7427B
:1005600020DB0CBF2046601EC1B2BC420CBF20463F
:10057000601CC3B209F101001FFA80F935F91400BB
:1005800050450BDD50B135F911108842A4BF35F943
:100590001310884202DB1FFA84FB03E0601E04B2E2
:1005A000B442DEDA93450DD04FEA4802294601985D
:1005B0000AF0A4F801984FEA490205EB4B0100EB61
:1005C000480004E0B81B4000821C294601980AF04C
:1005D00095F808EB090004B080B2BDE8F09F2DE962
:1005E000F0479CB0844624988A464FF00008017872
:1005F00040784446CDF80080CDF80480CDF80880DE
:10060000CDF80C80CDF81080CDF81480CDF818808E
:10061000CDF81C80CDF82080CDF82480CDF828803E
:10062000CDF82C80CDF830804FEA8109CDF83480A8
:10063000CDF838801094119414941F4686001294BB
:100640001394159416941994179418941A944B466D
:10065000224669466046CDF83C801B94FFF743FF75
:100660000546334622460EA95046FFF73CFF044696
:10067000002109F10200854214DC0020002DC8BFD2
:10068000E9460FDD09EB400239F91030B2F902C03A
:10069000BCEB030248BFA3EB0C021144401C00B2A8
:1006A000A842EFDBA6EB08000022801CA042A4BFFA
:1006B0000020002CC8BF0DF138080FDD08EB400307
:1006C00038F910C0B3F90260B6EB0C0348BFACEBCD
:1006D00006031A44401C00B2A042EFDB88009100E0
:1006E000B0FBF5F0B1FBF4F10844400838841CB0CD
:1006F000BDE8F0877047704770470028DCBF0020D6
:1007000070474FF480714FEA002C00200B129CFBC5
:10071000F3F30A46991801EBD1714910531A48BFF7
:100720008B1A802B02DB401C6428EFD30812704721
:100730002DE9FF4F85B01F4616460D46002402F0F6
:1007400039FE0190B6F900E0B6F90200029028796E
:1007500003906A79E87995F806A0A446654666464E
:100760000090824229DC0398504521DC029902EB7B
:100770008203C1EB430303FB03FB019902FB010866
:10078000059931F918100A290EDD00EB8008CEEB2F
:10079000480808FB08F903FB08F809FB01CC0BFB30
:1007A000015508FB01660C44401C00B25045E4DDD5
:1007B000501C02B200988242D5DDDFF8908088FBA1
:1007C0000C104111A1EBE07188FB05204211A2EB56
:1007D000E07288FB06304311A3EBE0734CB10802D2
:1007E00011021A0290FBF4F091FBF4F192FBF4F287
:1007F00002E000200146024600FB01F302FB123238
:100800000844C0F1000C1412A0000CFB0CF1C0EB6A
:100810002120001241000029D8BF002019DD0D025F
:100820004FF480700021031295FBF3F302469818F1
:1008300000EBD0704010131A48BF831A802B02DBE4
:10084000491C6429EFD303E0CDCCCCCC1F85EB5100
:100850000012000200EBD070DCEB60010CEB6000DA
:10086000C0F100027C6148BF4942F960002AB8BF6C
:10087000524201EB8100400088FB0030C310A3EB23
:10088000E0703A61FF28C8BFFF2049115211FF29CB
:1008900088BFFF21FF2A88BFFF22002912BF002A3C
:1008A00001210A46002808BF012087F87D0087F84B
:1008B0007E1087F87F2009B0BDE8F08F2DE9F04168
:1008C00017460C46064602F075FD054602F076FD19
:1008D000014623786078002BCCBF5A1E0022A5F178
:1008E000010C6345B4BF5C1C64460028CCBF431EAA
:1008F0000023A1F1010C6045B4BF401C60464FF0DD
:10090000000C83420FDC1146A24208DC03FB0518F1
:10091000491C36F9188009B2C444A142F6DD591CBD
:100920000BB28342EFDDC7F81CC0BDE8F08170B5A3
:10093000044602F03FFD054602F040FD21780246E4
:1009400000291CBF681E814206D0607800281FBFA6
:10095000511E8842002070BD012070BD70B50D464B
:10096000044602F027FD064602F028FD2278012306
:100970000146002A1CBF701E824206D06078002803
:100980001EBF491E8842002000D11846002818BF0B
:1009900085F86730002070BD2DE9F007A0F1020A4C
:1009A000DDE90A54DDE90896079F4FF0000804EBE3
:1009B000400C8A45B2BFA3F800803CF804ACA3F811
:1009C00000A0431E8B42B2BFA7F800803CF8021C77
:1009D000398034F81010A9F80010411C91428EBFE4
:1009E000A6F80080BCF802103180801C90428EBFB7
:1009F000A5F80080BCF804002880BDE8F007704727
:100A00002DE9F0018A1ADDE90847DDE90565DDF821
:100A10001CC0994202BF20F832C0BDE8F001704707
:100A2000AB1BACEB0501A4EB0C05CB1A2EB2711A73
:100A300001EB41013C1B49000FB203EB4303A11B37
:100A40005B0001EB41011DB249000BB2794205EB9D
:100A50008101C3EB031421448C00002CC8BF891111
:100A600004DC890049420912494209B24C4203EBB5
:100A700084031DB24B1B002B03DD2B2463431B128D
:100A800005E06FF02A0463431B125B421BB26C103B
:100A900001EB45012B256943A6EB21210DB29E00F8
:100AA00000215F0106EB041607EB84174FF06C087A
:100AB00003FB08F304EBC40403EB041305EB450448
:100AC00006EB851607EBC51703EB841306EB0C2624
:100AD00007EB0C2703EB0C2346F30F2647F30F27F6
:100AE00043F30F2400EBC20320F832C05E80491CA0
:100AF0009F8089B2DC800429F4D3BDE8F0017047FF
:100B00002DE9FF4F03F1010885B01E4615468146C9
:100B10001146424532BF002709B0BDE8F08FB2460A
:100B2000881EA842B2BF3B4609EB410030F9043CA5
:100B30004A1EAA42B2BF3A4609EB410030F9022CE4
:100B400039F911C04C1C54458EBF384609EB4100A1
:100B5000B0F9020001F1020BB3458EBFBA4609EBB2
:100B6000410ABAF904A0CDF808C0CDE90032CDE9B8
:100B7000030A33462A460698FFF742FFA1B24145D1
:100B8000CDD309B0BDE8F08F30B48278037890F807
:100B900003C04478D21AACEB040C0B70D2B20CF048
:100BA000FF0483784FF0000C8B70052A26D209E0F1
:100BB00023B38D7883F001036D1E8D70521ED2B267
:100BC000052AF5D242784A70C078C870052C3CBF1F
:100BD00030BC7047BCF1000F01BF4878401C487022
:100BE0004FF0010C1FBFC878401EC8708CF0010C7C
:100BF000601EC4B2052CEDD230BC70470B785B1C74
:100C00000B700123DAE72DE9FF4FF5B01C46DDE953
:100C10008295074602F0D2FB064602F0CBFB8046E7
:100C200070A909F10400FFF7AFFF9DF8C00100288B
:100C300018BF401EC0B28DF8C0019DF8C211A8F1C6
:100C4000010291420CBF1146491CCAB28DF8C22163
:100C50009DF8C111002918BF491E8DF8C1119DF8DA
:100C6000C311731E99420CBF1946491C8DF8C3115C
:100C7000101A20709DF8C3019DF8C111E946401A71
:100C8000607028789DF8C0119DF8C141401AC6B225
:100C9000A878B5F90450001B00F0FF089DF8C301C7
:100CA000A04224BF4FF0000ADFF888B639D3CDF850
:100CB00088A1CDF88CA1CDF890A1CDF894A1CDF864
:100CC00098A1CDF89CA1CDF8A0A1CDF8A4A1CDF814
:100CD000A8A1CDF8ACA1CDF8B0A1CDF8B4A1CDF8C4
:100CE000B8A1CDF8BCA1DBF800009DF8C2319DF899
:100CF000C021C07962A9604307EB4000FFF700FF05
:100D00009DF8C1013822201AC0EBC00009EBC000D9
:100D100062A909F0F3FC601CC4B29DF8C301A042B3
:100D2000C5D2B700C8EBC808FCB209EBC80138222D
:100D3000769809F0E3FC6FF0020000EB86003A1DA4
:100D4000824218DD9DF8C0119DF8C231591A00EB9E
:100D5000880339F913309D4209DA002807DBB0EB2C
:100D6000810F04DCC4B204EB880339F91350401C32
:100D700000B28242EBDC9DF8C3119DF8C121002036
:100D8000891A58BF71AA0BD4C0EBC00304EB8303CC
:100D900039F8133022F81030401CC0B28142F3DA27
:100DA000CBB2002271A87799FFF7AAFE79B0BDE80F
:100DB000F08F2DE9F05F14460E46054602F0D2FA98
:100DC000DFF870A500F138072078DAF800206178A4
:100DD00094F805C0D27901FB0200385C00F03F08AE
:100DE000E079401C60458CBF4FF00009BDE8F09FE2
:100DF0002379A079401C984221D9DAF8001007EB3A
:100E0000030BC87900FB0CF20CFB003012F80B202E
:100E100002F03F02424518BF25F8109009D136F97B
:100E20001020B1F90C108A42CCBF25F8102025F80B
:100E30001090581CC3B2A079401C9842DDD80CF128
:100E4000010000F0FF0CE079401C6045D0D8BDE8FF
:100E5000F09F2DE9FF4F87B00E461598446802F0C9
:100E6000A9FA059002F0AAFA00210291079A0091CE
:100E7000019103910491116031800746220E4FF0D9
:100E80000009C4F307200599C846EA460692824243
:100E900024BF04F0FF0EC4F3074B3DD3F446E345F3
:100EA00035D3059A00FB02C3149A32F913400A2C79
:100EB0000EDB3288521C3280B84238BF07464045AC
:100EC00088BF80468C4538BF6146CC4588BFE14627
:100ED00000233AF91320A2420FDA0822082B09D284
:100EE0000AEB420535F8025C2AF81250521ED2B2C3
:100EF0009342F5D32AF8124003E05A1CD3B2092BCF
:100F0000E7D30CF1010202F0FF0CDC45C9D9401C0B
:100F1000069AC0B29042C1D9A9EB01000999401CC0
:100F200008700A99A8EB0700401C08700020079978
:100F30003AF91020401C0968C0B20A4407990928F0
:100F40000A60F4D30BB0BDE8F08F2DE9FF4F0546E2
:100F5000F948174697B0D0E90012CDE90E12D0E952
:100F60000212249ECDE91012D0E90412CDE912122A
:100F7000D0E90610CDE9141002F0F4F938300690EB
:100F800002F018FA044602F019FA09901898EB4991
:100F9000B0F9022000780490189890464378002019
:100FA00002900C91089011020D9109990A90491E26
:100FB0000591611E834682460B90814684460391CB
:100FC000002126F810100EA931F81CE00499714494
:100FD0000FFA81FE10A9CDF800E031F81C10194479
:100FE00009B2019101FB04E109B2079101990029BD
:100FF000A4BFDDF814E08E454EDB00990029A4BFA4
:10100000DDF80CE08E4547DB079935F911105A29B8
:10101000C4BF09F1010909F0FF0926F810100029E1
:1010200003DC012126F8101021B136F910E00D99EA
:10103000B1FBFEF14FF0010EBEEB112F07D2DDF830
:1010400028E00EF1010E0EF0FF0ECDF828E0DDF8DD
:1010500030E08E4588BF0C91DDF820E08E4538BF2A
:1010600008918B440299DDF82CE0491CC9B2029129
:1010700036F9101000917145C8BF0B91DDE9061ECD
:1010800011F80E1000291CBF0AF1010101F0FF0A3E
:10109000009941440FFA81F8401C0CF1010101F064
:1010A000FF0CC0B2BCF1040F8AD3029904297DD091
:1010B000032906BF0899ABEB0101CDF820B076D02B
:1010C00000214FF0000C26F810C00DF1480C3CF840
:1010D00011E0DDF810C0F4440FFA8CFE0DF1500C55
:1010E000CDF800E03CF811C09C440FFA8CFCCDF820
:1010F00004C00CFB04EC0FFA8CFCCDF81CC0DDF82E
:1011000004C0BCF1000FA4BFDDF814E0E6452CDB01
:10111000DDF800C0BCF1000FA4BFDDF80CE0E6452F
:1011200023DBDDF81CC035F91CC0BCF15A0FC4BF6D
:1011300009F1010909F0FF0926F810C0BCF1000F00
:10114000DCBF4FF0010C26F810C0DDE906CE1CF81C
:101150000EC0BCF1000F1CBF0AF1010C0CF0FF0A1D
:1011600036F810C0C4440FFA8CF8401C491CC9B2B0
:10117000C0B20429A5D31A9880F800A00B98104497
:1011800000B200900298002814BFBBFBF0F60026C6
:10119000009800281CBF4FEA0821B1FBF0F00002C4
:1011A000002E14BFB0FBF6F0002001E04DE052E04D
:1011B0000190462A7EDADDF810B0002003F1010A22
:1011C00003FB04B10FFA81FC35F91C10B2EB010EE0
:1011D00048BFA1EB020EBEF10A0F3EDA012B16D476
:1011E000ACEB040E35F91EE0BEF1140F0FDA0CEB78
:1011F000040E35F91EE0CDF808E0BEEB010E44BF49
:10120000DDF808E0A1EB0E0EBEF10A0F16DADDF8EC
:1012100024E0F24514DA0CEB040E35F91EE0BEF1C1
:10122000140F0DDAACEB040C35F91CE0BEEB010C2D
:1012300048BFA1EB0E0CBCF10A0F01DB401CC0B291
:10124000ABF1010101F0FF0BBAE70899ABEB010C20
:101250000C99ACEB0101089132E70499491C43E079
:1012600003FB04B10FFA81FC35F91C10B2EB010E3F
:1012700048BFA1EB020EBEF10A0F39DA012B16D4DA
:10128000ACEB040E35F91EE0BEF1140F0FDA0CEBD7
:10129000040E35F91EE0CDF808E0BEEB010E44BFA8
:1012A000DDF808E0A1EB0E0EBEF10A0F18DADDF84A
:1012B00024E000E023E0F24514DA0CEB040E35F9EB
:1012C0001EE0BEF1140F0DDAACEB040C35F91CE096
:1012D000BEEB010C48BFA1EB0E0CBCF10A0F01DB09
:1012E000401CC0B20BF1010101F0FF0BA345B7DBBD
:1012F000022888BF022023D001D987F876000899F8
:10130000009A4FEA1620A7F84A203865A7F84880C7
:1013100001984FEA5121C7E9151087F874900A988F
:1013200087F875001898008CA7F862001BB0BDE81C
:10133000F08F0000984200206CE90100F0490200A3
:101340000498A4F103018842C8BF0120D7DDD4E787
:101350002DE9FF4F81B014460F460546FE484FF079
:1013600000080068B0F92CB0B0F92E10009190F888
:10137000BFA0B5F9026002F01DF8814602F01EF828
:101380000346B34524DDB4F900000028C4BFB4F916
:101390000210002903DD0844304400B210E0B4F923
:1013A00004100029C1BFB4F90620002A881830446F
:1013B00005DC6288314410440844E188084400B2E6
:1013C0000099884204DAA88B504538BF4FF00108D5
:1013D0003046002234F812100844511C0AB200B200
:1013E000042AF7DB002287F86820B8F1000F22D02A
:1013F0000499491C90FBF1F081B2687810B35B1E30
:10140000984204BF95F800C0BCF1000F07D0984285
:1014100022D195F800C0A9F10109CC451CD10320C7
:1014200087F86800002034F91030B6EB430F1DDA5E
:1014300087F868201EE0A98900291CBF90FBF1F005
:1014400081B217E095F800C0BCF1000F1CBFA9F1F4
:10145000010AD445D3D1E2E7002818BF984209DA3F
:101460002878002808BF012004D1D9E7401C00B229
:101470000428D8DBA7F85C1005B04046BDE8F08F23
:101480002DE9FF4F85B00C4606460025DDF8489053
:1014900001F090FF039001F091FF029096F8008018
:1014A0007778B68901F09BFFB4F90020B4F90210F7
:1014B00001911144B4F90430B4F9062000924010AF
:1014C0001A449142CCBF11B209B2B4F908C0B4F9C0
:1014D0000EA0B4F90A30B4F90C200CEB0A0B03EBA4
:1014E000020EF345CCBF0FFA8BFB0FFA8EFB3FB910
:1014F000DDF804E08645C4BF00F1010EA4F800E069
:10150000DDF808E0AEF1010E774505D1B4F90070C1
:101510008742C4BF471C6780B8F1000F04D1009F09
:101520008742C4BF471CA780039F7F1EB84505D1D3
:10153000B4F904708742C4BF471CE780B4F9047053
:101540008742C4BFB4F9068080451CDD8445BEBF18
:101550008342B4F90030834206DB8245BEBF82423B
:10156000B4F90220824200DA0125052E20D2079824
:10157000401CB0421CD1594522DCB9F1010F1FD9E2
:101580000898E8B920E0B4F900808045C4BFB4F9F8
:1015900002808045E9DD8445BCBF82428742E3DBAF
:1015A0008342BEBF8245B4F906208242DCDBDCE721
:1015B000594500DD25B1B9F1010F01D9089818B1DD
:1015C00009B00020BDE8F08F09B00120BDE8F08F20
:1015D0002DE9F04186B014460F468046002501F003
:1015E000C1FE064602A8009001AB2246394640469D
:1015F000FFF7ABFC307D002804BF96F82E000028D2
:1016000007D19DF8043002AA21463846FFF7A0FE14
:101610000546002084F85E5084F8650006B0BDE8F9
:10162000F08170B515460C4601F09CFE0146002085
:101630000A7D002A06BF097B002970BDA1891E29E9
:1016400081BF95F87E104B29E18B072906D895F8C4
:101650007E10642986BFE18B062970BD012070BD14
:101660002DE9F74FAEB09246074601F083FE2B906E
:1016700001F078FE259000208DF890000646054682
:10168000BAF1000FC8BF4FF0010B40F3EA802F986A
:1016900005EB850100EBC10494F82500012840F01A
:1016A000DB80842101A809F024F8002022902390F7
:1016B00001A84FF000092A9001F054FE804626A8A8
:1016C00000902CAB214638462A9AFFF73EFC98F84A
:1016D0001400002804BF98F82E00002807D19DF8B8
:1016E000B03026AA20462A99FFF732FE8146002014
:1016F0008DF862908DF8690001F05CFE0346D4E934
:101700000401A269002804BF002108460AD001EBA9
:10171000810189004000B1FBF0F102EB82029200EE
:10172000B2FBF0F0ADF888100C4AADF88A00A2FBCD
:1017300001C1A2FB0020C908C00800FB031101ABD6
:1017400037F81100ADF88C0022AA21463846FEF782
:10175000EFFF01F007FE03E098420020CDCCCCCC97
:10176000017D4FF00009002904BF007B002811D142
:10177000A0891E2881BF9DF882004B28E08B072896
:1017800006D89DF88200642884BFE08B062801D922
:101790004FF00109B9F1000F1CBF259880F830B057
:1017A00001F008FE804601F009FE0146207800287D
:1017B0001CBFA8F10102904206D0607800281EBF2D
:1017C000491E8842002000D15846002818BF8DF8D5
:1017D0006BB09DF89000842200EB4001C1EB4011FA
:1017E0002B9800EBC1082068C8F800006068C8F8B2
:1017F0000A002298C8F80400BDF88C00A8F8080078
:1018000001A908F1140008F06FFFA068C8F80E00E5
:101810002069C8F81800A089A8F81400A08BA8F8BF
:10182000740094F8240088F8DF0094F8260088F803
:10183000E00088F8DEB088F8E1909DF89000401C48
:10184000C0B28DF890000A282CBF0120002040B9BA
:10185000A089B04288BF0646681C05B25545FFF610
:1018600016AF259886809DF8900031B0BDE8F08FC6
:10187000F0B5ADF2B44D0F46064601F073FD0446D7
:1018800001F082FD05464FF49661684608F031FF8D
:10189000207D012805D195F82A203146384607F0E9
:1018A000D0FB6A463946304604F09AF884F828009E
:1018B000024669463046FFF7D3FE0546207D0128E3
:1018C00003D12946304608F05CF801F0E7FD002816
:1018D00006BF002084F83E040A2D04D22946304673
:1018E00001F0C6FB054684F829500DF2B44DF0BD59
:1018F000FD4800787047FD490968B1F8B410884385
:10190000F949C04388607047F7488068C043704712
:101910000346F64800688279C0795200424301EBE1
:10192000011000EB4110F24901EB4010194608F09C
:10193000E5BEF0494FF6FF7221F8202001EB80014F
:101940004A80ED4A00211154921C1154EB4A42F88E
:10195000301002EBC0025160E94A1154D21D02F866
:10196000101002EB40004170704700B50020FFF7F7
:10197000E0FF0120FFF7DDFFDB490020087000BD1C
:10198000DE4A002102EBC0035B682E2B84BF52F8B5
:101990003020202A09D9DB4A02EB40035B78042B74
:1019A00022BF12F810000428012108467047F0B445
:1019B000D049D54D31F82210AB5C401A00B2002856
:1019C00008BF1946B8BF0121C8BF02214FF0010668
:1019D000CC4CDFF828C313B38B425CF832300BD108
:1019E0000028B8BF404218444CF8320014F81200E6
:1019F000401C04F812000EE00CEBC20700287B60CC
:101A0000B8BF40424CF8320004EB420314F8120015
:101A1000587004F81260A954F0BC012070470028E7
:101A2000B8BF40424CF83200F3E72DE9FF4FAF4812
:101A30009FB0AF4A0068837990F80790002000902B
:101A400001900290049003900590069007900990F1
:101A500008900A900B900C900E900D900F901090A3
:101A60001190139012901490159016901890179052
:101A700019901A901B901D90A9F101001FFA80FA8D
:101A80001C9001EB011000EB411002EB401B09B16F
:101A9000012970D000224FF0010E00263346354652
:101AA0003446B446724598BF0EAF24D81D995145AF
:101AB0001DD802FB0910DDF87C8038F810803BF857
:101AC0001000A8EB000000B232280CDD2DF8110048
:101AD00000FB015500FB0244761C27F8120003446A
:101AE0006045C8BF8446481C81B25145E1D9501CAD
:101AF00082B27245DAD91C9A00210120012AC8BF9E
:101B0000E84615DD08EB400738F9102037F902AC3C
:101B10005245A2BFB7F90270BA42322A03DD801CD7
:101B2000491C80B2C9B2401C1C9A80B29042E9DBC9
:101B3000BDF90000BDF902209042A8BF3228C4BF01
:101B4000481CC1B2684600EB490030F9022C30F95C
:101B5000040C8242A8BF322AC4BF481CC1B2002E66
:101B600018BFBCF1320F01DD01290AD023B00020DB
:101B7000BDE8F08FFFE7981E82B2581E1FFA80FE64
:101B80008BE705EB85004000B0FBF3F004EB84012C
:101B90004900219AB1FBF3F110802298018023B013
:101BA0000120BDE8F08F2DE9F04F89B04068002496
:101BB00006AB05AA21460090FFF737FF054603ABA9
:101BC00004AA01210098FFF730FFDFF838A1079041
:101BD0000AF104092800494FA9F10F08A3464FF064
:101BE000010608F1040535D02878002853D198F86B
:101BF0000000002808BF88F8006022D00022BDF84D
:101C00001810BDF81400FFF7D2FE00284FF00000B6
